:020000040800F2
:100000000000022009170C088D170C083DC40608D3
:100010008D170C088D170C088D170C0800000000B8
:100020000000000000000000000000008D170C0818
:100030008D170C08000000008D170C083D4A0508BC
:100040008D170C088D170C088D170C088D170C08D0
:100050008D170C088D170C08AD2B0508B12B050862
:10006000B52B0508B92B0508BD2B0508754D0408EF
:10007000894D04089D4D0408B14D0408C54D040880
:10008000D94D0408ED4D04088D170C088D170C0888
:100090008D170C088D170C088D170C08C12B05083F
:1000A0008D170C088D170C088D170C08F5570408D0
:1000B000095804081D58040831580408B5400408BC
:1000C000A9400408E5400408D94004088D170C082D
:1000D0008D170C08B9620408C5620408D1620408CF
:1000E000C52B05088D170C08000000006D5804088A
:1000F000BD580408E558040859580408014E04087E
:100100008D170C08AD9B0408455804088D170C0882
:10011000DD6204088D170C088D170C0829B004083F
:10012000154E0408294E04083D4E0408514E04089B
:10013000654E04088D170C088D170C088D170C08D8
:1001400000000000000000000000000000000000AF
:10015000794E04088D4E0408A14E0408E962040893
:10016000194104080D4104088D170C088D170C085F
:100170008D170C088D170C088D170C080000000057
:100180008D170C088D170C08F5620408016304082C
:100190008D170C088D170C088D170C088D170C087F
:1001A0008D170C088D170C088D170C088D170C086F
:1001B0008D170C088D170C088D170C088D170C085F
:1001C0008D170C088D170C088D170C088D170C084F
:1001D0008D170C08DD9B04088D170C088D170C0873
:1001E0008D170C088D170C088D170C088D170C082F
:1001F0008D170C088D170C088D170C088D170C081F
:100200008D170C088D170C088D170C088D170C080E
:100210008158040895580408A95804088D170C083B
:100220008D170C088D170C088D170C0800000000A6
:10023000B19B04088D170C08000000008D170C08F6
:100240008D170C088D170C088D170C088D170C08CE
:100250008D170C088D170C088D170C088D170C08BE
:100260008D170C088D170C088D170C088D170C08AE
:100270008D170C088D170C088D170C080000000056
:100280008D170C08000000008D170C0800000000FE
:08029000000000008D170C08AE
:08029800B0060C00010000009B
:1002A00030AB0124020100000200140050AB012415
:1002B000020200000200140070AB0124020A0000D8
:1002C0000200140090AB012402030000040014009B
:1002D000B0AB01240208000004001400D0AB0124DC
:1002E000010B000000017700F0AB0124010C0000BD
:1002F0000001760010AC012401100000000176001E
:1003000030AC0124010D01000001770050AC012444
:10031000011200000001760070AC012401140000FD
:1003200000001E0090AC0124011A000000000D0026
:10033000B0AC0124011B000000002C00D0AC012453
:100340000115000000000C00F0AC012401160000B3
:1003500000000C0010AD0124011C000000000E0084
:1003600030AD0124011D000000001E0050AD01242D
:100370000117000000000C0070AD012401180000FE
:1003800000000E0090AD01240119000000000C00D7
:10039000B0AD0124011F000000000C00D0AD01240D
:1003A0000120000000000C00F0AD01240129010033
:1003B0000001180010AE01240121000000014800D6
:1003C00030AE0124012200000001490050AE01249A
:1003D0000123000000014A0070AE01240124000046
:1003E00000014B0090AE01240125000000014C00EB
:1003F000B0AE01240126000000014D00D0AE012462
:100400000127000000014E00F0AE01240128000089
:1004100000014F0010AF0124012C00000000290052
:1004200030AF0124012D01000000290050AF01244C
:10043000012E01000000700070AF012401300000A7
:100440000000310090AF0124012F01000000520094
:10045000B0AF01240131010000012800D0AF012418
:100460000132010000012800F0AF01240135000035
:1004700000003C0010B00124013800000000200002
:020000040804EE
:10000000836B5A6D12F0500F5A6D1AD1196842F471
:1000100000725A650A6812F0080FCA6816D012F406
:10002000406F15D1CA68920412D45A6D22F48072BE
:100030005A655A6DD1040BD45A6D42F001025A65CB
:100040007047D20604D4DB6CDB6C18479007ECD009
:10005000704700BF704700BF836B5A6D42F040028B
:100060005A659A6D42F004029A6570473649024615
:1000700003688B4233D01831591AB1FA81F149091A
:1000800069BB324883423ED0183083423ED018309C
:10009000834234D0183083423BD0183083423ED064
:1000A000183083422AD000F55670834235D0284953
:1000B0008B4231D018318B4234D018318B4234D03E
:1000C00018318B4234D018318B4234D018318B42E6
:1000D00034D018318B4234D023F0FF0011E0DBB272
:1000E0001C491D48103BA1FB031310B41B091B4CFA
:1000F000E15C5DF8044BC2E916017047162118480F
:10010000D1659065704710211348F9E71621124810
:10011000F6E706211248F3E706211248F0E710211E
:100120000F48EDE710210F48EAE716210D48E7E7F1
:1001300000210D48E4E706210B48E1E710210A48B9
:10014000DEE716210848DBE71000024040000240CD
:1001500028040240ABAAAAAA0000024090A10C0801
:1001600004000240000402400404024002685549B1
:1001700038B5554B554D564CAA4218BF9A420CBF44
:10018000012300238A4208BF43F001033031A24219
:1001900008BF43F0010330348A4208BF43F0010333
:1001A0003031A24208BF43F0010330348A4208BF15
:1001B00043F0010301F55C71A24208BF43F0010363
:1001C00004F55C748A4208BF43F001033031A24257
:1001D00008BF43F0010330348A4208BF43F00103F3
:1001E0003031A24208BF43F0010330348A4208BFD5
:1001F00043F001033031A24208BF43F001038A42B9
:1002000008BF43F0010313B9324B9A4208D10423CB
:1002100080F83530136823F001031360002038BDE7
:100220002D4B2E4D1168AA4218BF9A422C4C21F03A
:100230000E0105F13C050CBF012300231160A24211
:1002400008BF43F0010311682834AA4208BF43F0F5
:10025000010321F00101A24208BF43F0010314345D
:100260001160A24208BF43F001031E498A4208BF41
:1002700043F0010313B91C4B9A4217D10123856D3A
:10028000D0E91714226801F01F0122F480728B401C
:1002900022606B60C36ED0E91921516033B11A68D6
:1002A000D0E91C1422F480721A604C6001210022F3
:1002B000036D80F8351080F83420002BAED09847BD
:1002C000ACE700BF4000024010000240280002409E
:1002D00058000240B80402401C5402580854025806
:1002E0003054025880540258945402580168002235
:1002F0000B6880F842205A0410B40ED50B6823F422
:1003000080430B6090F84130292B10D090F8413099
:100310002A2B24D05DF8044B70471B04F2D50B68E0
:1003200023F400430B6090F84130292BEED12822B2
:10033000212380F841200022036390F841300C68AB
:1003400003F02803282B14BF6FF0F2036FF0420371
:1003500023405DF8044B0B6080F840207047282252
:10036000222380F841200022036390F841300C687A
:1003700003F02803282B14BF6FF0F4036FF044033D
:1003800023405DF8044B0B6080F84020704700BFAD
:100390000023202210B4174C4363C462036380F827
:1003A000412080F842304B07026811D5526A436AF7
:1003B0001A70436A028D013343624AB1438D013A98
:1003C000013B02859BB24385436C43F004034364C5
:1003D0000368102490F84120002190F841201A6809
:1003E00022F0FE021A60DC615DF8044B80F84010D8
:1003F000704700BF0000FFFF70B5574B002590F815
:100400004120044680F84250283AC3624585436C37
:10041000022A41EA0301036841642FD890F8411091
:1004200090F84120282001F0280102F02802282914
:1004300014BFF6214621282A1A680CBFC9436FF061
:10044000F6010A4045491A6084F84100A06B226B0E
:10045000616318B1112A42D0212A40D0E06B18B153
:10046000122A51D0222A4FD094F84130602B4FF0FD
:1004700000032DD0236384F8403070BD90F84120F4
:1004800090F841201A6822F0FE021A609A699207D9
:1004900000D59D629A69D60703D49A6942F0010299
:1004A0009A6194F84120602A10D0202284F84120DB
:1004B0009A6995060AD59A69D00605D51022DA619F
:1004C000626C42F0040262642022DA610021BDE71E
:1004D000202284F8403084F84120236370BD1A68DC
:1004E00051042CD490F83530012BBDD000221C4B88
:1004F000036584F8402090F83520022A24D0802219
:100500004265BDE8704018471A68120403D51A689E
:1005100022F400421A6090F83530012BA4D000225A
:100520000F4B036584F8402090F83520022AE6D16D
:10053000FFF71CFE0028A0D0E06B036DE1E71A680E
:1005400022F480421A60CDE7FFF710FE002894D015
:10055000A06B036DD5E700BF0000FFFFDD050408B9
:100560002D09040803689A69196810B4D40528D5C0
:100570000C0606D4416C11F00B0F1FD15DF8044B33
:100580007047416C4FF4807441F0010141645105A2
:10059000DC6120D5416C4FF48064920541F0080184
:1005A0004164DC61E6D5426C4FF4007142F0020216
:1005B0004264D961416C11F00B0FDFD05DF8044B40
:1005C0001AE7540502D50906E4D4D3E79405D1D53A
:1005D0000906E8D4CEE79205E5D4CBE7F8B590F864
:1005E00040300D46C16A012B00F008810123AE06A0
:1005F000044680F8403001D5900656D4EB0619D554
:10060000D70617D5638D9BB2002B40F0F98094F884
:100610004130B1F1007FDBB240F0D580282B40F0B3
:10062000D28029462046FFF7B3FE0023184684F8FF
:100630004030F8BD68071AD42F0701D516074AD4F1
:10064000A807F2D59307F0D5638D9BB2002B00F07D
:10065000FA80616A236811F8010B228D9862638D1C
:10066000013A6162013B22859BB26385DDE7530756
:10067000E2D5638D9BB26BB12268636A526A1A70CD
:10068000638D606A228D013B0130013A9BB260624A
:1006900022856385638D9BB2002BC6D111F5803F07
:1006A000C3D02046FFF722FEBFE723682021186849
:1006B000E66A94F84120D961213A092A1ED8DFE878
:1006C00012F0C70015001D001D001D001D001D00BB
:1006D000F000C700150094F84130226803F02803A9
:1006E000282B00F0C5800823D3619EE794F84120B1
:1006F0001A6822F0FC021A60222222635A68894991
:1007000042F400425A605A680A405A609A69910756
:1007100001D500229A629A69D20703D49A6942F0FD
:1007200001029A6147047BD51A6822F480421A605C
:10073000A26B1AB111684A6892B262856A070BD53A
:100740005A6A25F00405636A1A70636A01336362AA
:10075000238D002B40F08580638D9BB21BB1636CB1
:1007600043F004036364EB061AD5C70618D5638DFE
:100770009BB2002B40F0AA8094F84130282B03D183
:10078000B6F1007F00F0C98094F8413016F5803F43
:100790002268DBB202D0292B00F0AD801023D36198
:1007A000002384F84230666C6363002E40F084803E
:1007B000E36A5D4DAB423DD194F84130202384F88B
:1007C0004130266331E794F841202368292A4FF00D
:1007D0001002DA617FF429AF11F5803F3FF425AFB5
:1007E0009A69960701D500229A629A69D5073FF562
:1007F00058AF9A6942F001029A6152E70220F8BDAF
:1008000023681022DA61636C43F00403636431F0FF
:1008100080737FF40AAF616C2046FFF7EDFD04E7BB
:1008200001048BD51A6822F400421A60E26B002A98
:1008300080D183E72046FFF759FD2023E56284F845
:1008400041302663F1E631F080737FF4EEAE28E7A5
:1008500094F841201A6822F0FA021A6021222263D9
:100860004CE7013B2385638D013B9BB2638573E7B6
:10087000E1689369022990699368D56836D1C3F31A
:10088000C21383EA104313F006032FD1A16C013188
:10089000A164A16C02297FF4C8AE0821A364D161D0
:1008A000C3E694F8412094F841201A6822F0FE0231
:1008B0001A600022226321E7616C2046FFF79CFD4D
:1008C00094F84130282B7FF4B0AEAAE623681022BA
:1008D000DA61636C43F00403636436F080737FF481
:1008E0005FAF616C2046FFF787FD59E7136823F07F
:1008F000B803136099E61023D3619369980701D573
:10090000002393629369D90703D4936943F00103E9
:1009100093612046FFF7EAFC42E729462046FFF7AD
:1009200037FD3DE700E800FE0000FFFF836B9A6B98
:100930000AB100211165DA6B0AB10021116593F843
:100940004120602A05D000221A63002283F840204B
:1009500070470022202183F841101A63002283F897
:1009600040207047016870B4CC072DD5914A1369B7
:10097000926A03F03803102B00F0E180182B00F08E
:10098000D9804368B3F5803F00F00581002B00F06B
:100990005A81B3F5A02F874B1A6800F0678222F4C2
:1009A00080321A601A6822F480221A60824B41F267
:1009B000883C804C1D6804E01A68521B624500F2B6
:1009C0003F8122689603F7D58A0768D4CD0631D5D2
:1009D000784A1369926A03F03803082B00F0C0804C
:1009E000182B00F0B880C369724C002B00F05F81B7
:1009F0002268714B42F0800222601D6804E01A6890
:100A0000521B022A00F21C812268D205F7D56B4BDB
:100A1000026A1D6841F20303B3EB154FC0F0448234
:100A20006368202A23F0F8430CBF43F0804343EA75
:100A3000826363600D0713D543695E4C002B00F0A1
:100A40001881626F5C4B42F0010262671D6804E02E
:100A50001A68521B022A00F2F380626F9207F7D5E0
:100A60008C0613D58369534C002B00F0118122684A
:100A7000514B42F4805222601D6804E01A68521BF8
:100A8000022A00F2DD8022689204F7D5490700F1BE
:100A90008880436A002B40F0BC80002059E0454A22
:100AA0001369926A13F038032BD1424AC368126863
:100AB000520701D5002B4BD03E4C226822F0190280
:100AC0001A433D4B22601D6804E01A68521B022A3B
:100AD00000F2B68022685607F7D5384B02691D68C8
:100AE00041F20303B3EB154F6368C0F0028123F4B6
:100AF0007C33402A0CBF43F4003343EA0233636083
:100B000064E7182B00F0F180C3682A4C002B00F03A
:100B1000DD80226822F019021A43274B22601D68EB
:100B200004E01A68521B022A00F28A8022685207E7
:100B3000F7D5D2E702F00302022A7FF422AF1D4B61
:100B40001B689B037FF540AF4368002B7FF43CAFED
:100B5000012070BC704702F00302012A7FF443AF0A
:100B6000144B1B68DC0502D5C369802BF0D1134CF4
:100B700041F20303026A2468B3EB144FC0F0BF8054
:100B8000202A00F09E810B4C636823F0F84343EA6F
:100B9000826363604EE7074A136843F4803313604F
:100BA00004E70749044B0A6842F480720A601C6833
:100BB0000CE000BF00440258002E00240010005C2E
:100BC000004802581A68121B642A39D80A68D505E9
:100BD000F8D58268012A00F06E81002A00F04E816B
:100BE000052A9F4A116F00F0748121F001011167FD
:100BF000116F21F0040111671D6841F28834984992
:100C000003E01A68521BA2421AD80A6F9207F8D55D
:100C10003FE793490A6902F03802182A00F0D580AC
:100C20000A68022B8F4B22F080720A606FD018681E
:100C30000A6892017FF531AF1A68121A022AF7D9B1
:100C4000032070BC7047864C41F28835854B226882
:100C500022F480322260226822F4802222601E6800
:100C600003E01A68921BAA42EAD822689203F8D4D9
:100C7000AAE6626F7B4B22F0010262671D6803E007
:100C80001A68521B022ADBD8626F9607F8D4E7E68F
:100C90002268744B22F4805222601D6803E01A68B7
:100CA000521B022ACCD822689604F8D4EEE62268B9
:100CB0006C4B22F0800222601D6803E01A68521B10
:100CC000022ABDD82268D605F8D4B3E62268654B5F
:100CD00022F0010222601D6803E01A68521B022AFA
:100CE000AED822685607F8D470E694077FF40CAFAC
:100CF000DBE623F0FE4343EA0263636066E6584C9A
:100D0000E36823F07C5343EA0263E36092E61C68E5
:100D100003E01A68121B022A92D80A689501F8D4D7
:100D20008C6A514A2240846A2243C46A42EA04120D
:100D30008A62D0E90D24013A013C5202240492B2A5
:100D400004F4FE042243046B013CC4F30804224370
:100D5000C46B013C240604F0FE4422430A63CA6AC1
:100D600022F00102CA624A6B846C6FF3CF0242EA3E
:100D7000C4024A63CA6A046C22F00C022243384C53
:100D8000CA62CA6A406C22F002020243CA62CA6A9C
:100D900042F48032CA62CA6A42F40032CA62CA6A43
:100DA00042F48022CA62CA6A42F00102CA620A6838
:100DB00042F080720A601968226890013FF56DAEBA
:100DC0001A68521A022AF7D93AE7012B8A6A0D6B80
:100DD0003FF4BEAE02F00303846AA3427FF4B8AED0
:100DE000C2F30512C36A9A427FF4B2AE036BC5F335
:100DF0000802013B9A427FF4ABAE436BC5F3462237
:100E0000013B9A427FF4A4AE836BC5F30642013BDB
:100E10009A427FF49DAEC36BC5F30665013B9D42CC
:100E20007FF496AE4B6B816CC3F3CC0399423FF4D5
:100E300034AE0B480B4BC26A22F00102C2621A6840
:100E400018688242FCD0064A536B6FF3CF0343EA23
:100E5000C1035363D36A43F00103D3621DE600BFAD
:100E600000440258002E00240CFCFFFF42F48022B4
:100E70001A601A6842F480321A6097E5194941F203
:100E800088350A6F22F001020A670A6F22F0040215
:100E90000A671C6804E01A68121BAA423FF6D0AE2B
:100EA0000A6F9607F7D4F4E5E36823F07C5343EA2E
:100EB0000263E360BEE50B490A6F42F001020A6774
:100EC0009AE6084A536823F0F84343F0804353609E
:100ED000B0E541F004011167116F41F001011167A4
:100EE0008AE600BF00440258334B30B4996A9C6ACA
:100EF000DD6A14F47C7F5A6BC4F3051036D0C2F35C
:100F0000CC0205F0010501F0030107EE900A05FB94
:100F100002F20129B8EEE77A06EE902AFAEEE96AC3
:100F200002D0022942D019B3DFED247A87EE876A16
:100F30001B6BC3F3080307EE903AF7EE005AF8EE86
:100F4000E77A77EEA67A77EEA57A67EE867A1A4B7D
:100F50001B6BC3F34623013307EE103AF8EEC76A62
:100F600087EEA67AFCEEC77A17EE900A30BC70477F
:100F70001A6892061DD51968F7EE005A104A1B6BC5
:100F8000C1F3C101C3F30803CA4007EE903A06EE6D
:100F9000102AF8EEE77AB8EEC66A77EEA66AC6EED1
:100FA000077A36EEA57A67EE877AD0E7DFED057A25
:100FB000BCE7DFED057AB9E7004402580024744A23
:100FC0000090D00320BCBE4B0024744C474A70B440
:100FD000946A956AD66A15F07C7FC5F30553516C07
:100FE0005BD0C1F3CC01C6F3002604F0030407EE86
:100FF000903A06FB01F1012CB8EEE77A06EE901A62
:10100000FAEEE96A03D0022C6AD0002C4AD0DFED58
:10101000387A87EE876A136CC3F3080307EE903AB9
:10102000F7EE005AF8EEE77A77EEA67A77EEA57A31
:1010300067EE867A2D4AB7EE006A136CC3F3462337
:1010400007EE103AB8EEC77A70BC37EE067AC7EEF4
:10105000876AFCEEE66AC0ED006A136CC3F30643D0
:1010600007EE103AB8EEC77A37EE067AC7EE876A0F
:10107000FCEEE66AC0ED016A136CC3F3066306EE8C
:10108000903AF8EEE66A76EE866A87EEA67AFCEE8D
:10109000C77A17EE903A8360704770BCC0E900339E
:1010A0008360704713689B061DD51468F7EE005ADD
:1010B000136C1049C4F3C102C3F30803D14007EE17
:1010C000903A06EE101AF8EEE77AB8EEC66A77EEB6
:1010D000A66AC6EE077A36EEA57A67EE877AA9E7A2
:1010E000DFED057A95E7DFED057A92E700440258D7
:1010F0000024744A0090D00320BCBE4B0024744CE2
:10110000836A1A0710B406D50168846B4A6822F412
:10111000004222434A60DC0706D50168C46A4A6877
:1011200022F4003222434A60990706D50168046B15
:101130004A6822F4803222434A605A0706D5016881
:10114000446B4A6822F4802222434A60DC0606D5BA
:101150000168C46B8A6822F4805222438A6099062F
:1011600006D50168046C8A6822F4005222438A6022
:101170005A060AD50168446C4A68B4F5801F22F407
:10118000801242EA04024A600BD01B0606D50268B0
:10119000C16C536823F400230B4353605DF8044B88
:1011A00070474A68846C22F4C00222434A60ECE72C
:1011B0000022836BA3F85E20704700BF124B41F200
:1011C000883C124A01461B68A2FB03235B0A0CFB06
:1011D00003F33BB14A6B12F0450F01D0920404D5E2
:1011E000013BF7D14FF0004070474B6B5B0707D4D2
:1011F000486B10F0010014BF0123054B8B6370474F
:10120000042318468B63704700000024D34D6210FE
:10121000C5002000036941681F2B70B431D9A3F1C8
:10122000200520224C68AA40224228D08269107CE6
:10123000022836D054681F2BD2681B485668226992
:101240001A4DC2F3032200EB8202926815F802C025
:10125000256856F80C2022F0010246F80C2062792D
:1012600000EB4200EA68008D00F4F05022EA000230
:10127000EA6010D9A3F1200220239340CB6070BC18
:10128000704720220C689A402242F8D08269107C74
:101290000228CFD105E0202202FA03F370BC8B6054
:1012A000704700201074C5E790A10C0840A30C08FB
:1012B000D0E907239A423CBFC1685218D01A704740
:1012C000D0E9092300699A4238BF12180138D31AAD
:1012D000C01A7047D0E90902101AB0FA80F040092C
:1012E000704700BF016A034640694A1C405CD968E8
:1012F0008A4228BF00221A62704700BF436A82698F
:1013000010B4D154436A416B046901330A68A342A3
:1013100028BF00235DF8044B42F0800243620A605C
:10132000704700BF436BD86910F0100002D0102244
:1013300001201A62704700BF2DE9F047046982B0AE
:10134000C3681C4046D0814688464FF0004501F1F5
:10135000500701F13806B4FA84F325FA03F21B3B77
:10136000D2431440C9F81020B8F1000F5FD0042B0D
:101370002ED8DFE803F052483D320300D8F8103091
:10138000D9F82CA033B19B6823B11FFA8AF108F178
:1013900008009847D8F8283033B19B6823B11FFA6A
:1013A0008AF108F120009847D8F8403033B19B68A3
:1013B00023B11FFA8AF108F138009847D8F858305D
:1013C00033B19B6823B11FFA8AF108F150009847A6
:1013D000002CC0D102B0BDE8F087D8F8103008F179
:1013E0000800D9F834105B689847002CB3D1F1E7B6
:1013F000D8F8283008F12000D9F838105B689847F1
:10140000002CA8D1E6E7D8F840303046D9F83C1097
:101410005B689847002C9ED1DCE7D8F858303846F6
:10142000D9F840105B689847002C94D1D2E7042B80
:1014300007D8DFE803F01903140F0A00D9F83C308D
:101440000193019B002C86D1C4E7D9F82C3001937D
:10145000019BF7E7D9F834300193019BF2E7D9F803
:1014600038300193019BEDE7D9F840300193019B9F
:10147000E8E700BF70B5124D124A2B68A2FB0323A8
:101480009B09013BB3F1807F01D3012070BD4FF078
:10149000E0220D4900240F2853614FF0F003064667
:1014A00081F823304FF0070394611361EDD80146B2
:1014B0004FF0FF3075F046FB20466E6070BD00BFF8
:1014C00000000024D34D621000ED00E0F0B50C46A2
:1014D000114602688646936913F0100C72D04FF0E3
:1014E000000C102338486546D36193699E065FD48B
:1014F00045B903685B1AA3423DD893699F06F8D5A6
:101500002023D3614CF0040C01209369D90552D5F6
:101510004FF480715F054CF0010CD16104D54FF49C
:1015200080614CF0080CD1619D0504D54FF4007327
:101530004CF0020CD3619369990701D500239362A3
:101540009369DB0703D4936943F001039361536804
:1015500020241E4901200B4000215360DEF8443056
:101560008EF8401043EA0C03CEF844308EF8414028
:101570008EF84210F0BD57689EF842309669DBB293
:10158000360408D57E0406D4202B04D0536843F4D7
:1015900080435360016893699F06A6D403685B1A71
:1015A000192BF8D993694FF0200C01259E069FD581
:1015B000002DA5D0A6E75E05B1D49C05B6D40028C1
:1015C000B9D1F0BD6046A0E7002E002400E800FE7F
:1015D0002DE9F04707689A46089EBB6931EA030384
:1015E0000CBF01230023934220D180460C461546B0
:1015F000DFF85C90324651464046FFF767FF20BB5C
:10160000D9F80030A3EB060CD44507D9BB6934EAFE
:1016100003030CBF01230023AB420AD0BB6934EAA9
:1016200003030CBF01230023AB42E3D00020BDE83D
:10163000F087D8F84430202288F840001343C8F8D7
:10164000443088F8412088F842000120BDE8F08746
:10165000002E00240C4A136903F03803102B0CD021
:10166000182B09D05BB913689B060AD51368074885
:10167000C3F3C103D840704736E4054870470548B6
:1016800070470248704700BF004402580090D003E2
:1016900040787D0100093D00184A136903F03803C2
:1016A000102B10B524D0182B09D01BBB13689B0638
:1016B00022D513681248C3F3C103D84001E0FFF7F5
:1016C00013FC0E490F4A8B698969C3F303230E4C3F
:1016D00001F00F0113440A4493F8301092F83030AF
:1016E00001F01F0203F01F03D0402060D84010BD5E
:1016F0000648E6E70648E4E70148E2E70044025806
:101700000090D00390A10C080000002440787D01D7
:1017100000093D00474A70B4946A956AD66A15F488
:101720007C3FC5F30533D16B5BD0C1F3CC01C6F36D
:10173000001604F0030407EE903A06FB01F1012CB9
:10174000B8EEE77A06EE901AFAEEE96A03D0022CB8
:101750006AD0002C4AD0DFED387A87EE876A936B27
:10176000C3F3080307EE903AF7EE005AF8EEE77A73
:1017700077EEA67A77EEA57A67EE867A2D4AB7EEEF
:10178000006A936BC3F3462307EE103AB8EEC77AAC
:1017900070BC37EE067AC7EE876AFCEEE66AC0EDEB
:1017A000006A936BC3F3064307EE103AB8EEC77AAC
:1017B00037EE067AC7EE876AFCEEE66AC0ED016A8C
:1017C000936BC3F3066306EE903AF8EEE66A76EEA4
:1017D000866A87EEA67AFCEEC77A17EE903A8360A7
:1017E000704770BCC0E900338360704713689B0684
:1017F0001DD51468F7EE005A936B1049C4F3C1026B
:10180000C3F30803D14007EE903A06EE101AF8EE43
:10181000E77AB8EEC66A77EEA66AC6EE077A36EEC3
:10182000A57A67EE877AA9E7DFED057A95E7DFED20
:10183000057A92E7004402580024744A0090D003CD
:1018400020BCBE4B0024744C0269836870B504460A
:1018500005681343C069626986B029681343AC4ABE
:1018600003430A40616A1343E2682B606B6823F408
:1018700040531343A2696B60A64B9D4200F0668102
:10188000236AAE681A43A44B33401A43AA60EB6A3A
:1018900023F00F030B43EB62A04B9D4228D0A04BDB
:1018A0009D421AD09F4B9D4217D09F4B9D4214D012
:1018B0009E4B9D4211D09E4B9D4219D09D4B9D4207
:1018C0000BD09D4B9D4208D0012000234FF0011208
:1018D0006367A266A36706B070BD984B5B6D03F0AB
:1018E0000703052BF0D8DFE803F09F7F8A925F792A
:1018F000924B5B6D03F03803282BE5D801A252F818
:1019000023F000BFB11A0408C9180408C918040854
:10191000C9180408C9180408C9180408C918040813
:10192000C9180408E9190408C9180408C9180408E2
:10193000C9180408C9180408C9180408C9180408F3
:10194000C9180408FF190408C9180408C9180408AC
:10195000C9180408C9180408C9180408C9180408D3
:10196000C91804080F1A0408C9180408C91804087B
:10197000C9180408C9180408C9180408C9180408B3
:10198000C9180408A9190408C9180408C9180408C2
:10199000C9180408C9180408C9180408C918040893
:1019A000C9180408DD190408B0F5004F644853D085
:1019B000644B626803EB4103B3F84030B0FBF3F0D3
:1019C00000EB52004FF6EF73B0FBF2F0A0F1100203
:1019D0009A423FF679AFE860002076E7B0F5004F15
:1019E0003AD04FF40040E3E7B0F5004F2DD003A804
:1019F000FFF790FE04980028EED0616AD8E7B0F5B2
:101A0000004F71D06846FFF7E1FA0198F3E7B0F5AF
:101A1000004F5ED0494B1A68920639D51B684A4878
:101A2000C3F3C103D840C3E7B0F5004F32D0FFF78E
:101A300033FE424A434BD269C2F30212134493F875
:101A4000303003F01F03D840D5E703A8FFF762FE4C
:101A500004980028C0D0616A3A4B626803EB4103E6
:101A60004FF6EF71B3F84030B0FBF3F0530803EBDF
:101A70004003B3FBF2F3A3F110028A423FF624AF16
:101A800023F00F02C3F3420392B21343EB60A3E7C8
:101A90002D488DE7FFF700FE284A2A4BD269C2F392
:101AA0000212134493F8303003F01F03D840D0E7FC
:101AB000B0F5004F1DD0FFF7EFFD204A214BD26952
:101AC000C2F30222134493F8303003F01F03D840CE
:101AD00091E71A4B1A68900640F1A5801B681A48D6
:101AE000C3F3C103D840B7E76846FFF76FFA019820
:101AF000AFE7FFF7D1FD114A124BD269C2F30222C0
:101B0000134493F8303003F01F03D840A1E700BF1F
:101B1000F369FFCF000C0058FFF4FF1100100140E3
:101B20000044004000480040004C0040005000408D
:101B30000014014000780040007C0040004402583E
:101B400000093D0090A10C080090D003A868374B15
:101B500003401343364AAB60EB6A23F00F030B4399
:101B6000EB62936D03F00703052B3FF6ADAEDFE8A4
:101B700003F0413C3303524F2D4B1A6895064CD469
:101B80002C482D4B656803EB410305EB4501B3F889
:101B90004020B0FBF2F399423FF696AEB3EB053F1F
:101BA0003FF692AE002319467FF094FD2A460902C3
:101BB000030241EA1061680818184FF0000341F170
:101BC00000017FF087FD1D4BA0F540729A423FF661
:101BD0007BAE1B4BD860FFE66846FFF7F7F901982C
:101BE00000283FF4F9AE616ACBE703A8FFF792FD46
:101BF0000498F5E7FFF750FD0D4A0F4B126AC2F348
:101C00000212134493F8303003F01F03D840E7E783
:101C10004FF40040B5E70B48B3E71B680548C3F332
:101C2000C103D840ADE7034816E700BFFFF4FF113A
:101C3000004402580090D00390A10C08FFFC0F0054
:101C4000000C005800093D00474A70B4946A956A38
:101C5000D66A15F47C7FC5F30513516B5BD0C1F3D5
:101C6000CC0106F0010604F0030407EE903A06FBEF
:101C700001F1012CB8EEE77A06EE901AFAEEE96A65
:101C80004ED0022C6DD0002C4DD0DFED387A87EE8F
:101C9000876A136BC3F3080307EE903AF7EE005A16
:101CA000F8EEE77A77EEA67A77EEA57A67EE867A8F
:101CB0002D4AB7EE006A136BC3F3462307EE103AC2
:101CC000B8EEC77A70BC37EE067AC7EE876AFCEECC
:101CD000E66AC0ED006A136BC3F3064307EE103AE1
:101CE000B8EEC77A37EE067AC7EE876AFCEEE66A88
:101CF000C0ED016A136BC3F3066306EE903AF8EE8B
:101D0000E66A76EE866A87EEA67AFCEEC77A17EE6A
:101D1000903A8360704770BCC0E9003383607047BD
:101D2000DFED137AB3E713689B06AED51468F7EEC0
:101D3000005A136B0F49C4F3C102C3F30803D14027
:101D400007EE903A06EE101AF8EEE77AB8EEC66A99
:101D500077EEA66AC6EE077A36EEA57A67EE877A40
:101D6000A6E7DFED057A92E7004402580024744CA0
:101D70000024744A0090D00320BCBE4B344A136840
:101D800030B423F08063334C1360256803E023688C
:101D90005B1B022B54D813681B01F8D4936A0568A7
:101DA00023F47C3343EA053393628368C568013BBF
:101DB000013D5B022D049BB205F4FE052B434568F3
:101DC000013DC5F308052B430569013D2D0605F0CE
:101DD000FE452B439363D36A456923F0C0032B432D
:101DE000D362D36A856923F020032B43D362D36A7D
:101DF00023F01003D362D36BC0696FF3CF0343EAC0
:101E0000C003D363D36A43F01003D362D36AD1B162
:101E100001290CBF43F4801343F40013D3620C4A2E
:101E2000136843F080631360216803E023685B1A42
:101E3000022B05D813681B01F8D5002030BC704771
:101E4000032030BC704743F40023D362E7E700BFB0
:101E500000440258002E0024344A136830B423F0A2
:101E60008053334C1360256803E023685B1B022B0F
:101E700054D813689B00F8D4936A056823F07C73E8
:101E800043EA055393628368C568013B013D5B02E9
:101E90002D049BB205F4FE052B434568013DC5F3B7
:101EA00008052B430569013D2D0605F0FE452B4332
:101EB0001364D36A456923F440632B43D362D36A26
:101EC000856923F400732B43D362D36A23F48073B0
:101ED000D362536CC0696FF3CF0343EAC00353640A
:101EE000D36A43F48073D362D36AD1B101290CBFA2
:101EF00043F4000343F08073D3620C4A136843F049
:101F000080531360216803E023685B1A022B05D815
:101F100013689B00F8D5002030BC7047032030BC0C
:101F2000704743F48003D362E7E700BF00440258E0
:101F3000002E0024F0B5354AB0F1804F344DA0EBAF
:101F400002020368A0EB050E4C69B2FA82F28F68B8
:101F5000BEFA8EFE0E684FEA52124FEA5E1E1FD086
:101F6000F2B9DFF8B8C0604537D00CF5806C604539
:101F700033D00CF5806C604512D0BEF1000F0FD14C
:101F8000244D254A904218BFA8422AD002F580620B
:101F9000904226D023F08003C76286621C4314E07F
:101FA0004D6823F07003D1F80CC02B43C7628662E2
:101FB00023F4407343EA0C0323F080031C4312B95B
:101FC000BEF1000F16D00B6903630368012243F0D2
:101FD0000403036042610460F0BD23F070034A68AB
:101FE0001343CA6823F44073C7621343866223F025
:101FF00080031C43074A084B984218BF9042E2D026
:1020000003F580639842DED0DFE700BF00000140A7
:102010000004014000400140004401400004004031
:10202000026810B452E8003F23F4907342E8003194
:102030000029F7D1144C02F1080353E8003F234074
:1020400002F1080C4CE800310029F4D1C36E012BD9
:1020500008D0002320225DF8044BC0F88C20436791
:10206000C366704752E8003F23F0100342E8003196
:102070000029EED052E8003F23F0100342E800317F
:102080000029EFD1E5E700BFFEFFFFEF436BDA6900
:10209000F0B5970683B0044642D5586AE36AC0B2E9
:1020A000002B00F09580216B9847636B1A681D46E2
:1020B00022F480721A609A6822F001029A609A698A
:1020C00042F008029A61DA69D6072DD4DA699007DE
:1020D00001D502221A62DA69510701D504221A6277
:1020E000DA69120701D508221A62DA69170612D5D1
:1020F000D4F8BC20212A0ED0D4E909128A4273D028
:10210000A169895C0132C9B299622169B2FBF1F01F
:1021100001FB1022A262DA69560608D403B0F0BDB2
:10212000DA691D46D607D1D501221A62CEE7DA69EF
:1021300040F60F0C1E6804F1340012EA0C0F996887
:1021400036D0B24F0F4040F0BB80DFF8CCC216EA69
:102150000C0F40F06381D4F8A050012D4CD0D50273
:1021600002D54F0200F16781150606D501F4000182
:1021700006F080050D4340F043815106CED572062E
:10218000CCD553E8002F22F0400243E8002141B1B2
:10219000626B52E8003F23F0400342E8003100291F
:1021A000F7D120220023C4F8BC20C4F8AC30B5E736
:1021B0009506D0D506F0200501F080573D43CAD0E2
:1021C000D4F8A830002BA9D003B0BDE8F0401847E0
:1021D000E3696269D054E369E2680133B3FBF2F169
:1021E00002FB1133E36160E70022A4F88A201A6839
:1021F00022F080021A608EE7D706B0D5F506AED57C
:102200001022B4F890501A629A68570640F11D8166
:10221000D4F8B40001684A6892B2002A00F05081F4
:10222000AA4280F04D81C169A4F89220B1F5807F67
:1022300040D053E8002F22F4807243E8002141B1DE
:10224000626B52E8001F21F4807142E80015002DF6
:10225000F7D103F1080252E8002F22F0010203F146
:10226000080545E800210029F3D103F1080252E8EE
:10227000002F22F0400203F1080545E80021002963
:10228000F3D12022C4F8C020C4F8A01053E8002FD6
:1022900022F0100243E80026002EF7D15C490D68B9
:1022A00040B190F83530022B00F01381802380F884
:1022B000346043650223C4F8A430B4F892302DE7AB
:1022C00012F0010F0CD016F4807F09D04FF0010CF2
:1022D000C3F820C0D4F8C4C04CF0010CC4F8C4C08A
:1022E00012F0020F7BD112F0040F0CD011F0010F8D
:1022F00009D04FF0040CC3F820C0D4F8C4C04CF08F
:10230000020CC4F8C4C012F0080F0CD006F0200C68
:102310005CEA070C07D008271F62D4F8C47047F0A6
:102320000807C4F8C47017050AD5770108D54FF41B
:1023300000671F62D4F8C43043F02003C4F8C430EF
:10234000D4F8C430002B3FF4E9AE92060CD506F069
:10235000200601F080510E4306D0D4F8A8301BB1FE
:1023600001909847656B0198D4F8C420AB6802F0DF
:10237000280203F04003134361D0FFF751FEAB681E
:102380005B067FF5CBAE05F1080353E8003F23F071
:10239000400305F1080141E8003262B1626B02F1CD
:1023A000080353E8003F23F0400302F1080040E82F
:1023B00000310029F3D1D4F8B40000283FF4AEAEC8
:1023C00090F83520134B022A03653BD1FDF7CEFE72
:1023D00000283FF4A3AED4F8B400036DF4E611F086
:1023E000010F90D04FF0020C12F0040FC3F820C080
:1023F000D4F8C4C04CF0040CC4F8C4C083D078E74F
:10240000D4F8AC30002B7FF4DFAE87E6010000107B
:10241000002E0024B11104082001000412F0010F65
:102420003FF471AF16F4807F7FF450AF12F0020FCB
:102430007FF469AF57E74FF480121A626EE6C4F872
:10244000C4306BE680224265BEE6B4F89220B4F850
:10245000921092B289B2AA423FF460AE00293FF4D2
:102460005DAE53E8002F22F4907243E8002141B1A1
:10247000626B52E8001F21F4907142E800100028BE
:10248000F7D1954803F1080252E8002F024003F10A
:10249000080545E800210029F4D12022C4F8A8103D
:1024A000C4F8C020C4F8A01053E8002F22F0100296
:1024B00043E800210029F7D10223C4F8A4302DE617
:1024C000AA427FF42BAEC369B3F5807F7FF426AEBA
:1024D000F2E70368814A824E824FB34218BF9342AB
:1024E00006F118060CBF01220022B34208BF42F0D9
:1024F00001021836B34208BF42F001021836B34257
:1025000008BF42F001021836B34208BF42F0010290
:1025100006F55676B34208BF42F001021836B342C0
:1025200008BF42F001021836B34208BF42F0010270
:102530001836B34208BF42F001021836B34208BF52
:1025400042F001021836B34208BF42F001021836C9
:10255000B34208BF42F00102A6F59266BB4218BF23
:10256000B34207F592670CBF01260026BB4208BFA5
:1025700042F0010256EA020779D0D3F800C02CF0ED
:102580001E0CC3F800C0D3F814C02CF0800CC3F8A4
:1025900014C0D0F860C076BBD0F860C0DCF8006032
:1025A00026F48076CCF800601A6822F001021A60E6
:1025B00003E00A68521B052A24D81A68D607F8D403
:1025C000D0E9165101F01F012FB33F238B40AB60C0
:1025D000C36ED0E91921516033B11A68016F22F43A
:1025E00080721A60436F4B600122002380F835200F
:1025F00080F834305EE6DCF8002022F48072CCF8FB
:102600000020D1E7202103220023416580F83430E7
:1026100080F835204EE6344A344EB34218BF934218
:1026200006F114060CBF01220022B34208BF42F09B
:1026300001021436B34208BF42F001021436B3421D
:1026400008BF42F001021436B34208BF42F0010253
:10265000012606FA01F1696025498B4208BF42F064
:102660000102002AB4D1234A9342B1D0BCE71E4EE6
:10267000DFF878C0634518BFB3420CF1140C0CBFEF
:1026800001260026634508BF46F001060CF1140C34
:10269000634508BF46F001060CF1140C634508BF02
:1026A00046F001060CF1140C634508BF46F0010624
:1026B000D3F800C02CF00E0CC3F800C0DFF830C017
:1026C000634508BF46F00106002E7FF465AF094E52
:1026D000B3423FF461AF67E7FEFFFFEF4000024007
:1026E0005800024028000240085402581C54025866
:1026F00080540258945402584B4B10B41B684B4CF6
:10270000A4FB03435B0A03FB02F25AB18446531E47
:102710004748DCF83420013B024201D0920406D540
:102720005C1CF6D14FF000405DF8044B7047DCF8BC
:1027300034305C0741D4DCF83430D80709D43D4B41
:10274000CCF83830DCF81030DBB2994205D00120EB
:10275000EAE70123CCF83830F9E7DCF814303648E2
:1027600018400028E0D0002B2CDB5A002DD49C0010
:102770002DD4D9002DD41A012ED45C012FD4D90127
:1027800030D41A0231D45C0232D499023CD4DA0239
:1027900037D45C0332D499032DD4DA0340D41C041B
:1027A0003BD4590436D49A0431D413F0080F0CBF2B
:1027B0004FF480304FF40000B6E704231846CCF8FD
:1027C0003830B1E74FF00070AEE74020ACE7802032
:1027D000AAE74FF48070A7E74FF40070A4E74FF426
:1027E0008060A1E74FF400609EE74FF480509BE7C4
:1027F0004FF4005098E74FF4802095E74FF40030F5
:1028000092E74FF400408FE74FF480408CE74FF49D
:10281000800089E74FF4001086E74FF4801083E7CB
:102820004FF4002080E700BF00000024D34D621069
:1028300045002000C500200008E0FFFD82B0002315
:10284000019302E00369002B09DB019B0133019333
:10285000019BB3F1706FF5D9032002B07047890175
:10286000002341F020010193016103E0036913F0AB
:10287000200307D0019B01330193019BB3F1706FDB
:10288000F4D9E9E7184602B0704700BF82B00023D0
:10289000019302E00369002B09DB019B01330193E3
:1028A000019BB3F1706FF5D9032002B0704700228D
:1028B00010230192036103E0036913F0100307D0B2
:1028C000019B01330193019BB3F1706FF4D9EBE7E6
:1028D000184602B0704700BF82B00023019302E0A7
:1028E0000369002B09DB019B01330193019BB3F1C9
:1028F000706FF5D9032002B070470023019303697C
:1029000043F00103036103E0036913F0010307D0FF
:10291000019B01330193019BB3F1706FF4D9E9E797
:102920001846E8E72DE9F843056807460C46C5F365
:102930001009B9F1000F35D1844B4FF6FF72B3F88F
:10294000803093424FD0002B4DD0814A02EA432879
:1029500008F10068454534BF4FF001084FF0020808
:102960007C4B9D4206D903F500339D4200F2C480A2
:102970004FF00109784E337E012B0FD00123B8F1BF
:10298000010F33764FF00003F36132D0022074F070
:1029900085F8002800F09180002333764FF0FF3057
:1029A000BDE8F8836C4E337E012B49D0012333768A
:1029B00005F17843B3F5801F46D3A5F10163B3F564
:1029C000801F3DD200230220F36174F067F80028D5
:1029D0006DD1624A4FF00208D2F80C3143EA080385
:1029E000C2F80C313DE0B5F1016F63D3052012F060
:1029F00055FD404674F052F80028CDD14046DFF82E
:102A00005C81D8F80C3023F4E663C8F80C30D8F8B1
:102A10000C3043EA092343F0A403C8F80C3074F0E7
:102A20003DF8D8F80C204E4B1340C8F80C30002865
:102A3000B2D105F178430122B3F5801F327603D37A
:102A40006FF00100BDE8F88300230120F36174F00A
:102A500025F860BB414A4FF00108D36843F00203F8
:102A6000D360BFF36F8FBFF34F8F04F1200254F890
:102A7000043B944245F8043BF9D1BFF36F8FBFF399
:102A80004F8F404674F00AF8B8F1010F334A2ED048
:102A9000D2F80C3123F00203C2F80C310023337654
:102AA0000028CDD13B6820333B60BDE8F88300238C
:102AB0003376C5E74FF0010852E7DFF8A080022027
:102AC000D8F80C3123F4E663C8F80C31D8F80C318F
:102AD00043EA092343F0A403C8F80C3173F0DEFF86
:102AE000D8F80C211E4B1340C8F80C319FE7D3686F
:102AF00023F00203D360D1E703F500339D4211D9DF
:102B000003F500339D4210D903F500339D4206D9E9
:102B100003F500339D420BD84FF005092AE74FF02B
:102B2000040927E74FF0020924E74FF0030921E7E2
:102B300003F500339D4206D9B5F1016FBFF456AFDE
:102B40004FF0070916E74FF0060913E700E8F11FF9
:102B500000FE1F00FFFF0108002E0024002000528D
:102B6000FBF8FFFF2DE9F04FF427A24D89B0044692
:102B700000FB07F705F10808EE194744F08973F0E8
:102B800019FBB08973F016FBD6F8F83008214FF422
:102B9000403C012B3363B2684FF0030ED4BF0023D7
:102BA0000123B26173620023C6E907C14FF480615B
:102BB000336486F83430F1634FF48071B363B362E9
:102BC0000393B98486F850304FF48053C6E911E37B
:102BD000F36E002B00F0B78093689E0003D59168D8
:102BE000854B0B4093609368D80015D42B688349BC
:102BF0009B099068A1FB031381499B0901400133A4
:102C000041F0805191600393039B2BB1039B013BE7
:102C10000393039B002BF9D19368D9001DD4F423AF
:102C2000012703FB0453D96E41F01001D966196FD7
:102C300039431967936813F0040F4FF0F40303FB53
:102C400004530CD0DB6EF42303FB0453DA6E42F022
:102C50001002DA6609B0BDE8F08F0027EAE7D96E06
:102C600011F01009EFD1D96E21F4817141F0020108
:102C7000D9669368DB0713D4624B9A4200F0D9827D
:102C800003F580739A4200F0D4825F4B9B68D907AA
:102C900006D45E498B6823F47C1343F440338B6085
:102CA0005B4B5C491B68D368194043F208030B4334
:102CB000D360936813F0040F936848D0F42303FBA8
:102CC00004539B69F42202FB0452516A012900F06B
:102CD0007E821A6B22F00F021A63F42202FB045266
:102CE000D16E21F0030141F00101D166002FB1D175
:102CF00092F8681004970129ACD0012182F868107D
:102D00009968890700F18C809968CE0740F1898025
:102D1000996801F00D01012900F02684D36E43F07B
:102D20001003D366136F43F001031367F4230021EC
:102D300003FB0453DA6E83F8681042F01002DA667F
:102D400009B0BDE8F08F336786F8683044E71B07A9
:102D5000B4D4D168304B0B4043F00303D360136904
:102D600023F001031361F42303FB0453D96C1369AB
:102D700023F070430B431361224B9A4200F05182BF
:102D800003F580739A4200F04C82204B9B6813F449
:102D9000403F14BF01230023002B00F02082FEF7E8
:102DA0007BFCF42303FB0453DB69B3F5003F00F025
:102DB000B782B3F5403F00F04184B3F5803F00F0A7
:102DC000AF82134B41F203021968F423B2EB114FA7
:102DD00003FB04539B69C0F0E983104B984240F217
:102DE0000284F42303FB04539B699A6842F48072C3
:102DF0009A6067E700000024C0FFFF5F632D3E0577
:102E0000C0FFFF6F002002400060025800630258BC
:102E10000010005C03C0F0FFFCBFFFFF002D31017C
:102E20009A68F420B149B24A00FB0450C66E3140A2
:102E300041F00201C16699680A4042F000429A607E
:102E40009A68AC49002AC0F2A4814FF0F40BAA4B57
:102E5000DFF8D0A20BFB04FBDFF8CCE2A74E05EBBA
:102E60000B0CA748A749DCF81020524518BF9A421E
:102E70000BF1740ACCF87C200CBF01230023C24460
:102E8000724508BF43F001034FF4005EB24208BF31
:102E900043F001034FF48066824208BF43F0010310
:102EA000DCF814008A4208BF43F001031831CCF863
:102EB00080008A4208BF43F0010318318A4208BFEC
:102EC00043F0010301F556718A4208BF43F0010344
:102ED00018318A4208BF43F0010318318A4208BF03
:102EE00043F0010318318A4208BF43F0010318314F
:102EF0008A4208BF43F00103DCF86C1021F00301A3
:102F000041F00101CCF86C107F498A4208BF43F0C0
:102F1000010318318A4208BF43F0010300218CF8F5
:102F20006810CCF8A010CCE92111CCE92A114FF49B
:102F30000061CCE923614FF48071744ECCE925E146
:102F40004FF400314FF0030ECCF89C10CCF8A4E005
:102F500031681BB96E4B9A4240F076864FF0F40C04
:102F600002234FF0000E0CFB045C8CF8B1301368A8
:102F70008CF8B0E023F00103136004E033685B1ABF
:102F8000052B00F21A811368DB07F7D4614BD2F8E6
:102F900000E0DFF8A0C11B685F4903EA0C0C5F4B3F
:102FA0000EEA0101BCF1005F43EA01030DD32E28B4
:102FB00040F24C813F38132807D8DFF87CC12CFA47
:102FC00000F0C00701D5564B0B43136050465369C0
:102FD00023F007035361FDF749F8F42303FB04537F
:102FE000D3F8D8203F2302F01F0293408360F423DC
:102FF000414903FB0453DA6F4A4B9A4218BF8A4295
:103000000CBF0121002100F0E482474B9A4200F0FE
:10301000218118339A4200F0148318339A4200F049
:10302000E38318339A4200F0E78318339A4200F0A2
:10303000228418339A4200F02E8403F556739A4284
:1030400000F02E8418339A4200F0288418339A42F4
:1030500000F0D58518339A4200F0F18518339A4272
:1030600000F0498618339A4200F0608618339A427D
:1030700000F0598618339A4200F078872B4B9A4219
:1030800000F03C8614339A4200F0388614339A429A
:1030900000F0D48714339A4200F0D08714339A4258
:1030A00000F0CA8714339A4200F0C88714339A425A
:1030B00000F0C48714339A4200F0C0870BF1100B64
:1030C000F422002102FB045208EB0B03C2F864A0B7
:1030D0004FF0010AC2F8B430154BC2F8D01003F11A
:1030E000480B82F8B1A0CDE900762BE0FDEEFFFFA2
:1030F000C0FFFE3F00F8C325100002405800024008
:10310000700002408800024088040240002E002423
:10311000B80402400010005C3F8010FE002D020049
:10312000002D1200280002404000024008540258BE
:10313000202E00240000FFFF0F030F000C339B45DF
:1031400000F0F280597D0029F8D093F90D10A142CA
:10315000F4D1002100981F6905918B499E7D01EBF8
:103160008001886D92F8681001293FF473AD916970
:1031700082F868A0D1F808C01CF0040F00F01C8190
:10318000D36E4FF0000143F0200382F86810D3663D
:1031900060E5049A01320492049A8A42FFF450AE28
:1031A000F423002103FB0453DA6E83F8681022F045
:1031B000120242F01002DA664CE5F42320210322C9
:1031C00003FB0453C3F8D01083F8B12042E5126B1F
:1031D000196B013A21F00F010A431A637DE56B4A2E
:1031E000936D03F44033B3F5803F00F09080B3F566
:1031F000003F00F029821BB913681E0100F13E83D5
:10320000634B1A6841F20303B3EB124F80F0EB817A
:10321000F42303FB04539B699A6822F440729A607A
:1032200050E55C4B9B6813F4403F14BF012300231F
:10323000B2E5594B996803F580739B68DE073FF54B
:103240002FADC8073FF52CAD524923E528287FF65E
:10325000BCAEB8E64FF00209504B4FF0010E002112
:103260004B440EFA09FEDFF844914FEA830CF42038
:1032700000FB0450D0F88430C0F8E4E0802BC0E9B3
:1032800037C900F02181D0F88030D8B2013B072B3C
:10329000CCF80000C9F804E000F21D81404BDFF8D3
:1032A00010C1624518BF9A420CF1140C0CBF0123E7
:1032B0000023624508BF43F001030CF1140C624582
:1032C00008BF43F001030CF1140C624508BF43F042
:1032D00001030CF1140C624508BF43F0010300F137
:1032E000FF3C13B9002900F000852E4901442E4807
:1032F0008900F423012203FB045302FA0CF2C3E910
:103300003A10C3F8F02000230B604260D6E6136841
:1033100098007FF575AF05A8FDF758FE079850E5B2
:103320001B0CB0FBF3F04CE5F4231B4A019E03FB9E
:103330000453D3F8F8109B69934200F0C28002F561
:103340008072934200F0BD80DFF868C0DCF808703E
:103350009A6850073FF57EACF42000FB045090F8CB
:103360006820012A3FF476AC07F01F0740F22122C3
:103370004FF0010EFA4080F868E012EA0E0240F0C9
:10338000438180F8682065E490A10C08004402584D
:103390000010005C00230240002002400082001068
:1033A000305402583F960016405902588008024097
:1033B0004454025800630258002F4FEA976C0DDB0B
:1033C000C7F3130EBEF1000F40F017810AFA0CF894
:1033D000D1F81CE04EEA080EC1F81CE04FEA901E3E
:1033E00001F1300800F01F000CF01F0C0EF00C0E65
:1033F0004FF01F090CFA00FC09FA00F958F80E000A
:1034000020EA090040EA0C0048F80E00886810F035
:10341000040F886847D1000745D44FEAD75CC7F34B
:10342000045001F1140E4FF007080CF0040C06FADA
:1034300000F908FA00F85EF80C0020EA080040EAFB
:1034400009004EF80C009748006800F07040B0F199
:10345000805FC86800D0C868086E4FEA876C00F0CB
:10346000F840B0EB876F03D1086E20F0004008668B
:10347000486E00F0F840844503D1486E20F00040CB
:103480004866886E00F0F840844503D1886E20F0CD
:1034900000408866C86E00F0F840844503D1C86ECD
:1034A00020F00040C8668868C6071DD50099002036
:1034B0000131C9B20091F42101FB045181F8680087
:1034C0003CE6DFF80CC241E70023C0F88030CCF8BE
:1034D0000030C9F804E0F423002203FB0453C3E9DD
:1034E0003A22C3F8F020E9E5D1F8C000C7F3130C85
:1034F000002F20EA0C00C1F8C000D7DA6A488142E8
:1035000000F0548100F58070814200F04F8100F19D
:10351000C050DFF898E100F58440D0F808C0DEF82C
:10352000088018F0010F40F03581DFF8A8810CF019
:10353000E079474500F04083DFF89C81474500F083
:103540001083DFF898E17745B0D11CF4800FADD13E
:10355000564FB942AAD1816821F0E07141EA0901D0
:1035600041F480018160A1E79968514A514E0A40B7
:1035700042F002029A6003221A6031689A68D20708
:103580007FF54FAC3268521A022AF7D99A68D007F1
:10359000F4D5F42303FB0453DA6E42F01002DA662A
:1035A0001A6F42F001021A67FFF7C0BB424A90420D
:1035B0007FF62EAE414A904268D9414A90429A68BD
:1035C00000F2158122F4407242F400729A60FFF713
:1035D00079BB5FFA82F93B4BA9F11009A3FB0939CA
:1035E0004FEA191938E6F42303FB04539B699A68E0
:1035F00022F480729A60FFF765BB97FAA7F8B8FAD1
:1036000088F80AFA08F8E3E69A68D20768D4D3F88B
:1036100008E02D4A1EEA020F00F0F380C36E43F06B
:103620001003C366036F43F001030367F423002212
:1036300003FB045383F86820FFF70CBB8008FFF7F7
:10364000C0BB4FF0030907E6D36C116803F0405389
:10365000490702D5002B00F017811C4A1268D605D5
:1036600003D5B3F1805F3FF4CBAD184A12689003E5
:103670007FF5C6ADB3F1005F7FF4C2AD094B1A68A8
:1036800041F20303B3EB124FBFF4ABABF42303FBE4
:1036900004539B699A6822F4407242F480729A60E3
:1036A000FFF710BB0010005C0020024000600258D1
:1036B000C0FFFF7F002E002421BCBE0041787D01A9
:1036C00081F0FA02ABAAAAAA3F0000800044025887
:1036D00000230240000084CB000052C70000B8CF96
:1036E0007148181A18BF0120F426704A06FB0456C8
:1036F000D6F86CC00CEA020242F48072F26607B19E
:1037000030B1F42202FB0452D06E20F48010D06657
:10371000F42202FB0452D06E10F480506FD0106F70
:1037200020F006001067F422614E624F02FB045243
:10373000DFF890C1506EC6641C26C0E90FC71E603A
:1037400000265F6882F8686047F010075F60576C7A
:10375000DA6822F003023A43DA6090F83420012A52
:103760000CD0012280F8342090F83520012A00F096
:10377000B1804FF4006380F834604365F4224E4B0F
:1037800002FB0452926991680B4043F0040393607A
:10379000FFF760BAF423002103FB0453DA6E83F8C9
:1037A000681042F02002DA66FFF754BA4348DFF8A7
:1037B0001881DFF8F4E0D0F808C0D8F80880DEF807
:1037C00008E01EF0010FE5D118F0010FE2D1DFF89B
:1037D000FCE077453FF46AAEDFF8F4E077453FF46C
:1037E00065AE0CF0E079ACE64FF0040934E542F444
:1037F00040729A60FFF766BA4FF005092CE5106732
:1038000091E79A68DFF8B080274802EA0802181AA0
:1038100042F0010218BF01209A60D6F800E0DCF8FF
:10382000082012F01F0F14BF024640F00102002AC8
:1038300000F008821A68D2073FF556AF9A68D2079F
:1038400005D49A6802EA080242F001029A603268DE
:10385000A2EB0E02022AEDD91A68D207EAD4F423A9
:1038600003FB0453DA6E42F01002DA661A6F42F07C
:1038700001021A67DAE64FF00609EDE405A8FDF744
:1038800049FF0598FFF79DBA13680D48C3F3C103BC
:10389000D840FFF796BA4FF00709DDE44FF0010971
:1038A00009F10809D8E400BF00210240FEF0FFFF43
:1038B0005900040855000408C0FFFF7F00230240A0
:1038C0000090D0030100040800200240000084CBD7
:1038D000000052C7AB4A4FF48C77DFF8D0E201EB1F
:1038E000810107FB042C0222A74F403380F83520CA
:1038F0004FEA810B02684665BA4218BF7245866D71
:103900000CBF4FF0010E4FF0000E00F0868118370B
:10391000BA4200F034821837BA4200F04B821837AE
:10392000BA4200F035821837BA4200F0C182183727
:10393000BA4200F0B4821837BA4200F0A78207F505
:103940005677BA4200F099821837BA4200F0F582F1
:103950001837BA4200F0E8821837BA4200F0DB822A
:103960001837BA4200F0CE821837BA4200F07C8293
:103970001837BA4200F06F821837BA4200F06282FC
:10398000824FDFF81C82424518BFBA4208F128086E
:103990000CBF01270027424508BF47F0010708F187
:1039A0001408424508BF47F0010708F114084245D2
:1039B00008BF47F0010708F11408424508BF47F067
:1039C0000107D2F8008028F00108C2F80080DFF873
:1039D000D881424508BF47F001071FB96C4FBA4272
:1039E00040F0EE82D0F86C80D0E919174F60B8F142
:1039F000000F00F0E881DFF8B891664FDFF8B4A15E
:103A00004A4518BFBA42D0E91C170CBF4FF0010954
:103A10004FF000094F60524514BF4F4649F001076F
:103A2000BEF1000F02D1002F00F0CD81C16D4FF02B
:103A30003F0901F01F0A816809FA0AF94029C6F80E
:103A40000890166826F480261660C2F804B000F0CC
:103A5000F2809360C2F80CC0BEF1000F40F0D2803B
:103A60004C4B9A4200F07F8118339A4200F06F81EC
:103A700018339A4200F05D81474B9A4200F08982E8
:103A8000464B9A4200F0758218339A4200F0FE824B
:103A900003F556739A4200F0ED8218339A4200F013
:103AA000DD8218339A4200F0D78218339A4200F030
:103AB000D18218339A4200F0CB8218339A4200F038
:103AC000C58218339A4200F0BF8218339A4200F040
:103AD0003D822E4B32498A4218BF9A4201F1280199
:103AE0000CBF012300238A4208BF43F00103116881
:103AF00021F00E0141F00A0111602A498A4208BFF3
:103B000043F0010314318A4208BF43F0010314312A
:103B10008A4208BF43F00103116841F004011160BB
:103B200021498A4208BF43F0010313B9184B9A4256
:103B300012D1D0F86C80036E1968C80303D51968D8
:103B400041F480711960B8F1000F05D0D8F8003049
:103B500043F48073C8F80030136843F00103136026
:103B60000CE61CF0807F7FF4A1AC71457FF49EAC25
:103B7000816821F0E07141EA090141F080718160C2
:103B800094E400BF00000030280002401C5402589A
:103B9000945402584000024088000240A0000240B5
:103BA00008540258445402588054025810000240ED
:103BB00058000240700002401CF4000F7FF476AC05
:103BC00071457FF473AC816821F0E07141EA09012D
:103BD00041F400018160BB482968B1FBF0F101317B
:103BE00049000591059900293FF460AC009E0599B4
:103BF0000139059105990029F9D1009656E44FF055
:103C000002094DE6136823F01E0343F01603136008
:103C1000136843F0080313608DE7176827F0010766
:103C20001760D0F86C80D0E919174F60B8F1000F19
:103C30007FF4E1AEFAE6C2F808C0D3600CE74FF0BB
:103C400003092DE610464FE59F4BA0498A4218BF55
:103C50009A4201F114010CBF012300238A4208BFDC
:103C600043F0010314318A4208BF43F001031431C9
:103C70008A4208BF43F0010314318A4208BF43F06F
:103C8000010314318A4208BF43F001031BB9904B72
:103C90009A4240F08E81F42102208E4B01FB0451A8
:103CA000DFF850C2134481F8B10014200091B3FB37
:103CB000F0F310689B0000EA0C0C42F2A0504CEAB2
:103CC00000004FF0000C81F8B0C010605046C1F801
:103CD000D830FCF7CBF900990122D1F8D81001F0C7
:103CE0001F018A404260FFF782B97B4901447B484B
:103CF0008900FFF7FEBA4FF00409D1E50121134610
:103D0000DBB277484FF0010EDFF8EC91083BA0FBE7
:103D10000303744800EB131C1B094FEA8C0C0EFACA
:103D200003FEFFF7A4BA4FF00609B9E54FF0050905
:103D3000B6E56D490B6F23F01E0343F016030B67C6
:103D40000B6F43F008030B67D0F86C80F3E666490D
:103D50008B6D23F01E0343F016038B658B6D43F0D0
:103D600008038B65F0E760490B6C23F01E0343F0FA
:103D700016030B640B6C43F008030B64E4E7DFF8F5
:103D80006881D8F8407027F00107C8F8407048E70C
:103D9000DFF85481D8F8707027F00107C8F8707008
:103DA000D0F86C80D0E919174F60B8F1000F7FF49C
:103DB00022AE3BE6DFF83081D8F8587027F00107D3
:103DC000C8F85870ECE7494FDFF830914A4518BF02
:103DD000BA4209F130090CBF012700274A4508BF44
:103DE00047F0010709F556794A4508BF47F0010732
:103DF00009F118094A4508BF47F0010709F11809F8
:103E00004A4508BF47F0010709F118094A4508BFAC
:103E100047F0010709F118094A4508BF47F00107B3
:103E200009F118094A4508BF47F0010709F11809C7
:103E30004A4508BF47F001071FB92D4FBA4240F06D
:103E4000BF80F3E5DFF8B880D8F8B87027F0010735
:103E5000C8F8B870C6E5DFF8A880D8F8A07027F0D9
:103E60000107C8F8A070BDE5DFF89480D8F8887025
:103E700027F00107C8F88870B4E5DFF88480D8F827
:103E8000107027F00107C8F81070ABE5DFF8588014
:103E9000D8F8B87027F00107C8F8B870A2E5DFF8C5
:103EA0004880D8F8A07027F00107C8F8A07099E5FD
:103EB000DFF83480D8F8887027F00107C8F88870D8
:103EC00090E500BF400D0300085402581C540258EE
:103ED00094540258F8ABFDA73F82001040090240FD
:103EE000CDCCCCCC0096001600000240A0000240D1
:103EF000B80402400F00FEFF8058025888000240BC
:103F000000040240DFF88881D8F8707027F00107BC
:103F1000C8F8707066E5DFF87881D8F8587027F037
:103F20000107C8F858705DE5DFF86481D8F8407083
:103F300027F00107C8F8407054E5DFF85481D8F83D
:103F4000287027F00107C8F828704BE55049D1F8D0
:103F5000B83023F01E0343F01603C1F8B830D1F88F
:103F6000B83043F00803C1F8B830EDE64FF0070968
:103F700096E44849D1F8A03023F01E0343F016031D
:103F8000C1F8A030D1F8A03043F00803C1F8A03048
:103F9000DAE64049D1F8883023F01E0343F01603D7
:103FA000C1F88830D1F8883043F00803C1F8883070
:103FB000CAE64023CCF8D0308CF8B1E0FEF74ABE18
:103FC000354FDFF8E080424518BFBA4208F11408C7
:103FD0000CBF01270027424508BF47F0010708F141
:103FE0001408424508BF47F0010708F1140842458C
:103FF00008BF47F0010708F11408424508BF47F021
:10400000010708F11408424508BF47F001071FB92E
:10401000224FBA427FF430ADC16D012701F01F0875
:10402000816807FA08F740297760C2F804B007D022
:104030009360C2F80CC013E5194B61E613465FE6C6
:10404000C2F808C0D3600BE5114993E71049A1E716
:104050000F496FE60E497BE60D4985E60C498B6AF0
:1040600023F01E0343F016038B628B6A43F00803B0
:104070008B6269E606490B6923F01E0343F01603C1
:104080000B610B6943F008030B615DE601495EE7D4
:1040900000040240000002400854025894540258A0
:1040A000585402581C5402580148FCF75BBA00BF30
:1040B000782E0024074810B4836FD0F8AC4099697B
:1040C0001A6824B1234678305DF8044B18475DF830
:1040D000044B7047002E00240148FCF743BA00BF90
:1040E000D02E0024084810B4D0F8D030D0F80441C5
:1040F00099691A6824B12346D0305DF8044B1847FB
:104100005DF8044B704700BF002E00240148FCF707
:1041100029BA00BF282F0024084810B4D0F828314D
:10412000D0F85C4199691A682CB1234600F5947067
:104130005DF8044B18475DF8044B7047002E0024CF
:104140002DE9F04FDFF8549300EB400583B04300B6
:1041500009EB85050093D5F8E4320193002B00F0BC
:104160005B818046B5F8EA0272F024F895F8E8021F
:104170000EF0D0FD044695F8E9020EF0CBFD08F1F3
:1041800001030746DBB2002C00F06B8140F60C12F5
:10419000A1882372E2802268002800F05681037211
:1041A00040F60C23C38091613B68BA889A61112163
:1041B000204609260EF06AFD112138460EF066FDF4
:1041C0006525002C00F02B812268A38811690B4221
:1041D00000F025811B04936110F082FC05468B469C
:1041E00010F07EFC401B61EB0B01052871F1000112
:1041F000F6D314B12368A2889A6110F071FC0546C9
:104200008B4610F06DFC401B61EB0B01052871F132
:104210000001F6D3013ED3D11CB1A38822681B0450
:10422000936110F05DFC05460E4610F059FC401BF2
:1042300061EB0601052871F10001F6D31FB1BB88BF
:104240003A681B04936110F04BFC05460E4610F0D3
:1042500047FC401B61EB0601052871F10001F6D314
:1042600014B12368A2889A6110F03AFC05460E4604
:1042700010F036FC401B61EB0601052871F10001CE
:10428000F6D317B13B68BA889A61009B20463E215D
:10429000434409EB830393F8EF4222460EF018FDE6
:1042A000224638463E210EF013FD764C5823019AE3
:1042B00003FB08439A67744B9A4200F0C180FDF7F4
:1042C000EBF9724BDA69C2F30212714B134493F8A3
:1042D000303003F01F03D840009B434409EB8303B5
:1042E00093F8EC32022B00F0B780032B00F0AF8084
:1042F000012B14BF4FF4C8714FF4487171F0E8FFFF
:1043000003465822002102FB0842C2F88010D367FE
:10431000C2E92211C2E925110121C2F8841092F8E4
:10432000B91001F0FF00002900F0A380582123F00C
:10433000706224264FF4004701FB084155488B6FFB
:1043400081F8B9601D6825F001051D601A619A6841
:1043500022F400429A609F605A6822F400625A6018
:104360005A681043D1F8902058601202D86820F49F
:104370000040D860DA6000221A60186840F001003E
:1043800018602020C1F8BC2081F8B900C1F8A8202D
:1043900081F8BA2091F8B9002028C5B217D191F858
:1043A000B800012813D081F8B960186820F0010026
:1043B0001860186820F48050186018681860186831
:1043C00040F00100186081F8B95081F8B820009BD6
:1043D00002210126304F434409EB830999F8EE523C
:1043E000284672F0AFFB05F01F036A0999F8ED52F9
:1043F00006FA03F30221284647F8223072F0A2FBA6
:10440000582303FB084405F01F036D0906FA03F364
:1044100047F8253084F8746003B0BDE8F08F013DA3
:104420002AD010F05DFB83468A4610F059FBB0EBB2
:104430000B0061EB0A01052871F10001F5D3C0E61C
:10444000FDF72AF9114B1A6A3DE79161AFE6C821E1
:1044500071F03EFF034654E7642171F039FF0346D3
:104460004FE700283FF4A3AE037240F60C23C3804D
:104470009AE682F8B80059E7002C3FF4ADAEA38865
:104480002268A7E6002E0024001C005800440258B1
:1044900090A10C080080000200E100E00000002470
:1044A0002DE9F04F441C85B017469DF83C202DD0D7
:1044B0005824DFF898831E46054600FB04F408EBF9
:1044C000040393F87490B9F1000F1FD044444900DD
:1044D000FF2F04F17804039100D0EEB9002A40F0D8
:1044E000C480582303FB058393F8B920202A04D104
:1044F000B6B94FF40072C3F8BC20B8F87C31284636
:1045000001339BB2A8F87C31FFF71AFE4FF0000987
:10451000484605B0BDE8F08F93F8B930202BECD1B8
:104520004FF0580A0AFB058A9AF8B830012BE4D0FC
:104530000122D8F800B019234FF400418AF8B820BE
:104540002046CDF800B0FDF743F80028D5D10E9BEA
:10455000DAF87810CAF89C302123B64A8AF8B930C4
:104560004023CAF8AC008AF8BA30CAF8BC0020462A
:10457000AAF8A2604B681340039A1343AE4A1A4349
:104580004A60594672F05CFA0246002840F0F78013
:10459000DAF87830802120469F620A23CDF800B0F7
:1045A000FDF716F8002840F0EA80BAF8A2309BB276
:1045B000FF2B40F21081DAF87810FF239F48AAF809
:1045C000A0304B689E4A0340039803431A434A6055
:1045D0005826DDF80CA05F46039506FB058605E02E
:1045E000B6F8A2309BB2002B00F00A813946204673
:1045F00072F026FA002840F0EC80D6F89C10B56FD7
:1046000011F8012BB6F8A030AA62C6F89C10013B45
:10461000B6F8A2109BB20139A6F8A03089B2A6F86C
:10462000A210B6F8A21089B2002BD9D10029D7D098
:1046300002460A23802120460097FCF7C9FFFF228B
:10464000002840F0C680B6F8A2309BB2934240F2F8
:104650009D80B16FA6F8A0204B68784A1340784A35
:1046600043EA0A031A434A60BAE74FF0580A0AFBC2
:10467000058A9AF8B930202B7FF43FAF9AF8B8300A
:10468000012B3FF43AAF0122D8F8007019234FF400
:1046900000418AF8B82020460097FCF799FF0028CF
:1046A0007FF42BAF0E9BCAF8AC00CAF89C302123D4
:1046B0008AF8B93010238AF8BA30CAF8BC00AAF8D0
:1046C000A260BAF8A2309BB2FF2B00F2C180BAF808
:1046D000A2309BB2AAF8A030002B40F0EA80DAF8B2
:1046E000781054484B68574A0340039803431A43D1
:1046F0004A605826AA4606FB0586B6F8A230394617
:104700009BB2002B00F0CD80204672F099F9002872
:1047100074D1D6F89C10B56F11F8012BB6F8A03003
:10472000AA62C6F89C10013BB6F8A2109BB20139F0
:10473000A6F8A03089B2A6F8A210B6F8A21089B2E5
:10474000002BDAD10029D8D002460A238021204646
:104750000097FCF73DFFFF2200284FD1B6F8A230AA
:104760009BB2934223D9B16FA6F8A0204B68334A7D
:104770001340039A1343324A1A434A60BDE7582351
:10478000002203FB058383F8B820B6E6B6F8A23012
:10479000B26F9BB229485168A6F8A030DBB2014045
:1047A0004AEA03430B4343F00073536018E7B6F83B
:1047B000A230B16F9BB2039A2048A6F8A030DBB2BA
:1047C00042EA03434A680240134343F000734B60DC
:1047D00093E7039D91E6BAF8A230DAF878109BB21D
:1047E000039A1648AAF8A030DBB242EA03434A68AB
:1047F0000240134343F000734B60E9E655467CE604
:1048000039462046039D72F0EDF800287FF475AE1E
:10481000B36F20210C4CD9615A6822405A6058234A
:10482000002286F8B91003FB058386F8BA0083F8E6
:10483000B8206DE6009800FC00200101009C00FCFF
:104840000000FF010020000200E800FE002E00240E
:10485000FF234FF47F00FE224FF08076AAF8A030AD
:10486000039BDDF838E01E4358231EF801AB03FB21
:104870000583DFF850C0996FC1F828A0A3F8A020E5
:10488000B3F8A220C3F89CE0013A92B2A3F8A220A8
:104890004B6803EA0C033343034343F400534B6078
:1048A00027E72046554672F09DF800287FF425AE94
:1048B000AEE7013B4FF000769AB2501CC0B2000444
:1048C000CEE700BF009800FC2DE9F04F441C85B0F6
:1048D00099469DF83C3000F096805825C64C064617
:1048E00000FB05F504EB050B9BF874A0BAF1000F73
:1048F00000F089802544FF2A90464FEA410705F1E0
:10490000780540F08680002B00F083809BF8B9305A
:10491000202B6FD19BF8B830012B6BD00122D4F83B
:10492000008019234FF400418BF8B8202846CDF8B9
:104930000080FCF74DFE00285CD10E9BCBF8AC004C
:10494000CBF89C3022238BF8B93010238BF8BA3087
:10495000CBF8BC00ABF8A290BBF8A2309BB2FF2B07
:1049600000F21781BBF8A230DBF878109BB2A348A5
:104970004A68ABF8A030DBB2024047EA0343134376
:104980009F4A1A434A604FF0580909FB0649B9F893
:10499000A2309BB2002B00F08A81D9F878309A6956
:1049A000520700F1378142460A212846FCF78EFD66
:1049B000002840F0FB80D9F878309A69910640F1E0
:1049C000FF809A699A6912F0100200F0F7801022B5
:1049D00020218C4DDA610422C9F8BC20D9615A68C3
:1049E0002A405A6089F8B91089F8B80089F8BA00E5
:1049F00022689B69B4F87C31304601339BB2A4F83D
:104A00007C31FFF79DFB4FF0000A504605B0BDE832
:104A1000F08F4FF0580B0BFB064B9BF8B930202B57
:104A2000E8D10E9B002B00F0AC80B9F1000F00F034
:104A3000A8809BF8B830012BDCD0236801224FF40A
:104A4000004128468BF8B820039300931923FCF704
:104A5000BFFD0028CED12223DBF878100E9A8BF808
:104A6000B9304023CBF89C208BF8BA30CBF8BC008F
:104A7000ABF8A290DFF884914A68CBF8AC002846E6
:104A800002EA09023A4342F490324A60039971F013
:104A9000D7FF0246002840F03681402328461946B9
:104AA000DBF87830C3F82880039B00930A23FCF7D7
:104AB0008FFD002840F02781BBF8A2309BB2FF2B6E
:104AC00040F22881DBF87810FF234F4AABF8A03082
:104AD0004B6803EA09033B431A434A604FF0580806
:104AE000B946039F08FB064805E0B8F8A2309BB220
:104AF000002B00F021810A23002204212846009780
:104B0000FCF766FD00287FF475AFD8F87830596A55
:104B1000D8F89C301970B8F8A210D8F89C30013938
:104B2000013389B2C8F89C30B8F8A030A8F8A210B8
:104B3000013BB8F8A2109BB289B2A8F8A0300029B6
:104B4000D3D0002BD1D102460A23802128460097DA
:104B5000FCF73EFDFF2200287FF44CAFB8F8A230EE
:104B60009BB2934240F2BD80D8F87810A8F8A020FC
:104B70004B68264A1340264A43EA09031A434A600F
:104B8000B3E758234FF4007203FB0643C3F8BC207D
:104B900030E7DBF87810FF231848ABF8A0304B68FB
:104BA000194A03403B431A434A60ECE6582303FB8F
:104BB00006439B6F9A6922689B691BE7C9F8BC2072
:104BC0002268A2EB08020A2A7FF6E9AE9A6912F07F
:104BD00004027FF4E4AE582101FB0641D1F8BC0089
:104BE00081F8B820202240F02000C1F8BC0081F8F4
:104BF000B9209B69FEE600BF002E0024009800FC4F
:104C00000024000200E800FE0024FF01009C00FCDC
:104C10000000FF015A6AD9F89C301A70B9F8A23026
:104C2000D9F89C20013B01329BB2C9F89C20A9F81D
:104C3000A230B9F8A030B9F8A220013B92B29BB2E1
:104C4000A9F8A030002A3FF4A2AE002B7FF49FAE5B
:104C50000A23002280212846CDF80080FCF7B8FC0A
:104C600000287FF4C7AEB9F8A2309BB2FF2B0CD955
:104C7000D9F87810FF233B48A9F8A0304B683A4A8E
:104C800003403B431A434A6081E6B9F8A230D9F8A1
:104C900078109BB233484A68A9F8A030DBB20240D2
:104CA00047EA0343134343F000734B606FE641460A
:104CB000284671F097FE00287FF49CAED9F8783032
:104CC00020212A4DD9615A682A405A6089F8B910C2
:104CD00089F8BA005822002302FB064484F8B83051
:104CE00093E6B8F8A230D8F878209BB21D485168F6
:104CF000A8F8A030DBB2014049EA03430B4343F07C
:104D000000735360F1E65823002203FB064383F847
:104D1000B8206FE6BBF8A230DBF878109BB24A6887
:104D2000ABF8A030DBB202EA090247EA03431343BF
:104D30000F4A1A434A60D1E60399284671F052FEA1
:104D4000034600287FF456AED8F878202020074D7F
:104D5000D06151682940516088F8B90088F8BA30AC
:104D6000B8E700BF009C00FC0000FF0100E800FE67
:104D7000002400020348D0F8143313B100F5427048
:104D800018477047000000240348D0F8343313B1AB
:104D900000F54A7018477047000000240348D0F817
:104DA000543313B100F552701847704700000024C7
:104DB0000348D0F8743313B100F55A7018477047A0
:104DC000000000240348D0F8943313B100F562705A
:104DD00018477047000000240348D0F8B43313B1DB
:104DE00000F56A7018477047000000240348D0F8A7
:104DF000D43313B100F572701847704700000024D7
:104E00000348D0F8F43313B100F57A7018477047AF
:104E1000000000240348D0F8143413B100F5816079
:104E200018477047000000240348D0F8343413B109
:104E300000F5856018477047000000240348D0F84B
:104E4000543413B100F589601847704700000024FE
:104E50000348D0F8743413B100F58D6018477047DB
:104E6000000000240348D0F8943413B100F5916099
:104E700018477047000000240348D0F8B43413B139
:104E800000F5956018477047000000240348D0F8EB
:104E9000D43413B100F5996018477047000000241E
:104EA0000348D0F8F43413B100F59D6018477047FB
:104EB0000000002410B41C46436884466FF30F03BF
:104EC00023434360036843F001030360036843F432
:104ED00000730360002C3AD040F2E930DCF8143063
:104EE0009B0748D5002A49D012F8013B40F2E9302F
:104EF0008CF82030DCF81430DB0720D40138F9D1ED
:104F0000214B9C450CD0A3F578439C4538D003F544
:104F100080639C4536D003F578439C450BD1032034
:104F20001A4A00EB400002EBC002B2F81C35013314
:104F30009BB2A2F81C3500205DF8044B70479CF82A
:104F40003000C0B209B101F8010B013CC4D1DCF85A
:104F500014301B07FBD5DCF8183001205DF8044B3A
:104F600043F01003CCF81830DCF8003023F00103D4
:104F7000CCF8003070470138B0D1C1E7FF23B5E766
:104F80000120CDE70220CBE70030014000000024E3
:104F90002DE9F84300242C4E8046036856F834501F
:104FA000AB4209D001340E2CF8D1284A002105204B
:104FB00008F0F6FC002019E0254B03EB8409D9F832
:104FC0008071AFB198F8051000204B1C01EB410235
:104FD00003EB430307EBC202DB00C2F80C80C2E91B
:104FE0000400F854182303FB01700830BDE8F8836F
:104FF0000721682008F05AFD0146C9F88001F0B188
:105000003946682283F062FFD9F8801106EBC404A8
:105010003B4689600C6009628963096556F8332054
:10502000954205D001330E2BF8D14F600F46C9E7EA
:10503000084F4C2202FB03774F600F46C2E7064A37
:10504000052008F0ADFCB5E728A20C082C4C0D0893
:10505000002E0024B82F0024544C0D0830B40C4C02
:105060000022234603E0013214330E2A0CD093F8B9
:1050700004C08445F7D1DD68294201D10029F2D16D
:10508000142303FB024000E0002030BC704700BF47
:1050900068050024F0B54468A37913F002025FD0DC
:1050A00002224FF0080C036864795B689B48204437
:1050B00093F83C40012C90F8080150D0012483F86B
:1050C0003C40142848D8DFE810F01500470047009E
:1050D000470084004700470047003B014700470066
:1050E0004700BB00470047004700F2004700470069
:1050F00047004D0018688A4C056A8A4E25F0020563
:10510000B04242EA0502056A25F0010505624768DA
:10511000856904EA050444F0600407D0824DA84282
:1051200004D005F57055A84240F04D8122F00802E8
:1051300047F440774CEA020222F00402476084619F
:1051400041630262826942F008028261826922F050
:105150000402826182698261002283F83C20F0BDF2
:105160009446A0E718686F4E046AB04224F4001415
:1051700044EA0252046A24F4801404626B4C4568C9
:10518000476D04EA070444F4C0440ED006F5806677
:10519000B0420AD0664F06F58046B04218BFB8420A
:1051A00003D006F58066B04201D145F48025456004
:1051B0004465C1650262426D42F400624265426D1F
:1051C00022F480624265426D4265002283F83C20F1
:1051D000C5E71868574C056A524E25F02005B042C5
:1051E00045EA0215026A22F01002026247688269EB
:1051F00004EA020444F4C04400F0DE804A4A9042CB
:1052000000F0DA804A4E4C4A904218BFB04203D0B8
:1052100002F58062904201D147F4406747608461A3
:1052200081630562826942F400628261826922F4CC
:105230008062826182698261002283F83C208EE76D
:105240001868384E046AB04224F4005444EA02322A
:10525000046A24F480540462364C4568C76904EA41
:10526000070444F4C0440ED006F58066B0420AD06C
:105270002F4F06F58046B04218BFB84203D006F55E
:105280008066B04201D145F480454560C461016447
:105290000262C26942F40062C261C26922F48062A1
:1052A000C261C269C261002283F83C2057E71868D6
:1052B0001C4E046AB04224F4003444EA0242046AF8
:1052C00024F4803404621D4C4568476D04EA0704E9
:1052D00044F060040ED006F58066B0420AD0144F48
:1052E00006F58046B04218BFB84203D006F5806686
:1052F000B04201D145F48035456044658165026264
:10530000426D42F008024265426D22F0040242659D
:10531000426D4265002283F83C2020E790A10C08F2
:105320008CFFFEFF0000014000040140FF8FFFFEE4
:1053300000400140FF8CFFFE004401408FFFFEFF54
:105340001868264C056A264E25F4007EB0424EEAC7
:105350000225026A22F4807202624768C26904EA86
:10536000020444F0600420D01E4A90421DD01E4E1C
:105370001E4A904218BFB04203D002F580629042AC
:1053800001D147F440574760C461C1630562C269F7
:1053900042F00802C261C26922F00402C261C2691D
:1053A000C261002283F83C20D9E625F4006E4EEA63
:1053B0000C2E2EF48065E4E725F0800545EA0C15F7
:1053C00025F0400528E705F58065A8423FF4AEAE1C
:1053D00005F58065A8427FF4B1AEA7E68CFFFEFF1D
:1053E0000000014000040140004001400044014031
:1053F00042685379032B0FD8DFE803F00B0805024E
:1054000010684030704710683C3070471068383082
:10541000704710683430704700207047D0E90002B0
:10542000064B517992790B44406893F80811530761
:1054300001D57AF06DB87AF0E7B800BF90A10C08FA
:105440004268C36812695B68C2F30322F0B5364C48
:1054500004EB82029668EFF31182102585F312881F
:105460004568324F95F805E0D0F80CC004EB4E04C7
:10547000D5F800E0258DDEF80C4005F4F05524EA5F
:105480000504CEF80C4017F806E0DCF8104053F89D
:105490000E501F2C25F0010543F80E5039D9203C41
:1054A0002025DCF804C005FA04F4CCF80C40D2B294
:1054B00082F31188BA5DDFF878C003EB020E46680C
:1054C0004569DEF8044004EA0C0C4CEA0101CEF810
:1054D00004107179032924D8DFE801F018151202AD
:1054E00031684031CEF80C500124CEF8081099589C
:1054F00041F0100199509958214399500474F0BD1E
:1055000031683C31EEE731683831EBE731683431EE
:10551000E8E72025DCF804C005FA04F4CCF80840DC
:10552000C5E70021DEE700BF90A10C0840A30C08EE
:105530000000FFFF03681A7E012A2ED0002293F894
:105540003010012909D093F8481001290ED093F8A2
:10555000601001291BD02ABB7047022142F48062EF
:1055600083F8301093F84810012904D1022142F445
:10557000006283F8481093F86010012907D01B6877
:1055800000211B685962D9680A43DA60704702211A
:1055900042F4805283F86010F1E702214FF4007268
:1055A0001976CCE74FF40072E9E700BF08B5204B4D
:1055B00098420ED003F5806398420AD01D4A03F545
:1055C0008043984218BF904203D003F5806398420D
:1055D0001BD1FCF761F81849184BCA69C969C2F3B5
:1055E0000222C1F302211A4492F8302002F01F0275
:1055F000D040114A1269C2F3C03241EAC2021344D8
:1056000093F80C3103FB00F008BDFCF745F80A499C
:105610000A4BCA69C969C2F3021CC1F3021103EB48
:105620000C0292F8302002F01F02D040E1E700BFE8
:1056300000000140004001400044025890A10C08C5
:1056400070B50E4605EE102AD0E90031013E1A6809
:105650000868B6B25C681568FFF7A8FF07EE900A05
:10566000B8EE455A9FED5D7AF8EE677A87EE850AC7
:1056700030EE070A7EF0A4FB23680138AB4280B20B
:1056800068D0C4E9005000238022E660A360A261D4
:10569000C4E9043394F83D3003F0FF02002B78D0C6
:1056A0000223211D284684F83D30FCF743FC4C4A78
:1056B0000123B5F1804FA5EB020284F84830B2FA1D
:1056C00082F284F83E3084F83F304FEA521284F878
:1056D000403084F8413084F8423084F8433084F814
:1056E000443084F8453084F8463084F8473084F8F4
:1056F0003D3034D09ABB3B4B9D420CD003F58063C8
:105700009D4208D003F580639D4245D003F5784360
:105710009D4241D070BD94F83C30012BFAD002225A
:10572000314B012184F83D20A8680340AB6084F828
:105730003D1084F83D206B68A96823F0700321F0C8
:10574000800101226B600023A96084F83D2084F869
:105750003C3070BD636883423AD0606093E794F850
:105760003C30012BD6D002211F4B002084F83D1085
:10577000A9680B400121AB6084F83D10022384F836
:105780003D306B68A9680AB90028D6D023F47003AD
:10579000D3E784F83C2083E794F83C30012BB9D060
:1057A0000221114B114884F83D10A968281A0B40BA
:1057B000B0FA80F00121AB600023400984F83D106D
:1057C00084F83C300A4B9D42D8D00028D6D170BD19
:1057D000E368B3427FF457AF70BD00BF0AD7233CE4
:1057E00000000140000400408800CEFF000401409A
:1057F000000C0040024B0348D3F88011FBF79CBD1E
:10580000002E002400000140034B4FF08040D3F8ED
:105810008411FBF791BD00BF002E0024024B03480A
:10582000D3F88811FBF788BD002E00240004004047
:10583000024B0348D3F88C11FBF77EBD002E0024E9
:1058400000080040024B0348D3F89011FBF774BDE9
:10585000002E0024000C0040024B0348D3F89C119A
:10586000FBF76ABD002E002400040140024B0348F0
:10587000D3F8AC11FBF760BD002E002400180040E7
:10588000024B0348D3F8B811FBF756BD002E002495
:1058900000400140024B0348D3F8BC11FBF74CBD5C
:1058A000002E002400440140024B0348D3F8C011ED
:1058B000FBF742BD002E00240048014010B5064C05
:1058C0000648D4F89C11FBF737FDD4F8B011044812
:1058D000BDE81040FBF730BD002E0024000401405D
:1058E000001C004010B5064C0648D4F89C11FBF78C
:1058F00023FDD4F8B4110448BDE81040FBF71CBDEB
:10590000002E00240004014000200040BFF34F8F10
:105910000549064BCA6802F4E0621343CB60BFF34B
:105920004F8F00BFFDE700BF00ED00E00400FA0567
:105930000021012008B50DF0BFFC72B6FFF7E6FFAD
:105940002DE9F043BFB0BFF35F8F9C4C0023626A28
:1059500022F480326262C4F894309DF843109DF8BE
:10596000445009069DF842200F9841EA057141EA2A
:10597000C2419DF8452041EA82419DF8462041EA16
:1059800042419DF8472041EA02419DF8412041EA09
:1059900002219DF8402041EA4201C4F898300133C9
:1059A000D4F8A020112B22F00102C4F8A020C4F8E2
:1059B0009C00C4F8A010F0D10523C4F89430636AA9
:1059C00043F480336362BFF34F8FBFF36F8F7C4824
:1059D0007C4A7D49121A82F051F9D4F888107B4B29
:1059E0000022012041F47001C4F8881018601A6187
:1059F000196841F08001196019680143196019683C
:105A000041F480311960196841F4805119609A613C
:105A1000DA611A629A62DA621A635A639A63DA6323
:105A20001A645A64196821F4802119601A664FF0CB
:105A300000636749C1F80801A3607AF0FDFE654A7A
:105A4000D36813F0040FD36840F0A380624B0021A9
:105A5000604A0591D96A21F00101D962DB6A03F03D
:105A600001030593936943F440439361936903F4FD
:105A700040430593059B93699E04FCD54C2200216D
:105A80000EA8564C83F022FA554A42F20303A4F1C1
:105A900010011268B3EB124F4FF000024FF00C03ED
:105AA00008BF0C460892E268A370002A4CD1494A0C
:105AB000494B916941F440419161926902F440423D
:105AC0000892DA6A42F00102DA62DB6A03F001034B
:105AD0000893089B3F4A93699D04FCD53B4B4FF4C8
:105AE000403540480321D3F8E02042F08002C3F85B
:105AF000E0200122D3F8E03003F080030793079BF6
:105B000085610D9BCDE9001300237AF043FD02234C
:105B100001204FF48031A288CDE917330C2319936B
:105B2000A379CDE90E01E079217A1C900EA81D9190
:105B3000CDE91A2308220023CDE91E23FAF712FF2C
:105B4000032838D0A0B1FEE7234BD96A21F0010128
:105B5000D962DB6A1F4903F0010308938B6923F4C0
:105B6000404313438B618B6903F440430893B0E7D0
:105B70001D4B1A6812F00E0F3AD11A6822F00F026C
:105B800042F002021A601B6803F00F03022B2FD0B1
:105B9000FEE723F00703154C43F00203D3602168AE
:105BA00005E023685B1AB3F57A7F3FF64FAF536881
:105BB0009F04F6D54AE7FFF7BBFE00BF00ED00E00B
:105BC00000000000C037000068CC0D0800440258F7
:105BD000008000510048025800040058900600243C
:105BE0000010005C001C025800200052002E00240F
:105BF0006C4A936903F070033F2B05D8936923F037
:105C0000700343F040039361664AD36903F0700365
:105C10003F2B05D8D36923F0700343F04003D361D1
:105C2000604AD36903F4E063B3F5806F05D2D369AA
:105C300023F4E06343F48063D3615A4A136A03F0A8
:105C400070033F2B05D8136A23F0700343F0400321
:105C50001362544B9A69140705D49A6922F00F0213
:105C600042F008029A614F4A936923F4706393618A
:105C7000136898018CD5136941F288314A4C23F09E
:105C8000070343F003031361206804E023681B1A31
:105C90008B4200F2A881136903F03803182BF5D169
:105CA000936903F00F03082B05D9936923F00F03C1
:105CB00043F0080393613D4A136803F00F03022B7E
:105CC0000BD9136823F00F0343F00203136013682A
:105CD00003F00F03022B00D05AE7324A936903F016
:105CE0007003402B05D9936923F0700343F0400300
:105CF00093612C4AD36903F07003402B05D9D36913
:105D000023F0700343F04003D361264AD36903F4C0
:105D1000E063B3F5806F05D9D36923F4E06343F4FE
:105D20008063D3611F4A136A03F07003402B00F2B3
:105D300052811C4EFBF78EFC1D4DB269B369C2F354
:105D400003221C4B134493F8303003F01F0320FA56
:105D500003F368682B60FBF78DFB002840F044815B
:105D60001023159017900EA80E93FAF7FBFD00284C
:105D700040F030813368104A43F080033360D6F836
:105D8000F43043F00203C6F8F430D6F8F43003F0F0
:105D900002030493049B136A43F001031362074B4D
:105DA000216810E000440258002E00240020005218
:105DB0000000002490A10C08000400588038010065
:105DC000013B3FF4F8AE22689142F9D02268236883
:105DD0009B1A0A2BFBD900214FF48020A64C4FF4CC
:105DE00040130026002730934FF00208CDE90E0142
:105DF0000EA879F0F5FCD4F8EC30A04941F203028A
:105E000043F002030EA8C4F8EC30D4F8EC3003F0F1
:105E100002030393039BD4F8943043F00203C4F8C5
:105E20009430D4F8943023F00203C4F894300B6813
:105E30009349B2EB134F934B934A28BF0A465A60DB
:105E40001A6822F47C5242F400521A601A6842F036
:105E500060021A6003220023CDE92C67CDE90E23EE
:105E600079F0BEFC4FF4E04200230EA8CDE926678E
:105E700000270326CDE90E233A9779F0B1FC1822CA
:105E800000230EA82F973497CDE90E2379F0A8FCB4
:105E90004FF4803200230EA81797CDE90E23052278
:105EA0004FF4FA73CDE91023042314934FF4803395
:105EB000CDE915772293CDE9128679F091FCD4F8DB
:105EC000E03042464FF4807143F001036F48C4F85C
:105ED000E030D4F8E03003F001030993099B3B461E
:105EE000CDE900677AF056FB23694246684823F003
:105EF000FE7343F088732361D4F8E03043F0040369
:105F0000C4F8E030D4F8E03003F0040306933B46D5
:105F100006994FF40071CDE900677AF03BFB2369E5
:105F200023F07E4343F0FC432361FBF793FB28609F
:105F3000BFF35F8F574C3E46574D4FF00108636AE1
:105F400023F480336362C4F8947028E0002A49D0B7
:105F50002F686B7A103515F8061C1B0643EA01738F
:105F600043EA420315F8052C43EA824315F8042C52
:105F700043EA424315F8032CC4F89860013643EA1B
:105F80000243D4F8A020032E43F0010322F00102C3
:105F9000C4F8A020C4F89C70C4F8A03025D06B6869
:105FA0002A7A002BD2D02F68002AD2D127F01F02E4
:105FB000A3EB0209B9F1200F38BF4FF02009484682
:105FC00081F0D2FD421E08FA02F1894508BF02465F
:105FD000D2B2BEE7FEE7136A23F0700343F040033A
:105FE0001362A6E6FEE7D3E5D2E50523C4F89430B4
:105FF000636A43F480336362BFF34F8FBFF36F8FE5
:10600000BFF34F8FBFF36F8F0022C4F85022BFF34E
:106010004F8FBFF36F8F636943F400336361BFF346
:106020004F8FBFF36F8FC4F88420BFF34F8FD4F826
:10603000805043F6E0761749C5F34E34C5F3C905E1
:10604000640104EA06002B4640EA8372013BC1F872
:106050006022F9D2203C14F1200FF2D1BFF34F8F10
:106060004B6943F480334B61BFF34F8FBFF36F8FA6
:106070003FB0BDE8F08300BF004402580010005C50
:106080007FBB2200008400407FBB2230000002580A
:106090000008025800ED00E0A00600243F4B586DB8
:1060A000012830B585B06ED03D494FF6FF003D4A1E
:1060B000CC683D4B04403D4D3D482243CA605A6F79
:1060C000C5F8E025D3F8F42042F00202C3F8F4202A
:1060D000D3F8F42002F002020392039AD3F8DC20F2
:1060E00042F00052C3F8DC20D3F8DC2002F000526A
:1060F0000292029AD3F8DC2042F08042C3F8DC20FE
:10610000D3F8DC2002F080420192019AD3F8DC201F
:1061100042F00042C3F8DC20D3F8DC20036802F030
:10612000004224480092009AD1F8FC40224A44F0F0
:106130008074C1F8FC40A2FB03420024920CC5F815
:10614000E4251E4AC0F8B02F1D4A4460A2FB032379
:1061500002689B0942F00102013B0260B3F1807FBB
:1061600007D34FF0E022136943F00403136105B035
:1061700030BD4FF0E022F0205361072381F8230067
:1061800094611361EDE700210DF096F80D4B1A684C
:1061900082F308885B689847FEE700BF004000581C
:1061A00000ED00E00003FA0500440258002E002430
:1061B00000000024001000E083DE1B4355CEACC578
:1061C000D34D62100098F01F2DE9F843384E9846E1
:1061D00006EB8003D3F81C41002C66D004F1D203F7
:1061E00006F59E760546B4F8D202A36104F5E9737C
:1061F00066601746E3614FF48073261DE160C4E9D1
:1062000004332368C4F8CC30A36300284AD194F83F
:10621000D1000CF07FFD18F0080F94F8D09034D125
:10622000BA0723D4FB0711D4052194F8D60270F0E5
:1062300089FC94F8D63201221E4903F01F005B0945
:10624000824041F823203046BDE8F88301354846B6
:106250000CF060FDEDB218B140F206630572C38028
:1062600094F8D42202210CF033FDDDE76B1CDBB285
:1062700018B1037240F20653C38094F8D52202216C
:106280000CF026FDFB07CFD5E0E70135EDB218B1E4
:1062900040F206730572C38094F8D52202210CF0F7
:1062A00017FDC1E76FF086FFB1E72646CBE700BFD9
:1062B00090A10C0800E100E00148FBF7E7BE00BF39
:1062C000D40600240148FBF7E1BE00BFAC0900245E
:1062D0000148FBF7DBBE00BF840C00240148FBF73C
:1062E000D5BE00BF5C0F00240148FBF7CFBE00BF46
:1062F000341200240148FBF7C9BE00BF0C1500246E
:106300000148FBF7C3BE00BFE417002470B5242288
:10631000456B00238168C0F8BC2004462A6800F160
:10632000340622F001022A602B606B60AB60827938
:10633000C0F8C43080F8B830C0F8BC30C364C0F8CE
:10634000C0304365C0F8A030C0F8A4309302816328
:1063500003F480534179C363130303F400530364CC
:10636000130203F480634364C36D01F00200C907A4
:1063700045D400287ED1A06412F0080254D0D4F88D
:10638000BC20002A00F08A802422C4F8BC202A689D
:1063900022F001022A60002B7CD13046FBF754FA30
:1063A000012812D06B68304623F490436B60AB68D1
:1063B00023F02203AB60AB6843F00803AB602B68AB
:1063C00043F001032B6079F043F86279D6070DD5CD
:1063D000D4F8C830196841F480711960996841F0A7
:1063E00001019960196841F020011960950705D5F0
:1063F000D4F8C820136843F08003136070BD0421F3
:10640000A16470B30C21D007A164B5D54FF48031DD
:1064100043F00203616643F001034FF40031E3658A
:10642000216612F00802AAD1D4F8BC1009B194F880
:10643000B82084F8B8202422C4F8BC202A6822F0AE
:1064400001022A6013BB3046FBF7FEF90128BCD0DD
:106450006B68304623F490436B60AB6823F02A03EB
:10646000ACE7D10788D543F002034FF48031E365F0
:10647000616681E70821A164D1077FF57DAF43F014
:1064800001034FF40031E3652166CAE73046FAF7AD
:1064900037FED8E73046FAF733FE7EE784F8B820B7
:1064A00072E700BF816031E741712FE781712DE70D
:1064B0002DE9F843434D3C20434C05F5B872B5F83F
:1064C0007631C4F8E825A4F8F435B5F87A21B5F8A2
:1064D0007E31A4F8F625A4F8EC350CF01BFC074639
:1064E00042200CF017FC064638200CF013FC8146C5
:1064F0001FB10D23FB8000233B721EB10D23F380DF
:1065000000233372B9F1000F05D00D23A9F806302E
:10651000002389F80830B5F882313920A4F8EE3527
:10652000B5F88631A4F8F035B5F88A31A4F8F2351B
:106530000CF0F0FB80463A200CF0ECFB05463B20CB
:106540000CF0E8FB0446B8F1000F05D00D23A8F8C5
:106550000630002388F808301DB10D23EB8000239E
:106560002B721CB10D23E3800023237248460CF0EC
:1065700081FB012148460CF089FB40460CF07AFB78
:1065800028460CF077FB20460CF074FB40460121B6
:106590000CF07CFB284601210CF078FB0121204601
:1065A0000CF074FB38460CF065FB30460CF062FBD7
:1065B000384601210CF06AFB30460121BDE8F84362
:1065C0000CF064BB90A10C08002E002438B5134DCC
:1065D00041F20D13124941F28832D5F83C06D5F844
:1065E000F8450004A060E068014020460B430D21FF
:1065F000E360FCF781F838B1D5F82C26034600207B
:106600001343C5F82C3638BD606900F4F050A0F58E
:106610000060B0FA80F0400938BD00BF002E0024B1
:10662000C0E0FEFF2DE9F04FA74D7C2200219BB07A
:1066300005F5BF6082F04AFC4FF48031D5F8E8459B
:1066400095F828362268C5F8FC154FF40031C5F8D6
:10665000F825C5F808160221C5F80C16002B00F025
:1066600088800422994B85F82826DA6C1B68D603AB
:106670000DD5180100F1D98001224FF0006385F893
:106680002826C5F82C3601201BB0BDE8F08F9C01F0
:10669000F2D50AAB18460193FBF7D6FA0B990029FD
:1066A000EAD0D5F8F8450A0A894B6668A3FB02329E
:1066B000884B894F33401009B94243EA1213636093
:1066C000236843F00303236040F2F9804300834AC8
:1066D000B1FBF3F3B2FBF3F2296802322B685B1AC9
:1066E0009A42FBD800237E4A0493A3607D4BE16865
:1066F00017680B4043F48053E3607B4BA3FB0737E1
:1067000041F288337F0A03FB07F73B46002B00F07A
:10671000CB80626B013B1106F8D5744B714AA363C1
:106720004FF4D573A360E3681A4041F20813134392
:10673000E3604FB13B46626B12F0450F02D092040A
:1067400040F1DC80013BF6D10023C5F83436A3606C
:10675000644BE268134043F48053E3603B46002BF4
:1067600000F0A280626B013B1106F8D55F4BA3637A
:10677000E3E05F4B9A425FD05E4B9A4200F00F819C
:1067800095F8F4050CF0C6FA834695F8F6050CF07A
:10679000C1FA824695F8EC050CF0BCFA814695F8F2
:1067A000EE050CF0B7FA804695F8F0050CF0B2FA59
:1067B000074695F8F2050CF0ADFA95F8F525064672
:1067C0000E2158460CF084FA504695F8F7250E2114
:1067D0000CF07EFA484695F8ED250E210CF078FA7B
:1067E000404695F8EF250E210CF072FA95F8F12548
:1067F00038460E210CF06CFA0E2195F8F325304640
:106800000CF066FA0221B4F9040070F09BF9B4F9B7
:106810000430002BFFF625AF03F01F0001225B09B7
:106820003549824041F823201BE70AAB1846019303
:10683000FAF770FF0C9932E7244BD3F8D42022F4F6
:106840008032C3F8D420D3F8D42042F48032C3F885
:10685000D420D3F8D42002F480320392039ADA6F62
:1068600042F48032DA67DA6F22F48032DA6787E73F
:106870002A684FEA134EA2EB09027346824213D8EC
:10688000002B40F03181C4F808E0E36803EA0A0312
:106890000B43E3603B46626B12F0450F02D092045B
:1068A00040F1F080013BF6D14FF00040012385F824
:1068B0002836D5F82C360343C5F82C36E3E6074ACC
:1068C000B2FBF1F2296808E7002E002400440258C8
:1068D000598B4F01002CC0FFFF340C001021010028
:1068E00000000024C0E0FEFFD34D6210C500200070
:1068F000007000520024024800E100E0636B5B0777
:1069000000F16F83636BDE0769D4636B580601D5B2
:106910004023A3630123704A37212046C5F834364B
:106920000023A360E3681A4041F23713134341F296
:106930008832E360FBF7E0FE70BB049A4FF6FE730B
:106940009A4200F23982DFF890A1DFF89881634E15
:10695000002241F2371337212046A260E26802EAA2
:106960000A02134341F28832E360FBF7C5FE0028B8
:106970009CD1C4F8088041F22913E26802EA0A02B5
:106980001343E36047B13B46626B12F0450F01D001
:10699000920427D5013BF7D14FF0805086E7504B4A
:1069A000D3F8DC2022F40072C3F8DC20D3F8DC201A
:1069B00042F40072C3F8DC20D3F8DC2002F4007249
:1069C0000292029AD3F8842042F40072C3F8842021
:1069D000D3F8842022F40072C3F88420D0E6012387
:1069E000A36397E7636B5B0758D4A6636269049B54
:1069F000002A03F101030493049B03DB4FF6FE71AD
:106A00008B42A5D904994FF6FE73994200F2178282
:106A1000500040F1D4814FF00108D5F80090C5F83E
:106A200030862368990700F0C4810023DFF8A8A00E
:106A30002046A36041F20233E26802EA0A021343ED
:106A4000E360FAF7BBFB00287FF430AF636941F2E3
:106A50000311C5F86436A369C5F86836E369C5F85B
:106A60006C36236AC5F87036A060E36803EA0A034F
:106A70000B43E360002F3FF417AFDFF860C041F233
:106A8000873007E7636B5B0722D4636BDE071CD498
:106A90002369DBB2032B06D0012007E704234FF064
:106AA0008050A36302E7C4F838C0636913F4604FF1
:106AB0003FF4DEAE590400F19D8213F4004F0CBF89
:106AC0004FF480304FF48050F0E60123A363E3E7F6
:106AD00004231846A363E9E6C0E0FEFFC5002000DA
:106AE00000440258000010C14FEA0E49C5F83CE6C8
:106AF000D44A2046C4F80890E3681A4041F20933AA
:106B00001343E360FAF75AFB00287FF4CFAE6269C3
:106B1000C5F85426A369C5F85836E769C5F85C7608
:106B2000216AC5F86016D4F818C04FEA1C5CC5F895
:106B300038C64FEA927C8DF828C0C2F3836C8DF87A
:106B400029C0C2F3016C8DF82AC0C2F3074C8DF83E
:106B50002BC0C2F3072CD2B28DF82CC08DF82D209B
:106B60001A0DADF82E20C3F303428DF83020C3F385
:106B7000C0328DF83120C3F380328DF83220C3F358
:106B800040328DF83320C3F300328DF834208DF875
:106B90003500B8F1000F00F01F811B0403F47C13D3
:106BA00043EA17430E934FF40073C5F844360E9B27
:106BB00001339B02C5F84036C5F84836C7F3803329
:106BC0004FF4007A20468DF84130C7F3C61307F022
:106BD0007F07C5F84CA68DF84230CB0F8DF8437077
:106BE00001278DF84430C1F341738DF84530C1F36E
:106BF00082638DF84630C1F383538DF84730C1F37B
:106C000040538DF8483000238DF84930C1F30043DC
:106C10008DF84A30C1F3C0338DF84B30C1F3803367
:106C20008DF84C30C1F340338DF84D30C1F3003353
:106C30008DF84E30C1F381238DF84F30C1F301231D
:106C4000C1F346018DF8503041F207138DF8511011
:106C500007218DF85270C4F80890DFF8E891E268D7
:106C600002EA0902134341F28832E360FBF744FD74
:106C700000287FF41BAEC4F808A041F2101BE368A3
:106C800041F288321021204603EA090343EA0B034C
:106C9000E360FBF731FD002840F0948095F828363A
:106CA000032B3FF4F0AC2F6863699A017ED44FF058
:106CB000400A41F2883210212046C4F808A0E36857
:106CC00003EA090343EA0B03E360FBF715FD002821
:106CD00043D1D5F83C36372120461B04A36041F24E
:106CE0003713E26802EA0902134341F28832E36093
:106CF000FBF702FD88BB4FF0FF330D216362C4F840
:106D000028A0E36A23F0FF0343F06303E36241F248
:106D10000D13A0602046E26802EA0902134341F223
:106D20008832E360FBF7E8FCB8B9019E04E02B6809
:106D3000DB1B013300F08A80636B13F4957F636B78
:106D400040F087801B04F2D506F12002D4F8803091
:106D500046F8043BB242F9D1E9E7D5F82C36C5F83C
:106D60002C36394B0122A363D5F82C3618434FF447
:106D70000073C5F82C06204685F82826A36041F24A
:106D80001013E1682F4A0A401021134341F2883260
:106D9000E360FBF7B1FC00283FF475AC2A4A0123FD
:106DA000A263C5F82C0685F828366CE44FF4006021
:106DB000D7E74FF0806079E5049A9A423FD84FF0C8
:106DC00000082AE6204BA363D5F82C360343C5F808
:106DD0002C3685F8287656E440F6FC7202EA8303E6
:106DE00043EA97730E93C7F3C2638DF83C30C7F341
:106DF00002638DF83D30C7F342538DF83E30C7F340
:106E000082438DF83F30C7F3C2338DF84030012301
:106E10000E9A9DF840001A4400F0070002308240AC
:106E20009DF8300000F00F00C5F840268340C5F8FB
:106E300044365B0A02FB03F3C5F84836BEE64FF062
:106E4000807033E5C0E0FEFFFF0FE01F4FF0004011
:106E500087E7180700F1C880636B990700F1C880C5
:106E6000636B9A0608D5C1E0D4F880202B6846F8F9
:106E7000042BDB1B0133E9D0636BDB04F4D40A9BE6
:106E80005E4AA263C3F381128DF81420C3F340124B
:106E90008DF815201A0A22F0FF0242EA1362DDE99A
:106EA0000B1392B209BAADF81620DAB206918DF83A
:106EB0001C20C3F307229DF83B108DF81D20C3F35F
:106EC00003521B0C8DF81E200D9A23F0FF03D0B245
:106ED00003432046ADF82030C2F385238DF82230DD
:106EE000C2F301238DF82330C2F3031302F00F0223
:106EF0008DF824304FF400738DF825208DF826107E
:106F00001021A3603E4AE3681A4041F21013134374
:106F100041F28832E360FBF7EFFB00287FF43EAFDD
:106F20009DF82430B8F1010F9DF82520DBB2D2B2D4
:106F300005D1134314BF4FF400784FF48078D5F88F
:106F40000406C5F850866FF04FFC00287FF49BAB19
:106F50002C6803E02B681B1B013330D06FF022FC40
:106F60000428F7D100230121D5F84026C5F82C3696
:106F7000C5F8243685F82816002A3FF484AB4FF470
:106F800080406FF031FC00287FF47DABD5F83036BF
:106F9000F3B1012B7FF477AB02201A4C85F874060D
:106FA000A4F124030FCB84E80F00A4F114031034E0
:106FB0000FCB84E80F0000201BB0BDE8F08F4FF02E
:106FC00000420123C5F82C2685F82836FFF75BBB65
:106FD000D5F83436002BE0D0012B7FF454AB1846A3
:106FE000DBE70423A36395E40820BAE62020B8E693
:106FF0000220B6E64FF4005058E400BF3A0F0018E4
:10700000C0E0FEFF78340024C74BD3F87816D3F8DD
:107010007C2670B58C0F93F87456100EC2F3072CB3
:1070200083F8A046C1F383640001012D83F8A146D3
:10703000C1F3016483F8A246C1F3074483F8A34671
:10704000C1F30724C9B283F8A446C2F3035483F8FA
:10705000A516A3F8A606C2F3C030B3F8A61689B2E7
:1070600041EA0401C2F30344A3F8A616C2F3403177
:1070700083F8A846C2F3803483F8A9064FF00000D5
:1070800083F8AA4683F8AB16C2F3003183F8AC1636
:10709000D3F8801683F8AD0640F2EF80022D00F0A1
:1070A000C3802A204FEA4C0C83F8B946C1F3C012C2
:1070B00001F07F010CF07E0C83F8BAC64FF0010C92
:1070C00093F8BA461443D3F8842683F8BA46D40F0B
:1070D00083F8BB16910D83F8BC46C2F3417401F0EE
:1070E0000C01C2F3815583F8BD46C2F3826483F874
:1070F000BE4683F8BF1693F8BF16D3F888462943D7
:1071000083F8BF16C2F3405183F8C016002183F8FC
:10711000C116C2F3004183F8C216C2F3C03183F82E
:10712000C316C2F3803183F8C416C2F3403183F82A
:10713000C516C2F3003183F8C616C2F3812183F865
:10714000C716C2F30121C2F3460283F8C816C4F37E
:10715000074183F8C926220E090283F8CAC683F8BC
:10716000CC26C4F30722A3F8CE162406B3F8CE1615
:1071700089B21143A3F8CE16D3F88C16C3F8D046C3
:107180000C0ED3F8D02642EA0442C3F8D0260A0AED
:10719000D3F8D04602F47F422243C1F30724C9B298
:1071A000C3F8D026D3F8D056D3F890262C43C3F892
:1071B000D04683F8D416110E83F8D516110C0906A3
:1071C000C3F8D8161102D3F8D8460A4601F47F0155
:1071D000214392B2D3F89446C3F8D816D3F8D81600
:1071E0000A43C3F8D826C4F30352D3F8D81641EAA9
:1071F0001461C3F8D81693F8DC161143C4F30722C0
:1072000083F8DC16210A01F47061A3F8DE16B3F8E6
:10721000DE1689B21143C4F34602A3F8DE1683F8E2
:10722000E02683F8E1C670BD1204C1F3072C0D0EF1
:1072300002F47C12C3F8B026C1F30742D3F8B0467B
:1072400044EA0524C3F8B046D3F8B04622434FF4CD
:107250000074C3F8B026D3F8B026C3F8F046013264
:1072600040F10004A40244EA92549202C3F8EC46AE
:10727000C1F38034C3F8E82614E74FEA8C2CC1F33D
:10728000C26594000CF44062C1F3072C04F47F74CF
:10729000C3F8B026D3F8B0261443CA0BC3F8B046DF
:1072A00002F00602D3F8B04644EA9174C3F8B0463F
:1072B000C1F3026483F8B456012583F8B546C1F3DF
:1072C000425483F8B646C1F3824483F8B746C1F30B
:1072D000C03483F8B82693F8B826224383F8B8263A
:1072E000D3F8B04693F8B82693F8A866023205FAA8
:1072F00002F2B540D617A2FB052EC3F8F05605FBE7
:1073000006EE04FB0EEE0134A2FB0424A644520A4E
:10731000C1F3803442EACE52C3F8E8264FEA5E2237
:10732000C3F8EC26BEE600BF002E0024704700BF65
:10733000704700BF704700BF01207047014B1868BD
:10734000704700BF00350024074B93F8A022012AA4
:1073500001D10020704793F8A002A0F10300B0FA19
:1073600080F04009704700BF00350024012380F8F9
:1073700049307047EFF31182702383F31288084974
:10738000D2B2D1E9B83182F31188581E8B42A0EBFA
:1073900001008CBF0023012300EB0330704700BFC6
:1073A0000035002470B5D0F8D442D0F8C86200EBA4
:1073B000840EDEF8C05245B301F00F040A4604EB18
:1073C000840C00EB8C0CDCF818306BB9DEF8C4329E
:1073D00000211B69C5F8141223B105F50471D5F815
:1073E00008029847002070BD04EBC40406EB840635
:1073F000F469B3FBF4F604FB1633002BE6D11A460E
:10740000CCF8183077F046FFECE7032070BD00BFE2
:10741000D0F8D42200EB820210B5D2F8C042ACB151
:1074200001F00F03D0F8C802D2F8C42204F50371AA
:1074300003EBC303D26800EB8303D4F80402D3F850
:107440006832C4F80C329047002010BD032010BDF4
:10745000D0F8D43200EB830010B5D0F8C04284B12C
:10746000D0F8C4325BB194F80002FF2807D09B68C3
:10747000214694F801229847FF2384F80032002027
:1074800010BD032010BD00BF30B52A4C86462378BE
:1074900065889D4241D9184619461A4602E0954230
:1074A00046D921780C440A44617892B20529F6D174
:1074B000A1788229F3D19C461A461E4903E0AA42CC
:1074C00034D291F800C06144624491F801C092B294
:1074D000BCF1050FF3D191F802C0BCF1010FEED160
:1074E000144A02E0A8421DD213781A44034492F8C9
:1074F00001C098B2BCF1050FF4D19378812BF1D182
:107500000CB11023A37119B10020022308714B7133
:107510001AB1002102231171537143230548AEF8BB
:10752000003030BD0022002CEBD1ECE70021D7E782
:107530000024C0E7B81A002430B52A4C86462378C8
:1075400065889D4241D9184619461A4602E095427F
:1075500046D921780C440A44617892B20529F6D1C3
:10756000A1788229F3D19C461A461E4903E0AA421B
:1075700034D291F800C06144624491F801C092B2E3
:10758000BCF1050FF3D191F802C0BCF1010FEED1AF
:10759000144A02E0A8421DD213781A44034492F818
:1075A00001C098B2BCF1050FF4D19378812BF1D1D1
:1075B0000CB11023A37119B10020402348710B7145
:1075C0001AB1002140235171137143230548AEF8CD
:1075D000003030BD0022002CEBD1ECE70021D7E7D2
:1075E0000024C0E7B81A0024A6E700BF03460A2219
:1075F00001481A80704700BFFC1A0024064B4FF068
:10760000120C064AA3F11400526DA1F800C0022A20
:1076100018BF1846704700BF1C1B002400400058CC
:10762000042301480B807047301B00241D48D0F80C
:107630000038D0F8082830B59B184FF01A040C8099
:1076400001D1194830BD184A0024D0F8040802F1CD
:10765000100511464FEA137EB3F1204FCC7001F1B3
:1076600002010EF1370C38BF0EF1300C8D424FEA9B
:10767000031381F800C0EDD102F108050024010FC9
:10768000B0F1204FD47402F1020201F1370338BF88
:1076900001F1300395424FEA00101374EFD1024814
:1076A00030BD00BF00E0F11F341B0024122301484D
:1076B0000B807047081B002400207047212808B564
:1076C00027D0222818D0202814D199B1072A11D107
:1076D000184A194B0868B1F804C0D2F8E822897931
:1076E000C3F89800A3F89CC083F89E1012B101461D
:1076F00000209047002008BD0029FBD0022AF9D1C4
:107700000C4BD3F8EC32002BF4D0098800209847BA
:10771000F0E70029EED0072AECD1074BD3F8980008
:10772000B3F89C2093F89E30086000208A808B710B
:1077300008BD00BF00350024B81A0024002070479F
:10774000034B93F81403003818BF0120704700BFA3
:1077500000350024034B93F81403032894BF002042
:107760000120704700350024004870471838002475
:10777000164B002030B493F82A4014B1DD698D42D5
:1077800005D0013010330828F5D130BC7047104BBC
:10779000BAB1D3F8601301EB40218A4201D1022C27
:1077A00008D093F8002512B9012283F800250122A0
:1077B00083F8492303EB0013012283F8722330BCC2
:1077C000704703EB001383F87223DEE74838002488
:1077D0000035002430B40023194C04F5527084F8AD
:1077E000EC3303E001331030082B1CD0C5698D4207
:1077F000F8D190F82AC0BCF1030FF3D1AAB1D4F8A4
:10780000601301EB43218A4208D094F8002512B995
:10781000012284F80025012284F8492304EB031493
:10782000012384F8723330BC7047D4F8E82304EBAA
:1078300003130421013283F87213C4F8E823F2E73A
:1078400000350024C0B1836823B10F4B072283F8B1
:107850004A2370470C4A042192F8480382F85C33AB
:10786000032882F84A13C2E9D53314BF4FF480735A
:107870008023C2E9D3337047034B012283F80025EC
:1078800083F84923704700BF00350024244910B510
:10789000B1F8A24091F8A0C0644531D96346A03147
:1078A000E646624603E0944238D991F800E071441C
:1078B000724491F801E092B2BEF1050FF3D191F854
:1078C00002E0BEF1810FEED1164A03E0A3421BD2C3
:1078D00092F800C06244634492F801C09BB2BCF1CC
:1078E000050FF3D192F802C0BCF1010FEED119B12E
:1078F000002402230C714B7100210223117153717A
:1079000020230380074810BD0029F9D0022300225C
:107910004B7120230A710380024810BD0021D3E778
:10792000B81A0024581B0024244910B5B1F8A2400D
:1079300091F8A0C0644531D96346A031E64662465D
:1079400003E0944238D991F800E07144724491F810
:1079500001E092B2BEF1050FF3D191F802E0BEF161
:10796000810FEED1164A03E0A3421BD292F800C069
:107970006244634492F801C09BB2BCF1050FF3D19D
:1079800092F802C0BCF1010FEED119B100244023DE
:107990004C710B710021402351711371202303801E
:1079A000074810BD0029F9D0402300220B71202385
:1079B0004A710380024810BD0021D3E7B81A0024A1
:1079C000581B0024244910B5B1F8A24091F8A0C07A
:1079D000644531D96346A031E646624603E09442ED
:1079E00038D991F800E07144724491F801E092B204
:1079F000BEF1050FF3D191F802E0BEF1810FEED197
:107A0000164A03E0A3421BD292F800C062446344CA
:107A100092F801C09BB2BCF1050FF3D192F802C0FD
:107A2000BCF1010FEED119B1002440234C710B7150
:107A3000002140235171137120230380074810BD9A
:107A40000029F9D0402300220B7120234A710380C2
:107A5000024810BD0021D3E7B81A0024581B0024A7
:107A600003460A2201481A80704700BF781B002491
:107A700038B5D0F8D432B03350F823507DB195F8F2
:107A80001C32044623B9D5F818320BB16B7A8BB18E
:107A90008121204677F078FA6B7A022B00D038BD2E
:107AA0002046812177F070FA20460121BDE8384058
:107AB00077F06ABA012177F067FA20468121BDE8A4
:107AC000384077F061BA00BFD0F8D42200EB8202D0
:107AD0002DE9F041D2F8C0420646002C4ED0B4F851
:107AE000643204F11007D4F870520846D2F8C42268
:107AF000394603FB05F5D2F81080B5F5007FD4F8C0
:107B00006C2228BF4FF40075B5FBF3F39BB2C0475E
:107B100000281BDB2B463A468121304677F0BAFB22
:107B2000B4F86422B5FBF2F2D4E99B1311449B1A1A
:107B3000D4F83822521BC4E99B13C4F8382213B17D
:107B40000020BDE8F08103232372F9E7D6F8D43290
:107B5000B03356F823208AB192F861320424112000
:107B600003F148010133DBB202F8314002EBC101FD
:107B7000A342888008BF002382F861324FF0FF30B3
:107B8000DFE700BF38B5084BD3F8703553B1DB6978
:107B900014460D4698474FF40073026800202A608F
:107BA000238038BD1B68FFDE0035002408B5064B76
:107BB000D3F8703523B11B699847013840B208BD2E
:107BC0004FF0FF3008BD00BF003500240020704793
:107BD000002070470A49D1F874350A685BB1002A61
:107BE000FCD0013A10B513F8014B0A60C1F87435A6
:107BF00012B1204610BDFEE76FF06AFB204610BDB3
:107C00000035002408B5064A0B68C2F874051360F5
:107C10000BB1002008BD6FF05BFB002008BD00BF6A
:107C2000003500242DE9F041012104464FF407708E
:107C300081F0F4FF054600286CD0D4F8D46204EB40
:107C40008606C6F8C002237CC4F8BC02002B40D0D4
:107C5000402302228121204677F08EF80121402323
:107C600002222046218777F087F84FF00108082389
:107C7000032282212046A4F8788177F07DF8294BF1
:107C80000027E364D6F8C432C5F804721B6898472D
:107C9000D5F80402C5F81472C5F8187200283ED051
:107CA000227CD4F8C83222BBC3F88C224FF4007473
:107CB0009A7903F51E71C3F88402012AA3F8788229
:107CC000C3F8884223D0186877F0D4F90020BDE8C3
:107CD000F08120464FF400730222812177F04CF8A6
:107CE00001214FF4007302222046218777F044F8E7
:107CF000BBE79A79402403F51E71C3F88C72012A00
:107D0000C3F88402A3F87882C3F88842DBD1C3F8B1
:107D10009402D8E7D4F8D432B03344F823000220D8
:107D2000BDE8F08101001000D0F8D432B03370B556
:107D300050F823402CB30026124B054684F83C1221
:107D4000C4F8303204F50C7226720D23812104F53B
:107D5000047477F09FFAD5F8C8321F220121C3F8C6
:107D60008C62A3F8781203F51E711868C3E9A1426A
:107D70009A79012A08BFC3F89442BDE8704077F0B1
:107D800079B970BD55534253D0F8D42200EB82022A
:107D90002DE9F041D2F8C0420646002C67D0B4F875
:107DA000643204F11007D4F870520846D2F8C422A5
:107DB000394603FB05F5D2F81480B5F5007FD4F8F9
:107DC0006C2228BF4FF40075B5FBF3F39BB2C0479C
:107DD000002834DBD4F83802B4F86422401BB5FB29
:107DE000F2F5D4E99B13C4F8380229445B1BC4E9BB
:107DF0009B13FBB1D6F8C80202FB03F3012200215A
:107E0000B3F5007FC0F88472A0F87822827928BF89
:107E10004FF40073C0F88C1200F51E71012AC0F8EF
:107E2000883208BFC0F89472006877F023F9002008
:107E3000BDE8F08119463046FFF776FFF7E7D6F840
:107E4000D432B03356F823208AB192F86132042438
:107E5000032003F148010133DBB202F8314002EBA9
:107E6000C101A342888008BF002382F861324FF02D
:107E7000FF30DDE7D0F8D43200EB83032DE9F04387
:107E8000D3F8C04283B0002C00F0B78016461278B9
:107E900005460F465A2A5FD85A2A00F29B80DFE82F
:107EA00012F04601990099005A0199009900990031
:107EB00099009900990099009900990099009900FA
:107EC0009900990099008E019900990099009900F4
:107ED000990099009900AC01CD01990099003D01EC
:107EE00099009900990099001002990036029900B2
:107EF0009900FA0099005E02990099009900990092
:107F0000E101990099009900990099009900990060
:107F10009900990099009900990099009900990099
:107F20009900990099009900990099009900990089
:107F30009900990099009900990099009900990079
:107F40009900990099009900990099009900990069
:107F5000990099009900F001A82A53D0AA2A00F0AC
:107F600064829E2A36D1D3F8C432084604F51972C9
:107F700004F51A715B6898470146002840F00983B0
:107F800094F86232022B00F00483D6F80A301ABA51
:107F9000E2601BB104F1100080F098FFD4F8683261
:107FA0000022013B190E61F30702190C61F30F2245
:107FB000190A61F31742B4F8641263F31F624BBAF3
:107FC0006383002362612383D6F80A301BBAE3601F
:107FD000002014E094F86122052620250221531C7C
:107FE0004832DBB204F8326004EBC200042B858017
:107FF00008BF0023617284F861324FF0FF3003B094
:10800000BDE8F08394F80880B8F1000F7DD194F9B1
:108010001C22002A80F2058394F86222022A00F0D2
:108020008083D3F8C43208469B689847002840F004
:10803000DE82D6F80230D5F8D4121BBAB031C4F8BB
:108040006C32D6F8062055F8211012BAC4F8702206
:108050000029D2D01344D1F86802834200F247834A
:10806000B4F8643202FB03F3D4F818229A424AD0DF
:1080700091F861320524202003F148020133DBB27C
:1080800001F8324001EBC202042B908008BF0023AC
:1080900081F86132B1E794F80880B8F1000F34D16B
:1080A00094F91C22002A80F2BC8294F86222022AEF
:1080B00000F03783D3F8C43238469B6898470028CD
:1080C00040F09582D6F80220D5F8D41212BAB03119
:1080D000C4F86C22B6F8073055F821105BBA9BB291
:1080E000C4F87032002988D01A44D1F86862B242CC
:1080F00000F27383B4F8642202FB03F3D4F818226D
:108100009A4240F0E182022323724FF40073394611
:108110002846E36003B0BDE8F043D5E4337900229C
:108120009B1AE26018BF012384F8623250E7D4F84A
:108130001822002A40F0398294F86212022900F0D5
:108140004683D3F8C43238469B689847002840F0ED
:10815000D382E0603CE7D4F81832002B00F025828F
:108160007021002294F8603221740C21C4F815208B
:10817000E17594F86112C4F811209942C4F81920ED
:10818000C4F81D2084F8212011D004EBC30191F81C
:108190004012A17404EBC3010133B1F84412DBB205
:1081A000A183042B14BF84F8603284F86022122368
:1081B000E36032799A4298BF1346E36008E7D4F847
:1081C0001822002A00F0F1817278D20740F1B181C3
:1081D000B378002B00F0CF81802B40F0E0810821A4
:1081E000CC4A04F1180304F11000E16012F8011DFB
:1081F00003F8011D8342F9D1EAE6D3F8C4323846C8
:10820000DB689847002840F074813279042A1346CD
:1082100028BF0423E360002A3FF4DAAE013BBD4AE5
:1082200004F1100099B201F111030A44234412F839
:10823000011903F8011D8342F9D1C9E694F86222BD
:108240003379012A03F0030300F06A81012B00F067
:108250006C81022B00F06A81032B00F06681002301
:10826000E360B5E6737813F0020340F09881D4E937
:108270009B210A44D4F868128A4200F2E581E36047
:10828000A6E6D3F8C4323846DB689847002840F0A9
:108290003881337A082B194628BF0821E160002B6A
:1082A0003FF496AE9C4A01F1100304F110000A4419
:1082B00054FA83F312F8011D03F8011D9842F9D115
:1082C00086E6D3F8C4320DF10202384601A95B6894
:1082D0009847002840F06F8194F86232022B00F03A
:1082E0006A81BDF802200821206152BA019BA06179
:1082F000013B62830C22E174E375190EE2601A0CF3
:108300001B0A217562750222A375227677E6D3F8DF
:10831000C43204F51972384604F51A715B6898473F
:10832000002840F0368194F86232022B00F031814F
:10833000D4F868320822A082013BE260190E1A0CC0
:1083400061F30700190A62F30F20B4F8642261F3A5
:10835000174052BA63F31F60E282206138E694F856
:108360000890B9F1000F40F00081D4F81822002ADB
:1083700000F08A8194F91C22002AC0F21582D3F8F9
:10838000C43238469B6898478046002840F0F18107
:10839000D5F8D432384605EB8303D3F8C432DB6812
:1083A00098470146002840F08281D6F80220D5F88F
:1083B000D40212BAB030C4F86C22B6F8073055F8BF
:1083C00020005BBA9BB2C4F8703200283FF415AEAF
:1083D0001A44D0F86862B24200F2C681B4F864224E
:1083E00002FB03F3D4F81822934240F0EC80B3F57B
:1083F000007F4FF0010004F1100428BF4FF4007318
:1084000004F8080C1A46D5F8C832C3F888229A79BD
:10841000C3F88C1203F51E718242C3F88442A3F89C
:10842000780262D1C3F894425FE0227A002A40F0D9
:108430009C80D4F81812002900F0838194F91C1252
:108440000029C0F22181D3F8C43238469B6898478E
:10845000D5F8D432002840F05A8105EB8303384622
:10846000D3F8C432DB689847002840F0F280D6F891
:108470000230D5F8D4121BBAB031C4F86C32D6F839
:10848000062055F8211012BAC4F8702200293FF4D2
:10849000B4AD1344D1F86802834200F22881B4F8E5
:1084A000643202FB03F3D4F8182293427FF4E0AD68
:1084B000B3F5007F4FF0010104F1100028BF4FF425
:1084C0000073217200241A46D5F8C832C3F88822F6
:1084D0009A79A3F8781203F51E71012AC3F8840271
:1084E000C3F88C4208BFC3F89402186876F0C2FD46
:1084F0006EE50A4A92F8DE3063F07F0382F8DE30E0
:1085000083E6064A92F8E33063F07F0382F8E330B3
:10851000BFE600BF941B0024981B0024B81A002457
:10852000022B3CD0012B7FF497AE002384F86232FB
:1085300095E6D3F8C43207EBC7013279D86900EB6E
:10854000810003790533934228BF1346E360002B73
:108550003FF43EAD03F110020344224413F8011D21
:10856000834202F8011DF9D132E53946284603B0AD
:10857000BDE8F04308E406219A4A04F1160304F129
:108580001000E16012F8011D03F8011D8342F9D1CA
:108590001EE53A220221284676F020FA2DE5242213
:1085A0000521284676F01AFA27E5202205212846DB
:1085B00076F014FA21E528463A22022176F00EFAE6
:1085C0004FF0FF301BE590F861320525202403F1C0
:1085D00048020133DBB200F8325000EBC202042B38
:1085E000948014BF80F8613280F8611205E5D5F8F7
:1085F000D432B03355F82320002A3FF4FEAC92F871
:10860000613202243A2003F148010133DBB202F85F
:10861000314002EBC101042B888075D082F86132B1
:10862000EBE494F861320520202103F14802013384
:10863000DBB204F8320004EBC202042B91807FF419
:10864000DAAC84F86182D8E42122052176F0C6F9FB
:10865000D3E4D5F8D432B03355F823208AB192F858
:1086600061320225272003F148010133DBB202F811
:10867000315002EBC101042B888008BF002382F82F
:10868000613205232372B8E494F861320525202075
:1086900003F148010133DBB204F8315004EBC101AE
:1086A000042B88807FF4A7AC84F86122A5E4D5F878
:1086B000D432B03355F82320002A3FF49EAC92F810
:1086C0006132022427209EE791F86132052520249B
:1086D00003F148020133DBB201F8325001EBC20270
:1086E000042B94807FF4D4AC81F8610285E491F886
:1086F000613205242120BFE43A220221284676F087
:108700006DF90523237278E482F8618275E4B03351
:1087100055F82320002AB4D092F8613202253A207D
:10872000A1E794F8613203F148010133DBB204F8A8
:10873000312004EBC1013A22042B8A807FF45BAC28
:108740007FE794F861320525202003F148020133C8
:10875000DBB204F8325004EBC202042B90807FF4A9
:108760004AAC84F8611248E490F86132052521246E
:108770002DE7D5F8D432B03355F82320002A3FF442
:108780003CAC92F8613202243A2003F148010133F3
:10879000DBB202F8314002EBC101042B88807FF488
:1087A0003DAF82F8619228E494F8613205202021DF
:1087B00003F148020133DBB204F8320004EBC202D9
:1087C000042B91807FF417AC84F8619215E43A226F
:1087D00076F004F9052323720FE491F86132052540
:1087E000212475E78A1B0024D0F8D432B03350F826
:1087F0002330CBB110B51A7A022A07D0033A012AE6
:1088000002D80021FFF790FA002010BD03F21F22CA
:1088100093F81D120446FFF72DFB0028F4DA01211E
:108820002046FFF781FAEFE700207047D0F8D432F6
:10883000B03370B550F8235025B12B7A044683B17C
:10884000012B01D0002070BD05F21F2295F81D12EA
:10885000FFF710FB0028F5DA01212046FFF764FA44
:10886000F0E7D5E98523C5F83832D0F8C832C5F825
:108870003422D3F88C321F2B04D12F4BD5F8102281
:108880009A421AD095F861324FF0050C202120460B
:1088900003F148020133DBB205F832C005EBC20236
:1088A000042B91804FF0020208BF00236A7285F802
:1088B0006132FFF7DDF8002070BD95F81D12012927
:1088C000E0D895F81E32013B0F2BDBD805F21F22B2
:1088D000FFF7D0FA00282B7A22DB013B022BB1D91B
:1088E000EE681EB3D4F8D432B03354F82310002904
:1088F000A8D02046D1F83842D1F8183205F110023C
:10890000A41BB342C1F838424FF0000428BF3346DD
:1089100081F83C4204240C72812176F0BBFC91E783
:10892000052B99D02046FFF7A3F88BE73146204668
:10893000FFF7FAF986E700BF55534243F8B5D0F880
:10894000C85240F20112044695F894342A87012B4C
:108950003ED00126002728683246314685F89464C7
:1089600076F018FD27873A4631462868A5F87862E0
:1089700085F8946476F00EFD4FF48173A4F8787155
:1089800032460221286885F89464A5F85C3076F0B8
:1089900001FD85F89474D4F8D432002504EB8303E8
:1089A000E564D3F8C0228AB1D3F8C4325B68984733
:1089B000D4F8D432B03354F8230080F0BFF9D4F89F
:1089C000D432B03344F82350C4F8BC520020F8BD70
:1089D00000224FF481710287A5F87832A0F878213F
:1089E000A5F85C10D7E700BFF8B5D0F8C85201264B
:1089F0000446002295F89434A5F87862B34227D053
:108A00003146286885F89464002776F0C3FC40F26C
:108A10000113A4F8787132463146286885F89464C9
:108A20002B8776F0B7FC85F89474D4F8D4320025FF
:108A3000B033258754F8230040B180F07FF9D4F893
:108A4000D432B03344F82350C4F8BC520020F8BDEF
:108A500040F20113A0F878212B87E6E7D0F8D43252
:108A600000EB8303F0B5002683B0D3F8C0728DF815
:108A70000560ADF806605FB191F800C004460D4690
:108A80001CF060022FD0202A05D0204676F0B8FADC
:108A9000032003B0F0BDCA884878002A42D01CF0F9
:108AA000800F00F08380D3F8C43239469B68984722
:108AB000EA8802234FF48071072AC4F8943228BF51
:108AC0000722D4F8C832C4E906225A629A799982F8
:108AD00003F11401012A1F629E6200D11F6318680E
:108AE00076F0C8FA22E04B780B2BCED801A252F8D0
:108AF00023F000BF318B04082D8B04088B8A0408F7
:108B00008B8A04088B8A04088B8A04088B8A0408E1
:108B10008B8A04088B8A04088B8A0408718B0408EA
:108B2000678B0408D3F8C4329B6898470020B0E7ED
:108B300090F89C32032BA8D10222D0F8C832002032
:108B4000C4F8942203F11401C4E906220DF10604CD
:108B50009862C3E908424FF480729A829A79012A96
:108B6000BDD11C63BBE790F89C32032BDED08CE7B1
:108B700090F89C32032B88D101220221D0F8C83210
:108B8000C0F8941203F11401C0E906220DF10500AA
:108B9000C3E908024FF4807200209A829A799862A1
:108BA000012A9CD10DF10500186398E7402A4FF087
:108BB000030387F8000228BF402287F80122C4F887
:108BC0009432D4F8C832C4F85821C4F85C2103F5B3
:108BD0001571C3F864229A79C3F86072012AC3F848
:108BE0006862A3F8546208BFC3F8707277E700BFE9
:108BF00008B520B904486DF0AFFA044808BD044830
:108C00006DF0AAFA014808BD704C0D08783A0024AE
:108C1000944C0D08024808B56DF09EFA014808BD55
:108C2000B84C0D08783A0024024808B56DF094FA63
:108C3000014808BDC04C0D08783A0024024808B528
:108C40006DF08AFA014808BDCC4C0D08783A002432
:108C500008B520B904486DF07FFA044808BD0448FF
:108C60006DF07AFA014808BDDC4C0D08783A002412
:108C7000FC4C0D08024808B56DF06EFA014808BDBD
:108C80001C4D0D08783A0024024808B56DF064FACE
:108C9000014808BD284D0D08783A0024554B0021A5
:108CA000554A1B685548A2FB032330B5DB0C544CD6
:108CB00083B0013BC4F88816C4F8801642F20F71E5
:108CC00094F8B526C4F87806C4F88416C4F87C363F
:108CD000002A00F08A8002254A49484884F8B5569F
:108CE000F9F728F90123484A0621372084F8C036CD
:108CF00084F8B63684F8B73684F8B83684F8B936CE
:108D000084F8BA3684F8BB3684F8BC3684F8BD36AD
:108D100084F8BE3684F8BF3684F8B536D2F8E83029
:108D200043F02003C2F8E830D2F8E83003F0200323
:108D30000193019B6DF006FF344B4FF400025A6023
:108D400094F8B536012B3BD1D4F87826304B314816
:108D5000B2F1804F18BF9A4284F8B556D1680CBF63
:108D60000123002341F00101824208BF43F00103C7
:108D700000F58060D160824208BF43F0010300F536
:108D800080602549824208BF43F0010300F5784026
:108D9000824208BF43F001038A4208BF43F0010347
:108DA00013B91E4B9A4207D191681D4B0B40062BFD
:108DB00006D0B3F5803F03D0136843F0010313607E
:108DC000D4F8D83204EB8303D3F8C43243B1154846
:108DD0000021154AC3F80802C3F81012C3F8042290
:108DE0000020C4E9BA0003B030BD02F0FF0084F8EF
:108DF000B40670E70000002483DE1B43001400402B
:108E0000003500247C3B00240044025800E100E0CF
:108E100000000140000400400018004000400140F4
:108E20000700010094560024944600242DE9F84FD1
:108E3000234E80468946D6F8C032D3F81422002A41
:108E4000FBD1B9F1000F37D008EB090ADFF874B095
:108E500008F1FF3870270AF1FF3AD6F8E42218F833
:108E6000011F531C0BF80210C3F30B03C6F8E432C6
:108E7000EFF3118287F31288D6E9B831D2B282F3C8
:108E800011888B42A3EB01038CBF0022012203EB6C
:108E90000233012B0ED10BF023FE04460D460BF0DE
:108EA0001FFE001B61EB0501B0F57A7F71F1000137
:108EB000F5D3DDE7D045D0D14846BDE8F88F00BFF7
:108EC0000035002494560024F8B50E4E96F8A032D2
:108ED000012B00D1F8BD96F8A032032BFAD10D4634
:108EE0001446D6F8C47608E0FFF7A0FFD6F8C436DB
:108EF000241A0544DB1B322BECD8002C21462846D3
:108F0000F2DCF8BD00350024F8B590F848305D1C5F
:108F10000344EDB280F8485083F8341090F849309B
:108F200053B1132D07D9002380F84830104F97F81C
:108F3000A032012B05D1F8BD80F84830002DF5D1C5
:108F4000F8BD97F8A032032BF5D1D7F8C46600F12D
:108F5000340429462046FFF769FFD7F8C4362D1A96
:108F600004449B1B322BE6D8002DF2D1F8BD00BF84
:108F700000350024F8B5002390F84850A0F8483098
:108F800005B9F8BD0D4F97F8A032012BF9D097F82D
:108F9000A032032BF5D1D7F8C46600F1340429467A
:108FA0002046FFF743FFD7F8C4362D1A04449B1B15
:108FB000322BE6D8002DF2D1F8BD00BF00350024D9
:108FC000F8B51F4FD7F8EC29B7F8F019D7F8703576
:108FD00091614BB39B69984730B30026D7F8703541
:108FE00013B11B69984790B9B6F57A7F25D00BF07D
:108FF00077FD013604460D460BF072FD001B61EB58
:109000000501B0F57A7F71F10001F5D3E6E7B6F519
:109010007A7F4FF0FF3018BF0020B7F8F039D7F84B
:10902000EC291B049361F8BD064B03F1E802D3F869
:10903000E830C7F870259847CFE74FF0FF30ECE7EE
:1090400000350024B81A00242DE9F84F344E90461C
:109050009A46B6F8FC29D6F8F8491304A361BAF188
:10906000000F50D0C8EBC853C24406F52A6901EB83
:10907000432B41F28937D6F870255AB10023546842
:10908000494640461A46A047A8B9D6F870350BB1F4
:109090001B699847013F3AD00BF022FD04460D466C
:1090A0000BF01EFD001B61EB0501B0F57A7F71F13D
:1090B0000001F5D3DFE741F28937D6F8703513B1F7
:1090C0001B69984780B9013F21D00BF009FD044688
:1090D0000D460BF005FD001B61EB0501B0F57A7F35
:1090E00071F10001F5D3E8E70BEB482008F1010826
:1090F0004FF4007249467EF0C1FDD045B9D1D6F893
:10910000F849B6F8FC290020A261BDE8F88FD6F82E
:10911000F8394FF0FF30B6F8FC299A61BDE8F88FB6
:10912000003500242DE9F84F364E90469A46B6F8A1
:10913000FC29D6F8F8491304A361BAF1000F54D002
:10914000C8EBC853C24406F52A6901EB432B4FF420
:1091500000720BEB482148467EF090FDD6F8702552
:109160000AB341F289370023D468494640461A467B
:10917000A047D6F87035B8B10BB11B699847013FCD
:1091800037D00BF0ADFC04460D460BF0A9FC001BDC
:1091900061EB0501B0F57A7F71F10001F5D3D6F8E6
:1091A0007025002ADFD1002341F2893713B11B69F2
:1091B000984790B9013F1CD00BF092FC04460D4635
:1091C0000BF08EFC001B61EB0501B0F57A7F71F1AD
:1091D0000001F5D3D6F87035E8E708F10108D0456D
:1091E000B5D1D6F8F849B6F8FC290020A261BDE84F
:1091F000F88FD6F8F8394FF0FF30B6F8FC299A61AD
:10920000BDE8F88F0035002410B5104CD4F8403379
:1092100023B119689A880B691A420AD0FDF702FA3D
:1092200038B994F808330133DBB2072B84F80833DC
:1092300003D9002384F8143310BDD4F8C4260123C5
:10924000C4F8042384F8143310BD00BF0035002493
:1092500010B50D4CD4F8403323B119689A880B69C6
:109260001A420CD0FDF7DEF948B9D4F8C426012320
:10927000A4F80803C4F8042384F8143310BD0023B1
:1092800084F8143310BD00BF0035002470B5174DAD
:109290000021174E6B6C2C681B04C6F81013154A7E
:1092A0000D21A3602046E3681A4041F20D131343D9
:1092B00041F28832E360F9F71FFA58B16B6B034350
:1092C0006B63D6F8C42609230020C6F8042386F869
:1092D000143370BD636903F4F053B3F5006FF0D13C
:1092E0000423022086F8143370BD00BFF833002435
:1092F00000350024C0E0FEFF70B50D4D04460E465B
:1093000095F81433042B0BD0082B07D1D5F80C3368
:1093100083420AD0FFF7BAFF022801D0012070BDB6
:109320000823C5E9C34685F81433022070BD00BF89
:109330000035002470B58A4C94F814536B1E082B2A
:109340001ED8DFE803F0796C7D1D4F05361D270020
:10935000844B5B6A002B6DD10722D4F8C436D4F855
:10936000FC5284F81423C4F80433002D62D0D4F8DE
:1093700000330120D4E9BC21A84794F814536B1E94
:10938000DBB2022B4FD9042D18BF082D0CBF0120D2
:10939000002070BDFDF71AF9002840F0D680D4F8FF
:1093A0000433D4F8C426FA339342ECD2FFF72CFFEF
:1093B000C2E7FDF70BF90028F1D0D4F810330022F2
:1093C000012B84F8082340F2C480D4F80C23013B1D
:1093D00008210132C4F8103384F81413C4F80C23A4
:1093E000012070BD5F4B1E6A002E6DD1FDF7EEF8B7
:1093F000002871D00423D4F8FC5284F8086384F860
:109400001433002DECD0D4F800333046D4F8F022D9
:10941000D4F8F412A84794F814536B1EB0E76DF01B
:10942000C1F9042867D0D4F8C436D4F804239B1AB1
:10943000C82B7FD8002070BD022384F814337BE74B
:10944000FDF7E2FD0028EED1474B0421C4F81003DC
:1094500093F82C2084F81413D88D196B84F81E23EC
:10946000090E1A6BA4F81C03120C84F81F13196B55
:10947000186B84F82023090A84F8220393F8340037
:1094800093F8352084F82113120984F8230393F804
:10949000350084F82823996B00F00F00DD8FDA8FF8
:1094A000C4F82413D98FC2F30B1384F8290343EAB9
:1094B000152301F00F0203F00F0384F82C2303F5AA
:1094C000FA63A4F82A3337E7D4F80433D4F8C4266F
:1094D00064339342BFF457AFFFF796FED4F8FC52C3
:1094E000002D3FF429AF0022D4F80033D4F8F41251
:1094F0001046A84720E7FDF787FD002893D11B4BB6
:109500001B78002BA3F10203B3FA83F308BF0125F4
:109510005B0984F80A5384F80B33FDF775FD0028C6
:109520007FF444AF104B03229B6C84F81423C4F8DF
:10953000183301E7FFF768FE94F81403042818BFF6
:1095400008280CBF0120002070BD042384F81433C8
:1095500046E7FAD1FFF79AFE94F814536B1E0FE713
:109560000035002478340024A0340024743400240E
:109570002DE9F04106460D4690461F46624C94F890
:109580001413042905D0082900F08C800120BDE8BF
:10959000F08106220123C4F8FC8284F814235B4A7C
:1095A00084F8F8325362EB06C4F80073C4E9BC5681
:1095B00062D1BFF34F8F564A05F500712B46C2F8B2
:1095C000683220338B42FAD1BFF34F8FBFF36F8FD6
:1095D000002D00F09280DFF8448198F83030012BA4
:1095E0004AD1731CD8F8501000228B42C8F834209E
:1095F00074D80323D8F80070C8F81C50182188F8D4
:1096000030304FF40073FA623846C8F82030D8F88A
:109610003830404A012B4FF0FF337B624FF4007328
:1096200018BF7602BB62FB6A23F0FF0343F090038E
:10963000FB62FB6843F04003FB609023BD6501259E
:109640003D65C8F82C30BE60FB681A4041F2181323
:10965000134341F28832FB60F9F74EF8002844D0FA
:109660002D4B0022BB63D8F834300343C8F83430A4
:1096700088F83050C8F82C2094F80933022B1CD8F5
:10968000013384F809330BF02BFA04460D460BF036
:1096900027FA001B61EB0501B0F57A7F71F100013B
:1096A000F5D373E7D4F80C33B3423FF472AFFFF74E
:1096B000EDFD02283FF463AF68E7002684F80963F4
:1096C000FFF7A2FDD4F8FC5235B1D4F8003332468E
:1096D000D4F8F4120120A847032058E7D8F8343012
:1096E00043F00073C8F83430C6E7FB6B84F8090315
:1096F00043F48D73FB63BDE8F081084A536B43F07C
:1097000000635363B8E700BF0035002478340024B9
:1097100000ED00E0C0E0FEFFFF0FE01FF833002483
:109720002DE9F84F664F0C468046164697F81413FD
:109730001D46042908D0082902D00020BDE8F88F72
:10974000FFF7A4FD0228F8D114F01F016AD101220D
:109750005C4B5D489A6002624FF40072C7F8A04CFF
:109760005A60002C00F09E80DFF868B19BF8303022
:10977000012B57D108F10100DBF85030CBF8341041
:10978000984200F295800323DBF800A04FF0010916
:109790008BF830305046DBF83830CAF82C101121E5
:1097A000012B4FF0FF33CBE90942CAF824304FF4C4
:1097B000007314BF4FEA48224246CAF82830DAF84C
:1097C0002C3023F0FF0343F09203CAF82C30DAF870
:1097D0000C3043F04003CAF80C308123CAF85840DB
:1097E000CAF85090CBF82C30CAF80820374ADAF87B
:1097F0000C301A4041F21113134341F28832CAF877
:109800000C30F8F779FF0346A0B3314ACAF8382084
:10981000DBF8342013430022CBF834308BF830903F
:10982000CBF82C2097F80933022B11D8013387F895
:1098300009330BF055F904460D460BF051F9001BA6
:1098400061EB0501B0F57A7F71F10001F5D374E7A2
:10985000002587F80953FFF7D7FCD7F8FC42002C06
:109860003FF46BAFD7F800332A46D7F8F4122846F6
:10987000A04762E787F809330522DAF83C3048460A
:10988000C7F8FC6243F49573C7F8005387F81423B4
:10989000CAF83C30D7F8C436C7E9BC48C7F8043327
:1098A000BDE8F88F0B4A536B43F000635363B9E78D
:1098B000DBF8343043F00073CBF83430B2E700BF4C
:1098C00000350024A041002478340024C0E0FEFFCD
:1098D000FF0FE01FF83300242DE9F04104464FF458
:1098E0001D707FF023FA054600285BD0D4F8D472AF
:1098F00004EB8707C7F8C002237CC4F8BC02002B26
:1099000045D0402302220121204675F035FA01227C
:1099100040234FF001082046A4F87821812102223B
:10992000002675F029FAA4F83880D7F8C4323046FA
:109930002E81A5F8606285F862621B689847D4F8AA
:10994000C84294F894342768434508D03846F8F75D
:109950009DFF41463846F8F771FF84F8946405F599
:1099600004751F220023384604F51E71C4F88C329A
:109970000123C4E9A152A279A4F878329A4208BF1F
:10998000C4F8945275F076FB0020BDE8F0814FF4E6
:10999000007302220121204675F0EEF901224FF4F6
:1099A0000073B6E7D4F8D4320220B03344F8235021
:1099B000EBE700BFF0B5002383B0ADF80630D0F878
:1099C000D43200EB8303D3F8C0524DB10A78044679
:1099D00012F0600036D0202805D0204675F010FB2C
:1099E000032003B0F0BD4878FE2849D0FF28F4D109
:1099F0004B88002BF1D1CE88002EEED11006ECD48E
:109A00004FF4807381212B8105F50475D4F8C84289
:109A1000204676F065FD2046012176F061FD1F228B
:109A2000012304F51E712068C4F88452A4F878322A
:109A3000C4E9A226A2799A4208BFC4F8945275F0EC
:109A400019FB46E04B780B2BC7D801A252F823F044
:109A5000D79A0408479B0408DB990408DB9904089B
:109A6000DB990408DB990408DB990408DB990408F6
:109A7000DB990408DB9904080F9B0408C79A0408C3
:109A80004E88002EA9D1CF88012FA6D11206A4D5C9
:109A9000D3F8C4329B699847022328604FF4807141
:109AA000C4F89432D4F8C832C4E906779A79998216
:109AB00003F11401012A5F621D629E6241D01868A1
:109AC00075F0D8FA05E094F89C32032B85D18B7899
:109AD0006B60002085E794F89C32032B7FF47DAF08
:109AE0000222D4F8C8320020C4F8942203F11401F1
:109AF000C4E906220DF106049862C3E908424FF456
:109B000080729A829A79012AD9D11C63D7E794F896
:109B10009C32032B7FF461AFD4F8C83201220221BA
:109B200004350020C4F894124FF48071C4E9062271
:109B3000C3E908529A79998203F11401012A9862C3
:109B4000BDD11D63BBE794F89C32032BC1D14B8878
:109B5000002BBED1D4F8C8628F8896F89434012BBC
:109B60000AD001233906306886F8943410D4F8F707
:109B70008DFE002386F894346B7A022B0DD03A06C2
:109B8000A7D5012BA5D001212046FEF7CDF8A0E7EF
:109B900007F00F01F8F752FEEBE72046812175F040
:109BA000F3F90121204675F0EFF992E76CF056BC0D
:109BB0006CF054BC10B51C2009F0ACF8044611211F
:109BC00009F064F8204609F05BF8C8200AF0B6FFF7
:109BD0002046BDE8104009F04DB800BF2DE9F04F18
:109BE000DFF804B38BB0DBF8ACACDAF8143013F068
:109BF000010902D00BB0BDE8F08FDAF81420DAF8D2
:109C000018301A42F6D0DAF808380AF50062C3F3C1
:109C10000D2301920BF58052C2F88031DAF814302E
:109C2000DAF8182013409D0705D5DAF8143003F050
:109C30000203CAF81430DAF81430DAF818201340A6
:109C4000DC061BD5DAF8183023F01003CAF81830F8
:109C5000DAF8203003F4F01203F00F01B2F5802F90
:109C600000F06785B2F5402F00F03E83CDF800A0EC
:109C7000009A936943F01003936101E0CDF800A0CE
:109C8000009A536992691340180300F1AC82009A5C
:109C90005369926913405F0300F1E081009B5A69A8
:109CA0009B691A4200F1F180009A5369926913404E
:109CB0001B0509D5019B9B68DF0700F18285009A8F
:109CC000536903F40063536100994B698A69134037
:109CD0001E0119D54B690A4603F000634B618049A8
:109CE00091F87831002B00F0D8827D4BD3F88C317D
:109CF00093F89C22042A04D093F89C22D2B283F8D1
:109D00009D22042283F89C22009A53699269134091
:109D1000DD0400F15381009A5369926913409C0459
:109D200000F1E480009A536992691340190700F129
:109D3000C98000994B698A6913401A0600F1818035
:109D40004B698A691340DB022AD59BF8B08CB8F1C5
:109D5000010F20D9634B0293029E0AF51267012579
:109D600004E0013520372436454514D096F83C30C0
:109D70003A68012BF5D1002AF3DA65F07F0086F806
:109D80003B30C0B26DF0EAF9EBE7009A5369926993
:109D90001340DA0204D5009A536903F48013536127
:109DA000009A5369926913409F0232D59BF8B07CA8
:109DB000012F29D90AF532624A4B012003E0B8424B
:109DC00003F1240320D093F87C1201301468203270
:109DD0000129F4D1002CF2DA414DD5F8805185EA01
:109DE0001445EE07EBD483F87B12DAF8181041F033
:109DF0008001CAF81810DAF814100D06DFD4019AA1
:109E0000536843F400735360009A536903F40013DA
:109E10005361009A5369926913405C0000F1C88055
:109E200000994B698A69134058077FF5E3AE4C6887
:109E3000610700F1D784DBF8AC3C5A6814435C60DE
:109E4000D8E6DAF818309BF8B07C23F08003012FB5
:109E5000CAF8183099D9234B01251E46029303E016
:109E600001352436BD4207D096F87B32012BF7D15D
:109E7000E8B26DF073F9F3E7009B5A699B691340F0
:109E8000DB028DD59BF8B08C66E7019A536823F00E
:109E900001035360124B93F87831012B00F01182CB
:109EA0000F4BD3F88C3193F89C22042A04D193F8F9
:109EB0009D22D2B283F89C22009A536903F000439A
:109EC0005361F1E6064BD3F88C0190F89C32032BDA
:109ED00000F0FC81009A536903F00803536128E7FE
:109EE00000450024AC41002400350024009AD2F83B
:109EF00000396FF30A03C2F80039D2F8043843F48A
:109F00008073C2F80438D2F80838980700F101824B
:109F100013F0060F0CBF00230F238BF8B33CF7F7A9
:109F2000BBFB9BF8B36C022E00F082844FF41053FD
:109F30000099003ECA6818BF012622F47052CA6018
:109F4000B34AD2F88C51CA681343CB600123002175
:109F500085F89C32D5F8B8326960C5F8A41285F846
:109F6000A012C5F894121BB15B680BB12846984744
:109F700000224024012740231146284674F0FCFEAD
:109F80002346002280212846C5F86041A5F8647167
:109F900074F0F2FE9E4BDBF8AC2CD3F88C31AF841E
:109FA0002C621E745369009203F400535361B9E6A6
:109FB000009A536903F08043536131E7019A1021FD
:109FC0000098536823F001035360F8F737FC9BF8BF
:109FD000B00CE0B10AF510634FF67F31996009F1DA
:109FE00001091A682033814522F4001243F8202C1D
:109FF000C3F8E811D3F8E02122F40012C3F8E021FD
:10A00000D3F8E02142F00062C3F8E021E6D1019AE2
:10A01000D36943F00113D3619BF8BB3C002B00F0E4
:10A020004581019AD2F8843043F00B03C2F88430A2
:10A03000536C43F00B035364DAF80038009C23F4AC
:10A04000FE63744A2046CAF800389BF8B21C74F0CC
:10A0500015FF636903F4805363615CE6009AD2F8EC
:10A060001878D2F81C381F40BFB2002F3FF416AE4C
:10A07000694D0AF510614FF00008CDF80CA01346A9
:10A080008A4644460295CDF8109008E07F0804F116
:10A09000010405F124050AF1200A00F03C81FE07C5
:10A0A000F4D5D3F8102804F00F01D3F834684FEA40
:10A0B0004419CE40F601F6B2164303F5106202EBE6
:10A0C000441292681640E2B2F007009222D50120B5
:10A0D000019A00FA01F1526B22EA010201994A63E6
:10A0E0009BF8B21C4A4A8142CAF80800D2F88C8117
:10A0F00000F088832B6A0593002C40F00883D8F881
:10A100009432022B00F0FC8398F8A03213B10023A4
:10A1100088F8A032320702D50823CAF80830F306BF
:10A1200002D51023CAF80830700602D54023CAF8B9
:10A130000830B10700F117813206DBF8AC3CA5D539
:10A14000D5E909068642A1D8811BEA6903F5106E9C
:10A150008A42CE4428BF0A46DEF81810033289B27C
:10A16000B1EB920F31D39BF8B28C03F5805C009475
:10A1700042460CEB043C98461346B04240F2A3839F
:10A18000811BEA69914228BF11462A6A01F103093D
:10A190004FEA990973B98CB20334A4080AD002EBD0
:10A1A000840452F8040BA242CCF80000F9D12A6AC8
:10A1B000D5E909060A440E442A62DEF81820AE6288
:10A1C00092B29145D9D9009C4346B0423FF65EAF6A
:10A1D00004F00F0201219140D3F8342822EA010251
:10A1E000C3F8342852E70098D0F81838D0F81C2863
:10A1F00013401F0C3FF44BAD074B0AF53066CDF80A
:10A200000CA04FF000089A460293CDF814900DE090
:10A210000045002448460024AC4100247F0808F192
:10A22000010806F120060AF1240A78D017F0010986
:10A23000F4D05FFA88F300F530624FEA48150093D6
:10A2400002EB48139C68D0F814180C40E1076CD45A
:10A25000210700F19480E50601D51023B360A00723
:10A260000FD5039B5B69190604D5019A536843F423
:10A27000806353609AF85732012B00F02783022342
:10A28000B360A20601D52023B360A30402D54FF426
:10A290000053B360DBF8AC0CC0E7012381F87831E0
:10A2A000536DC3F38303C1F87C312DE5019942F26C
:10A2B0002B034A6913434B610B6943F00B030B619A
:10A2C000BAE60023B64A82F87831F5E5D0F8B8321C
:10A2D000002B3FF4FFADDB69002B3FF4FBAD98474B
:10A2E000DBF8AC3C0093F5E501EBC101C3F30A13C5
:10A2F000AB4C0BEB81020AF58051D2F8140F0344EA
:10A300000868C4F848010968C2F8143FC4F84C1141
:10A31000ACE4022301E6DDE903A90093BEE4DDF825
:10A320000CA0DDF814900090B1E40121B1609BF81D
:10A33000B21CD0F840E00129D3F808C000F0B38285
:10A3400098498E4500F0AA83DBF8103F58EA0303D2
:10A3500000F05984924BDAF860220099D3F88C010E
:10A3600074F0BEFF74E721460398F8F767FAEB7DB7
:10A37000012B00F0C7830223CAF80830DCE6DBF8C3
:10A38000AC2C0823B36002F53063126C2B441046EA
:10A390000492854A9968904204D90A0402D54FF480
:10A3A00000429A607E4AD2F88C5192F8483105F208
:10A3B000AA2085F8AA3292F849E1079085F8ABE225
:10A3C000B2F84A11A5F8AC1206910121B2F84CC1BD
:10A3D000A5F8AEC2B2F84E21C5F8941203F01F01E1
:10A3E000A5F8B0220129C5F8982200F0B18202290F
:10A3F00000F01383002940F0EA8203F06003202B71
:10A4000000F0F783402B00F0F483A3B9BEF1090FED
:10A4100011D8DFE81EF0F400CD001000E4001000B9
:10A4200081006700100041002500D5F8B4325B6957
:10A43000002B40F0D485284674F0E2FD5A4B049A74
:10A440009A427FF608AF9BF8B21C01297FF403AF54
:10A45000029BDBF8AC0C03F29C4274F00FFDFAE6B1
:10A460009DF81890514BB9F1010F83F89890E2D8FC
:10A4700095F89C22D1B2022A069100F01785032993
:10A4800000F0E984284674F0BBFDD5F8B83249469F
:10A4900028465B689847D1E7012ACCD195F89C12F1
:10A4A0000229CBB200F2B884002BC4D0D5F8C83250
:10A4B000002128464FF0020C40F8081FC5F894C24E
:10A4C000C5E90622C3E9092118624FF4807203F13D
:10A4D00014019A829A79012A08BF1863186874F0E7
:10A4E000C9FDABE7069B00221B0AADF82620013B05
:10A4F000062BA0D801A252F823F000BFE1A6040861
:10A50000C5A604089BA6040837A4040837A40408B9
:10A5100039A60408F3A6040852EA0C0C8BD1069B5A
:10A520007F2B88D895F89C32032B84D00698D5F8D9
:10A53000C8325FFA80F985F89E9293F89424012A34
:10A5400012D01A684FF0000C83F81190D2F800185E
:10A5500021F4FE61C2F80018D2F8001841EA001197
:10A56000C2F8001883F894C40422002003F11401F7
:10A57000C5F894224FF48072A8619A829A79986201
:10A58000012AC3E9080008BF1863186874F072FD57
:10A59000B9F1000F40F08584012385F89C324DE726
:10A5A000004500240A31544F0A30544FF845002426
:10A5B00095F89C32013B022B3FF63DAF069B012BE9
:10A5C0007FF43CAF0020D5F8C832C5F8A402A861DA
:10A5D0000422C5F894229862C3E9080075E7069B37
:10A5E000012B00F07A84069B022B7FF424AF4FEA04
:10A5F0001C2CD5F8C832002085F8A0C2E7E795F8F2
:10A600009C32013B022B3FF616AF022A7FF413AFB8
:10A61000D5F8A4322846002B18BF4FF0030940F8A4
:10A620000C9FD5F8C832C5F89422C5E90622C3E9C3
:10A63000080200229A6248E72B7C002B7FF4FBAED5
:10A64000D5F8B8320DF126005B6B98470346B5F894
:10A65000B002002800F04484BDF82620002A3FF410
:10A66000EAAE82424FF0020128BF0246D5F8C80286
:10A67000C5F8941200F11401C5E90622C0E90832B8
:10A68000002282624FF4807282828279012A08BF9E
:10A690000363006874F0EEFCD0E69DF8180005280E
:10A6A0003FF6C9AE01A353F820F000BF17B004086D
:10A6B00009B00408FBAF0408EDAF04082BA404089C
:10A6C000D3AF04082A7CD5F8B832002A40F07E8443
:10A6D0009B6A0DF126009847022203464270B6E7B6
:10A6E000D5F8B4320DF12601287C1B689847034643
:10A6F000ADE72B7C002B7FF49EAED5F8B8320DF180
:10A7000026001B6B98470722034642709FE798F884
:10A710009C32032B7FF4FEACD8F8B8325B69002B77
:10A720003FF4F8AC002240460099C8F8D42298477C
:10A73000F0E447F6F07213423FF498AA01EBC1022D
:10A74000C3F388144FEA131CC3F301130BEB82020B
:10A75000CE00D2F80C7F002C00F008830AF5805E52
:10A76000002238460132DEF80050944240F8045B83
:10A77000F8D107EB8404002B00F0EC810AF580523D
:10A7800023441568002225FA02F0083204F8010B70
:10A790009C42F8D173180BEB8303D3F80C7FDBF8E2
:10A7A000AC3C00937318CCF30A0C0BEB83036744A7
:10A7B000D3F8142FC3F80C7F6244C3F8142FFFF7AB
:10A7C00057BABC4BD3F88C3193F89C22042A04D09E
:10A7D00093F89C22D2B283F89D22042283F89C2213
:10A7E000FFF76DBAB34B0122D3F88C01D0F8B83221
:10A7F00080F89C22002B3FF41EAB5B6801799847E0
:10A80000FFF719BBD5E9070202442A62002C7FF446
:10A810007EAFDBF8CC0CDBF8D02C0590002A7FF45F
:10A820006EAC1846029B03F29C4274F027FB66E470
:10A83000A14BA24A0344934240F27D81A04BA14A1E
:10A840000344934240F282819F4BA04A03449342C7
:10A8500040F238829E4B9F4A03449342C0F06E827E
:10A860009D4B9E4A0344934240F296829C4B9D4AE4
:10A8700003449342C0F094829B4B9C4A034493420E
:10A88000FFF454AB9A4B9B4A03449342C0F0DF82DF
:10A89000994B9A4A034493422CBF4FF4C0534FF450
:10A8A000E053FFF745BB1CF0080F00F04881944AC5
:10A8B00096457FF6CDAC1CF4004F3FF4C9AC4FF485
:10A8C00000429A60C4E4009C434681E400238AF875
:10A8D0005732784BD3F88C01D0F8D432AE3350F8DD
:10A8E0002330002B3FF4CBAC90F89C22032A7FF45A
:10A8F000C6AC5B6A002B3FF4C2AC00999847BEE43B
:10A90000D8E90732934200F2288100F09A8198F842
:10A910009C32032B00F0CA818021404674F034FB46
:10A9200005230020C8F89432D8F8C8329A7903F584
:10A930001571C3F86802012AA3F85402C3E998000C
:10A9400008BFC3F87002186874F094FBFFF7DCBB13
:10A9500003F060025B0602D5402A7FF46CAD95F8E7
:10A960009C32013B022B3FF666AD5FFA8CFCBCF1DA
:10A97000030F3FF660ADD5F8B8329B68002B3FF46B
:10A980005DAD4FF0000907992846C5F8D492984765
:10A99000B5F8B022002A7FF451AD00287FF44EAD07
:10A9A0000422D5F8C832C5F81890C5F894224FF49F
:10A9B000807203F11401C3F828909A829A79012ACF
:10A9C000C3E908997FF48AADC3F8309086E51B0689
:10A9D000D5F8C85200F12F81002385F8553205F5CE
:10A9E000157301224FF000099A7083F8009095F8D2
:10A9F000941491423FF422AD286885F894245A7843
:10AA00001978069074F086FA069805F29C42A979A6
:10AA100074F034FA85F8949410E503F06003202B69
:10AA200000F07E81402B00F07B81002B7FF403AD92
:10AA3000BEF1010F5FFA8CF100F04881BEF1030F07
:10AA400000F08081BEF1000F7FF4F5AC95F89C32E8
:10AA5000022BDAB200F0A881032A7FF4ECAC01F0FB
:10AA60000F0314221CF0800F02FB035340F0B68149
:10AA7000B3F86431002B3FF4DEAC02FB015202F567
:10AA8000AA70002940F0318200230360D5F8C83253
:10AA90000222C5F89422C5E90622C8E51CF4004F3D
:10AAA0007FF40DAF1CF0200F3FF454AC20229A60CD
:10AAB00050E400BF00450024405327FFFF340C0042
:10AAC000401E1BFF3F420F0000DC0BFF7F4F1200B8
:10AAD000808CF9FE20D6130060B6E5FE5FE3160019
:10AAE00000D3CEFE40771B00C05BB3FEC0912100B7
:10AAF00000CA91FE20753800E05459FEE09C4100E8
:10AB00000A30544F0023EB75C14BD3F88C01D0F8B9
:10AB1000D432AE3350F82330002B3FF42CAC90F8F5
:10AB20009C22032A7FF427AC1B6A002B3FF423AC42
:10AB3000009998471FE44FF47053FFF7F9B91CF0E0
:10AB4000200F37D020229A60FFF782BB4FF460536A
:10AB5000FFF7EEB9CDF800A024E69A1AD8F8C8326B
:10AB6000C8E906225A6203F11401059A1A6200220A
:10AB70009A624FF480729A829A79012A01D10598DB
:10AB800018631868CDE9050374F074FA069B002079
:10AB90009A7903F51571C3F86802012AA3F85402E3
:10ABA000C3E9980008BFC3F87002059874F062FA10
:10ABB000FFF7AABA974A964503D91CF4004F7FF4D1
:10ABC0007EAE1A69DAF87432C2F312029B1ACAF81E
:10ABD0006832B8F1000F7FF4BDABDBF8102F002A0C
:10ABE00000F0D280DBF80C2F1A44CBF80C2FFFF7C3
:10ABF000B1BBD5F8D43228460799AE3355F8233087
:10AC00009B6898471AE4016C824B994203D91368F8
:10AC1000002BFFF69FAB00231361136943F400235D
:10AC20001361136943F018031361136943F0C043C0
:10AC30001361FFF78FBB4FF001036B7505F1140330
:10AC4000CFE6D8F8182093423FF661AED8F8983294
:10AC50009A42BFF45CAED8F8C83200204FF480723C
:10AC6000C8F8180003F114019A829A799862012AAF
:10AC7000C3E9080008BF18631868CDE9050374F03C
:10AC8000F9F9069B4FF0000C059803F51571C8F80B
:10AC900098C29A79C3F868C2012AA3F854C2C3E9DA
:10ACA00098CC7FF451AEC3F870C24DE6D8F8B832F4
:10ACB000DB68002B3FF430AE00224046C8F8D422B7
:10ACC000984729E64FF45053FFF732B995F89C3274
:10ACD000022BDAB24CD0032A7FF4ADAB069B002BDB
:10ACE0007FF4ACAB4806D5F8C89240F00A81042244
:10ACF000002309F11401D9F80000C5F894224FF49B
:10AD00008072AB61A9F8142099F80620C9F82830A0
:10AD1000012AC9E9083308BFC9F8303074F0AAF92C
:10AD2000D5F8B83200229B68C5F8D422002B3FF436
:10AD300085AB079928469847FFF780BB4FF44053EF
:10AD4000FFF7F6B895F89C32022B5FFA83FC0FD020
:10AD5000BCF1030F7FF46FAB480603D0069B13438F
:10AD600000F0CB80D5F8C832002030E43C4602E544
:10AD70004B0628463FF460AB74F006F92846802164
:10AD800074F002F9FFF75ABB029B012103F29C42C7
:10AD900074F074F8FFF7DEBA4FF43053FFF7C8B819
:10ADA0004FF42053FFF7C4B84A067FF444AB1CF0BD
:10ADB000800FD5F8C8324FF002024FF0000114BFE7
:10ADC00005F1140005F5AA700160C5F89422C5E9E3
:10ADD0000622C3E909211862FFF777BB9B8C002B81
:10ADE0003FF429AB01F07F01481C00EB800005EB2C
:10ADF000800000293FF448AE2422D5F8C83202FB77
:10AE000001318A7D003A18BF0122026040E600BF8E
:10AE1000004500240A30544F032B7FF40CABD5F8C7
:10AE2000C8320221C5E90622C5F8941204355A62D7
:10AE3000002203F114011D629A624FF480729A821B
:10AE40009A79012A7FF44AAB1D63FFF747BB4FF4A1
:10AE50000053FFF76DB8B9F1000F00F0AB806968DF
:10AE600001293FF47FAFD5F8B822C9B2284652680D
:10AE700090476C4B93F89810D5F8B8326960002B66
:10AE80003FF470AF1B682846984700283FF46AAF2C
:10AE9000284674F0B5F8D5F8B832297928465B68A9
:10AEA0009847022385F89C32FFF7C8BAB9F1000F22
:10AEB0003FF476AD0121D5F8B8326960002B55D04A
:10AEC0001B6828469847002850D0284674F098F808
:10AED000069B85F89C32FFF7B1BAC5F8A43241E76A
:10AEE000D5F8C832A861FFF773BB2422D5F8C83261
:10AEF00002FB013191F8562284E7284674F044F8A9
:10AF000030E701F00F0199F804308B42FFF4EFAE07
:10AF100001EBC1031CF0800F4FEA830341D103F51D
:10AF20001573002209EB030C242303FB019383F820
:10AF300055224FF000038CF800108CF8023099F87D
:10AF40009434012B3FF4D3AE0123D9F8000089F8E3
:10AF500094349CF804309CF801209CF8001073F0A5
:10AF6000B3FF4FF0000389F89434C0E60422D5F80B
:10AF7000C8320020C5F894224FF48072A86103F112
:10AF800014019A829A799862012AC3E9080008BFDD
:10AF90001863186874F06EF8032385F89C32FFF785
:10AFA0004DBA1433012209EB030C242303FB019354
:10AFB0005A75BEE7022349462846C5F8049085F82D
:10AFC0009C32D5F8B8325B689847E9E4DB6AFFF752
:10AFD00080BBD5F8B4329B69002B3FF42CAA0DF14D
:10AFE0002601287C98470346FFF731BBD5F8B432D9
:10AFF0001B69002BF3D1FFF71EBAD5F8B432DB681A
:10B00000002BECD1FFF717BAD5F8B4329B68002BB0
:10B01000E5D1FFF710BAD5F8B4325B68002BDED16A
:10B02000FFF709BAF84500242DE9F0474A4FD7F851
:10B030007856EE682C69A30701D5B00736D46107AE
:10B0400001D572072AD4230701D530071ED4E106A3
:10B0500001D5F20612D4E30701D5F0073BD414F46E
:10B06000025F2BD031066CD4600601D571066ED418
:10B07000A20601D5B30629D4BDE8F0876FF010030E
:10B080002B610023EA6987F89436E4E76FF0080340
:10B090002B610023EA6987F89436D8E76FF0040340
:10B0A0002B610023AA6987F89436CCE76FF002037E
:10B0B0002B610023AA6987F89436C0E7E305D3D54E
:10B0C0003706D1D56FF480732B61CDE76FF0200385
:10B0D0002B61BDE8F0876FF001032B611F4B9D4290
:10B0E000BDD1D7E9B8839845B9D098BFA3EB08097B
:10B0F000D7F8D8321A4A88BFC8F5805907EB8303BE
:10B100004244D3F8C432002BA9D0D3F814A2C3F818
:10B110000822C3F81092BAF1000FA0D10121C8444F
:10B120001048C3F814124B468121C7F8309074F0D0
:10B13000B1F8B8F5805F14BF43465346C7F8E03214
:10B140008DE76FF40253E2052B618DD5BAE76FF0FE
:10B1500040032B618CE700BF003500240014004041
:10B16000945600240435002402784368022A11D042
:10B170000D490269D1F86405023A184010B4400A3A
:10B18000D1F85C45D1F8581504FB02005DF8044B7A
:10B1900008447047044AD2F85015D2F84C2502EB07
:10B1A000410202EB53207047003500242DE9F04F97
:10B1B00083B002F00207854D019308B9002F6CD1CE
:10B1C000D5F85445002C53D14FF0FF3E804C4FF042
:10B1D000000CF146F046F246E36994F82A60984282
:10B1E00000F0A380002E3BD0012E05EB0C1B0AD1F2
:10B1F0009BF87363F30706D416F07E0F03D1F609AC
:10B2000000F09680E0460CF1010C1034BCF1080F00
:10B21000E2D1BEF1000F04DAB8F1000FC0F29A805B
:10B22000C646D5F8E4430EF1020605EB0E180134CC
:10B2300005EB061CC5F8E4430CF5527CCCF8044041
:10B24000C8E9D9040024CCF8084005EB061494F8AA
:10B250005243042C21D8DFE804F02B461C4648005A
:10B26000E6460CF1010C1034BCF1080FB4D1D0E764
:10B27000D5F85C65D5F8583506FB0434A042A3D355
:10B2800095F8003513B9012385F80035012385F8B9
:10B290004933002003B0BDE8F08F95F80035002B4E
:10B2A00054D00123022085F8493303B0BDE8F08F64
:10B2B00012F00104D5F860C374D105EB0610019BB0
:10B2C0004FEAE20C90F85383032B6CF3C71880F815
:10B2D000538365D94FF6FF70834228BF034605EBC1
:10B2E0000610A0F85033002F46D1500707D505EBC4
:10B2F000061090F8533343F0010380F85333D3061C
:10B300000AD505EB061696F85333C3F3450201320E
:10B3100062F3460386F85333D5F86033012003EB1C
:10B320004E230B6003B0BDE8F08FC6B9E64678E760
:10B33000666A1034B24588BFE1460CF1010C88BF43
:10B34000B246BCF1080F7FF447AF62E7012385F8EE
:10B350000035A6E7B9F1000F9BDBCE4661E7D5F8D3
:10B36000E4430CF10206E646013405EB061CC5F881
:10B37000E443CCF84C4368E7D5F8E803D5F8E43368
:10B3800001300133C5F8E80305EB0E10C5F8E433CE
:10B39000C0F8683305EB0613042083F85203A4E7D2
:10B3A00023469CE7D5F87035002B3FF472AF5C68FC
:10B3B0000CEB4E210023074AA04700283FF469AF59
:10B3C00005EB0616022386F8523362E700350024A7
:10B3D000483800247177040870B5114D82B00E46CC
:10B3E00095F84833022B16D1020AC4B2D5F84C05A1
:10B3F000002301A910440322FFF7D8FE012808D139
:10B4000095F84833019A022B0CBF22F8146042F8D9
:10B41000246002B070BDC0F3D41200F07F04E5E7F1
:10B42000003500242DE9F04F444E0D4683B01746F9
:10B4300096F848132B6803293ED0022961D14FEAC0
:10B4400013294FF4807A5FFA83F8421E012A23D829
:10B450004FF0010B9F421AD901288CBF0024012410
:10B46000D6F8C4241AB1D6F8E01499424CD0D6F8D4
:10B470004C050023092201A94844FFF797FE012843
:10B4800023D0022814D020B12B689F42E8D8032093
:10B490002F6003B0BDE8F08FB8F1000F13D096F81D
:10B4A000003513B9012386F80035012386F84933A6
:10B4B000022003B0BDE8F08F4FF0800AC3F3D41927
:10B4C00003F07F08C1E7D346C4E796F84813022982
:10B4D00013D00329ECD1019B53F8282022F07042AD
:10B4E000B2FA82F22B685209A2421FD0D8445B44C0
:10B4F000D0452B601DD20229EDD1019B33F81820D5
:10B50000EEE74FF4807AD9E7D6F85C15013A02EB02
:10B5100041224902B2FBF1F21344B3FBFBF20BFBF5
:10B5200012320AB15B449B1A2B60AEE79F42B0D83F
:10B53000ADE709F101094FF00008A6E70035002446
:10B540002DE9F04FDFF884918B4685B0174699F8C6
:10B5500048C30968BCF1020FD9F84C5540F082800D
:10B56000CEB24FF4807305EB1125A6EB0108904491
:10B570009844B94208F1FF38B8FBF3F84AD200F01A
:10B580000103A8446FF0404A0193BCF1030F07EB9D
:10B590000604A8EB0503284614BF4FF480728022EE
:10B5A000641A03A9944228BF1446944228BF002E6F
:10B5B00014BF012200220A32FFF7F8FD01282AD128
:10B5C00099F848C3DBF800E0BCF1020F0EF101036B
:10B5D00024D0B44255D9039806EB0A02011F00EBB0
:10B5E000820201EB840142F8043F8A4203F1010325
:10B5F000F9D1DBF80030A11B19448F42CBF80010C1
:10B6000002D1019B002B48D18F4205F101054FF07B
:10B610000006BAD8012005B0BDE8F08FB44246D983
:10B6200003986FF00042811E324401EB440100EBAD
:10B63000420222F8023F914203F10103F9D1A11B1A
:10B6400071448F42CBF80010DED1019B002BDBD080
:10B6500086466FF000434FF6FF72012023442EF818
:10B660001320D8E701F07F06C1F3D413BCF1030F18
:10B67000A6EB01081D4414BF4FF48073802390444F
:10B6800076E7AEEB060E0EEB04018F42CBF800100E
:10B69000BAD1019B002BB7D003986FF040434FF015
:10B6A000FF32234440F82320DBF80010ACE7AEEB78
:10B6B000060E0EEB04018F42CBF80010A4D1019BC3
:10B6C000002BA1D0DDF80CE0C3E700BF003500245B
:10B6D00030B50446C06983B010B9012003B030BD55
:10B6E0000D460023032201A9FFF760FD0128F5D1D3
:10B6F000B4F92020002A19DB019B012D4FEA4211E9
:10B7000003EB421203D0022D1BD1E5205854A3684D
:10B71000D3612378032B04D10023137753779377D6
:10B72000D377636A190C53839182D6E7064A92F85D
:10B73000001509B982F800050123022082F8493377
:10B74000CCE7E368E4E700BF003500242DE9F041D1
:10B75000044682B00D4694F83C30042B7ED8DFE8D6
:10B7600003F02B0369493A003D4E4FF6F777DFF8B7
:10B77000F48016E0BA425BD86AF0C2FC01284FF0B0
:10B78000000134D1206BFFF727FE01282FD1019A49
:10B79000D6F86015531E22638B4228BF0B46C6F8AD
:10B7A000603596F8482301A9236B032A18469AB2FC
:10B7B000E0D14345E0D93BE06900204601F0FE01BD
:10B7C000FFF786FF01283FD1636B002B18BF0220D3
:10B7D00084F83C00BFE794F82830042B02D1002302
:10B7E00084F82830A36B0BB120469847012002B0A3
:10B7F000BDE8F0811A4E0021E26AD6F8E03406F284
:10B80000BC40C6F8E0249B1AD6F85C2502FB03F383
:10B81000D6F8C42402EB4322C6F8C424D6F8C824C0
:10B8200002EB4322C6F8C824FFF752FF01280BD1D0
:10B830000420CDE7626B04F130010020FFF780FEA9
:10B84000012801D10320C3E70228D0D194F8283081
:10B85000042BCCD1002384F82830C8E70220F5E778
:10B8600000350024F7FFFF0F38B5044694F8343054
:10B87000052B60D8DFE803F031251D130D0394F884
:10B880002830082B3FD02D4B0122022083F80125C0
:10B8900038BD94F82830082B30D0012038BD002165
:10B8A0002046FFF715FF012845D1042084F8340015
:10B8B000DCE7D4E90B01FFF78FFD01283BD1032022
:10B8C000F4E74FF0FF31206BFFF786FD012832D1FE
:10B8D000E36A002BF3D00220E8E7184D04F13001B1
:10B8E0000120D5F854250232FFF79CFD012813D022
:10B8F0000238C0B201281ED80520D7E70023012056
:10B9000084F82830CAE700230122022084F8283076
:10B910000A4B83F80125BBE7E368D5F85C15226B79
:10B9200003EB4123C5F86025C4E90332E36A002B29
:10B93000BCD16262BAE7002038BD00BF00350024E8
:10B94000F8B5044694F83830032B4CD8DFE803F000
:10B9500021180B0200212046FFF7BAFE431EDBB27E
:10B96000012B41D9F8BD0120626B04F13001FFF7D2
:10B97000E7FD01284FF00303F0D184F83830E1E708
:10B9800000211E48FFF7A4FE01284FF00203F4D067
:10B99000E4E71B4BE66893F84823D3F85C15032AC9
:10B9A000D3F8C454D3F8E00414BF4FF4807280225B
:10B9B000206102FB01F1871A0244A5EB412506EB49
:10B9C0004126E660C3F8C454D3F8C854C3F8E02451
:10B9D000A5EB4121C3F8C814E36AC4E90C025BB9C2
:10B9E00060620123C9E7022094F82830062BB9D100
:10B9F000002384F82830F8BD2763F2E7BC3900241F
:10BA0000003500244368C3F308020A44B2F5007FFE
:10BA10002DE9F041054682B00C4605D223446B6007
:10BA2000012002B0BDE8F08190F91A10481C0AD03C
:10BA3000474A02EB011292F8731321F0010182F8D8
:10BA40007313FF22AA7695F91B20511C16D0404E85
:10BA5000023206EB021191F85313C1F3450101299B
:10BA600044D9013901F03F0106EB0212FF2692F89A
:10BA7000530361F3460082F85303EE762A78022AD4
:10BA8000CCD0334ED6F85C25B4EB422F4FEA422897
:10BA90002EDCD6F864751F407A42A24228DCE219F7
:10BAA0002869424513D32A7E12072DD5D6F8E02403
:10BAB000411C8A421ED300D100214344A4EB080854
:10BAC00068610846DB1B08EB070429616B600028EE
:10BAD000A6D096F84823032A35D080B24FF6F772E5
:10BAE00090429DD81A4614446C6099E70021BBE748
:10BAF000002096E796F800250ABB012386F800355A
:10BB000086F849336B68D8E701A96AF0F9FA012889
:10BB1000EED16B68A4EB0804286998442978686121
:10BB20003C44A8EB0703019802291A466B60286180
:10BB3000CDD1D6F86C15B3EB412FD4D370E70122E9
:10BB400086F84923B9E7034A90423FF669AFC9E74F
:10BB500000350024F7FFFF0F2DE9F0474FF00108F3
:10BB600082B0044694F83830032B00F2A680DFE858
:10BB700003F055170C020020236C84F8280003B151
:10BB80009847022002B0BDE8F0870022236C84F8B9
:10BB900028200BB120469847012002B0BDE8F0876D
:10BBA00023786768022B03D0454BD3F864351F40D8
:10BBB000C7F34F272046FFF7D7FA414E3F1A0546F5
:10BBC000BFB207EB050C022201A9002328461FFA89
:10BBD0008CF9FFF7EBFA01284FF400724FF00001E7
:10BBE000D0D101987DF072F9E3694FF400712046DD
:10BBF0000BB16368EBB1D6F85C355A1E914547D25C
:10BC00000135FFF7FFFE0028DBD196F8003513B9A8
:10BC1000012386F8003586F84983D2E72046FFF7EE
:10BC200023FE012802D0022847D1032084F83800DF
:10BC300098E7019B4FF020324FF0100E4FF02E0C82
:10BC400042F62E6AC3F80120C3F80520A3F80920A4
:10BC500083F800C0D4F824C0A3F820A083F80BE038
:10BC6000C3F82220C3F8262083F82A20E26BA3F829
:10BC70001AC02CFA0EFC5A8722FA0EF2A3F814C04E
:10BC80009A8683F82BE0D6F85C355A1E9145B7D3D7
:10BC9000C3EBC3532046590201F50071FFF7B2FE12
:10BCA00028B996F8003523B1012386F849330220DC
:10BCB000BCE7012386F80035F6E7002062E700BF05
:10BCC00000350024B1F904300F2B2DE9F0410D4669
:10BCD00082B00446164634D02046FFF745FA94F960
:10BCE0001B80B8F1FF3F3DD05C4F07EB0813D3F842
:10BCF0006433984212D097F80035002B70D001239E
:10BD000087F849332378022B60D02269002A75D145
:10BD100000230120336002B0BDE8F081D7F8601342
:10BD200001EB4821002967D0AB88204601331BB2C4
:10BD300001EB4311AB803160FFF716FA2860012058
:10BD4000E9E74FF40071FFF75DFE002844D04FF69D
:10BD5000FF732046AB80FFF707FA94F91B80B8F118
:10BD6000FF3FC1D12378022B3ED02269002ACFD0D9
:10BD70003A4F97F84833032B67D093B24FF6F771D9
:10BD80008B4294BF00230123002BBFD130B997F819
:10BD90000035002B4CD0012387F8493300231122B2
:10BDA00001A9FFF703FA012826D10199D7F86033DA
:10BDB000CB1A48BF03F2FF13B3F5805F4FEA63224B
:10BDC0002CD24FFA82F884F81B80ABE7D7F86C25A9
:10BDD0006368B3EB422F9BD2002002B0BDE8F08134
:10BDE000012387F800358AE71C4F6368D7F86C2574
:10BDF000B3EB422FCAD38BE7237884E797F8483315
:10BE0000032B19D093B24FF6F772934294BF0023DD
:10BE10000123002B7FF47CAF0020DEE797F800358C
:10BE200013B9012387F80035012387F84933CAE79E
:10BE3000012387F80035AEE7094B9A4294BF0023EF
:10BE40000123002B7FF464AFE6E7054B9A4294BFD1
:10BE500000230123002B7FF459AF97E7003500241E
:10BE6000F7FFFF0F2DE9F047044688B094F8303013
:10BE7000042B11D8DFE803F0501361035A00237E2E
:10BE80009A0640F1F9800023112204A9E069FFF726
:10BE90008DF9012800F0F08008B0BDE8F087C64DAC
:10BEA00003AE04F11C0705F20459324639464846F0
:10BEB000FFF708FF012800F0FA800228ECD195F97D
:10BEC0001E355F1C0AD005EB0313FF2193F8732383
:10BED00085F81E1522F0010283F8732395F91F35AA
:10BEE0005E1C17D0023305EB031292F85323C2F302
:10BEF0004502012A40F25E81013A02F03F0205EB61
:10BF0000031393F8531362F34601FF2283F853138C
:10BF100085F81F25042306E0A8486BF0F5FB4FF6D3
:10BF2000FF720123228484F830309FE70020E36A07
:10BF3000207008B0BDE8F04718479F4D95F82C35A4
:10BF4000002BA9D104F11C0705F2045803AE3246B8
:10BF500039464046FFF7B6FE012840F01881039BA2
:10BF6000002B00F0F1801A780AB1E52AEFD1D5F85C
:10BF700060239A1A48BF02F2FF12B2F5805F4FEABF
:10BF8000622180F04C8109018D4A0A44917B042989
:10BF90000CD0D5F8E4130131C5F8E4135160042145
:10BFA0009173D5F8E8230132C5F8E82395F91E25E9
:10BFB000501C0AD005EB021292F8731321F0010114
:10BFC00082F87313FF2285F81E2595F91F25511C51
:10BFD00017D0023205EB021191F85313C1F345015A
:10BFE000012940F26481013901F03F0105EB0212A1
:10BFF000FF2085F81F0592F8530361F3460082F88D
:10C0000053032022002118467CF060FFD4F8311041
:10C010000346D4F8352005A819605A6094F83B20EF
:10C02000B4F839109A721981627E0193DA7202F0C3
:10C030000FF8019B002800F0DB809DF816009DF8AA
:10C0400017209DF8191042EA4012BDF8140049016A
:10C05000A0F2BC7042EA40229DF81A0041EA500169
:10C060009DF8180092B241EAC02188B2D9811A82A3
:10C070001A83D882032356E720466BF045FB2369D9
:10C08000002B00F08980237E03F0F70213F00403F5
:10C09000227640F09780122A00F0AD800022E36AF9
:10C0A000204684F8282008B0BDE8F0471847DDF89E
:10C0B0000C80B8F1000F00F0BE8098F80030002B23
:10C0C00000F0B98098F80BA01AF0080F7FF4EDAEDD
:10C0D0000B2204F1310140467BF04CFD00287FF437
:10C0E000E4AE637E8AEA0303DF0640F1E48095F95B
:10C0F0001E355E1C0AD005EB0313FF2193F8732352
:10C1000085F81E1560F3000283F8732395F91F2547
:10C11000511C3FF4FFAE023205EB021393F8533388
:10C12000C3F34503012B40F20981013B03F03F03B8
:10C1300005EB021292F8531363F34601FF2382F8D2
:10C14000531385F81F35E5E695F804350922022BCF
:10C150003FF4E0AE95F82C35002B7FF4DBAE85F88C
:10C160003C354046C5F84035C5F8443585F8383586
:10C17000D5F8183585F82C25C5F83035D5F8603553
:10C18000C5F83435FFF7E8FC01283FF4E0AE02289B
:10C190007FF482AE0423C6E6237E1B077FF57EAFC5
:10C1A000054B93F8E424002A7FF476AE072283F847
:10C1B000E42473E70022A2E600350024043A0024B8
:10C1C000643800240023A5682046E66A294684F8DE
:10C1D0002830FFF717FC002863D194F82830002B93
:10C1E0007FF45AAE0223C4E90B6584F8283053E685
:10C1F00044F281723BE7E06A0421626AA063204650
:10C2000084F83C3084F8281063636362C4E90B222D
:10C21000C4E9023308B0BDE8F0476BF075BA95F891
:10C22000002512B9012285F8002501226FF00F01C7
:10C2300085F84923A8E695F91E35591C0AD005EB67
:10C240000313FF2193F8732385F81E1522F00102D2
:10C2500083F8732395F91F355A1C16D0023305EB6A
:10C26000031292F85323C2F34502012A21D9013A5D
:10C2700002F03F0205EB031393F8531362F34601F8
:10C28000FF2283F8531385F81F25237EDB067FF5F5
:10C2900041AE2C486BF038FA4FF6FF72022322842D
:10C2A00041E6002E3FF4F8AD2046334641E600213A
:10C2B0009CE60022DEE7B8F81420B8F81A3043EA0A
:10C2C0000243D5F85C2563625202D8F81C30B3FBF8
:10C2D000F2F102FB1131A36009B113445B1AE36070
:10C2E00084F819A095F91E355A1C0AD005EB0313E2
:10C2F000FF2193F8732385F81E1522F0010283F8BD
:10C30000732395F91F25531C3FF4B4AE023205EB9D
:10C31000021393F85333C3F34503012B10D9013BA8
:10C3200003F03F0305EB021292F8531363F3460147
:10C33000FF2382F8531385F81F359BE60023F7E6A9
:10C340000023EFE7043A002410B50378044690F880
:10C3500018C0023B012B02D91CF0060F6ED11CF055
:10C36000200F44D194F91A20511C0AD03A4BFF21D6
:10C3700003EB021393F8732322F0010283F8732373
:10C38000A17694F91B305A1C16D03349023301EBC5
:10C39000031292F85323C2F34502012A4BD9013A02
:10C3A00002F03F0201EB031393F8531362F34601CB
:10C3B000FF2283F85313E2761CF0080F0ED02649B3
:10C3C00091F8E434072B06D091F80035002B3DD0CE
:10C3D000012381F84933002381F8E4340023E26A21
:10C3E000237084F8283042B3BDE8104010471B4A40
:10C3F0000023E069D1691032884206D00133082B4E
:10C40000B0D0D16910328842F8D11349023301EB20
:10C41000031292F85323C2F34502012A1AD9013AB2
:10C4200002F03F0201EB031393F8531362F346014A
:10C4300083F8531396E70022B4E710BD0121FFF7FC
:10C4400047F90128F9D194F818C088E7012381F849
:10C450000035BDE70022E5E7003500244838002418
:10C4600038B51A4C94F82C352BB970B190F82820B7
:10C470001AB1184638BD002038BD0146442204F2E6
:10C4800004507BF0FBFB012038BD04F2045501464B
:10C49000442228467CF01AFD94F8483303224FF6D4
:10C4A000FF71022B2846A4F81E1518BF1346D4F8B6
:10C4B000681584F81C25102284F80435C4F8281562
:10C4C00084F81D256BF020F9DDE700BF003500245E
:10C4D000314A4FF0FF31F8B5A2F5527C00230C46EB
:10C4E00003E001331032082B14D092F82A000428FC
:10C4F000F7D10CEB031090F87303C607F1D4651C59
:10C50000106A01D08142ECD91C4601330146103239
:10C51000082BEAD1002C01DA0120F8BD1F4DA61C22
:10C5200005EB0613D5F87025B3F85013E9B92701C8
:10C530002F44D5F86013D5F87035D7F8640301EBB4
:10C540004421DBB1DC680023154AA047B0B10228C2
:10C5500009D1D5F8E83305EB06160122013B86F830
:10C560005223C5F8E8330020F8BD05EB041327017A
:10C57000D3F8640312B193689847D9E7D5F8E83344
:10C5800005EB061603210122013B86F8521385F8BC
:10C59000EC23C5F8E833E6E74838002400350024EA
:10C5A000D57704082DE9F04390F8283083B004468D
:10C5B000013B082B0BD8DFE803F0383C1F2305298B
:10C5C0000A2E33000121FFF7C1F8012802D003B081
:10C5D000BDE8F08300222378216C84F82820002B0A
:10C5E000F5D00322E162D4E9010384F828208342D4
:10C5F00038BF03462046A36003B0BDE8F043A3E67E
:10C60000002103B0BDE8F043FFF7A0B803B0BDE8D8
:10C61000F043FFF795B903B0BDE8F043FFF724B945
:10C6200003B0BDE8F043FFF797BA03B0BDE8F043AD
:10C6300018E4DFF834914368D9F86465026B194651
:10C640001E40D9F85C0594F800C0B5184702B5EB58
:10C65000402F41D34FF6F778BCF1020F14D0256973
:10C660002846002D5AD16168A3680020E26A8B42F7
:10C6700084F8280038BF0B46A360002AA7D02046C4
:10C6800003B0BDE8F04310476168D9F86C05B1EB21
:10C69000402F5CD22069217E090732D5D9F8E014F9
:10C6A000451CA9422AD299F80015002943D101233B
:10C6B00089F8003589F84933226B636894F800C023
:10C6C000D21B3B4432449B1B0026974219466360B1
:10C6D0002263C4E90450BFD9BCF1020F37D02569E9
:10C6E000002DC1D099F84833032B36D0ADB24FF6A8
:10C6F000F7739D42B8D811446160B5E7E0D10025D9
:10C70000DEE701A969F0FCFC01287FF460AF206935
:10C71000019D94F800C06368226BD1E799F8481333
:10C7200003290ED0A9B2414594BF0021012100295F
:10C73000B1D06168D4E7012189F8491394F800C0A9
:10C74000BEE708498D4294BF00210121EFE7D9F8E7
:10C750006C35B1EB432FCED386E7024B9D4283D895
:10C76000C9E700BFF7FFFF0F00350024704700BF87
:10C77000DFED0A7AB7EE007A0023C0ED020A20EE60
:10C78000270A0360C7EE007A30EEA77AC0ED017A7F
:10C79000C0EE877AC0ED037A704700BFDB0FC94057
:10C7A000024A136823EA000313607047A06600245E
:10C7B000007970470079C0F3401070470079400954
:10C7C000704700BF704700BF704700BF03685A1C26
:10C7D00002601970704700BF03685A1C026019702C
:10C7E000704700BF024B586803681B68184700BFBA
:10C7F000A06600242DE9F0413A4E33787E2B03D019
:10C8000000273846BDE8F08108214FF4FC4341F28F
:10C8100021041AB25B00002A84EA42009BB2B8BF2E
:10C8200083B20139F5D1B6F80140002C37D02E4A39
:10C830002E4DAA42E4D2052CA2F106028CBF00279D
:10C8400001271444AC4228BF47F00107002F46D10E
:10C8500041F2210EA24214D0501E04F1FF3810F80C
:10C86000011F082283EA012319B25B0000298EEA26
:10C87000410C9BB2B8BF1FFA8CF3013AF4D140458A
:10C88000EDD1218861B1A21DAA42BAD2052904EBDB
:10C8900001002246B5D9A842B3D20446DAE7144CC7
:10C8A000671E41F22105BC4617F8012F83EA0223D7
:10C8B000082219B25B00002985EA41009BB2B8BF8B
:10C8C00083B2013AF5D16445EDD16788094AFF1A70
:10C8D000231DB7FA87F79B1B7F09138191E70F464A
:10C8E0008FE700BF000002080700020800000408EC
:10C8F00001000208A066002490F83C20034602F0E4
:10C90000FF0012B1002283F83C2070474FF480539F
:10C91000838170474FF40063838170474FF4006355
:10C92000838170474FF40063838170474FF4006345
:10C9300083817047074B10B403F11001002453F8B2
:10C94000042B824208BF43F8044C8B42F7D15DF8B8
:10C95000044B7047AC66002470B5374C608DA38BD8
:10C96000B4F934501B1A208DB4F922C000FB03F334
:10C97000B4F93200266C05EBE335C00290FBF5F00C
:10C9800000EBE330B4F92E30A0F57A6EA0630EFB15
:10C990000EF50EFB0CFC2D134FEAEC2C05FB03F3FC
:10C9A0000CEBE32CB4F92C3005FB03F3B4F9245061
:10C9B0001B140EFB05F503EB6533B4F9205002336D
:10C9C0000CEB850CB4F93C509B10E48C0CFA05FC84
:10C9D00003F500430CF1020C04FB03F34CF250345A
:10C9E000A6EBAC0C2C41DB0B04FB0CF4002C1EDB87
:10C9F0006400B4FBF3F389B11C1240F6DE3504FB8E
:10CA000004F405FB04F40D4D241403FB05F504EBBD
:10CA1000254404F6CF6403EB24130B602AB100EB2A
:10CA200080004000083000111060012070BDB4FB90
:10CA3000F3F35B00DFE700BFA066002443E3FFFFE2
:10CA400001207047012070472DE9F04F734D85B0EC
:10CA50000F46686CB5F848300092C3EB2014B5F966
:10CA60004C205B00B5F954E004FB04F4B5F84E80AB
:10CA7000C3EBE003CDF80CE02413B5F95660B5F92B
:10CA8000581002FB04F4B5F94A20029602FB03F3A6
:10CA9000A413B5F9502004EBE3246B6EA4F5FA302F
:10CAA0000193B5F9523080FB00EA4FEAE37B82FB49
:10CAB000002C03FB0AF94FEA0C3C2C660EFB0B9989
:10CAC000A3FB0E3B4CEA125C1203CB441B0A43EA65
:10CAD0000B639B184CEB2B2BA3FB08320BF5004B85
:10CAE00008FB0B2B4FEAEB734FEA6B0953EA6B0B16
:10CAF00000F09280029E01FB0AFA019A86FB000870
:10CB0000039EC2F5801C4A464FEA48484FEAE17945
:10CB100048EAD0380EFB09A94004A1FB0E1E4118BB
:10CB2000F1444FF000000CF0004E49EB08094EEACA
:10CB30005C0E41184FEACC7C09EBC609BCEB010C3A
:10CB40006EEB090E1CEB0C084EEB0E0118EB0C08FB
:10CB50004EEB01014FEA88104FEA811918EB0000F3
:10CB600049EA986941EB0901890041EA9071800026
:10CB700010EB0C004EEB0101890041EA907180003E
:10CB800010EB0C004EEB010174F054FDB5F95E3072
:10CB90004FEA613884464FEA503EB5F95A204FEAD1
:10CBA000E37A03FB08F94EEAC14EB5F95C000EFBCF
:10CBB0000A99A3FB0E35A94403FB08F50EFB0955A2
:10CBC000A3FB0E3E75445B0E4FEAE07E43EAC513BD
:10CBD00013EB0C0341EB656500FB01F10EFB0C113F
:10CBE000A0FB0C0C6144C00C40EA41301B1845EB23
:10CBF000E1451B0A43EA056303EB02130FB11B0A6D
:10CC00003B60009B23B104EB8404803424121C603D
:10CC1000012005B0BDE8F08F0023EFE7A0660024F7
:10CC200031B10A4BD3ED217AFDEEE77AC1ED007AFE
:10CC300052B1064B9FED067AD3ED227A67EE877AE2
:10CC4000FDEEE77AC2ED007A01207047A06600246D
:10CC50000000C8422DE9F04F5F4D934685B0B5F80E
:10CC60009A30D5F88C001B02B5F898E0B5F89640DC
:10CC7000C21AB5F89430019167EB0707AEFB020CBE
:10CC80001B04B5F892100EFB07CCC009B5F89C60E8
:10CC9000C90340EA4C604FEAEC1CC018A4FB023EFA
:10CCA00004FB07EE4FEA13234CF1000C43EA0E633A
:10CCB0004FEA2E2E5B18A6FB021406FB07444FEA30
:10CCC000D1514EF1000E41EA4421E41511F5FA6804
:10CCD00044F10006B8F5FA6F029676F1000630DAF4
:10CCE00001FB04F60394A1FB014A0AEB460AA600E5
:10CCF0004FEA8A09361949EA9479384C4AEB09090E
:10CD00004FEA560AB6084AEAC97A46EA8976B0EB8B
:10CD10000A0A6CEB690C9E1B50466EEBA90E33465B
:10CD2000A045029E4FF0FF34A64126DB02FB07F729
:10CD3000A2FB022101EB4701D20F42EA4102B8EB0C
:10CD40000208019C84B1D5F8A010A1FB033201FBBD
:10CD50000E225B0D43EAC22352151B1A62EB0C0232
:10CD6000DB0B43EA42432360BBF1000F01D0CBF859
:10CD70000080012005B0BDE8F08F40F6AC56039C62
:10CD8000891944F1000401FB04F4A1FB016101EBEA
:10CD90004401F4004FEAC109341B49EA567961EBBA
:10CDA000090924184CEB090C2046B41941EB010980
:10CDB000A41941EB09094FEA890949EA9479A400C9
:10CDC000A41B69EB0109610841EAC971591A6EEBAC
:10CDD000690E0B46AAE700BFA066002424FAFFFFF5
:10CDE00001207047104B10B4104C1B68D4F8A400FD
:10CDF0001B1AFA2B0BD811B1D4F8B0300B6012B15A
:10CE0000D4F8B430136001205DF8044B7047D4F8B7
:10CE1000A830002223F00403104684F8AC20C4F8A4
:10CE2000A8305DF8044B7047C43B0024A066002482
:10CE30002DE9F8430D46D0E9003113448B4220D848
:10CE40000446AE18076BCAB14FF0000900F10C0898
:10CE500001E0AE4212D0E36A5A1C2344E262202A67
:10CE600015F8011B1973F4D14146204617B9F5F79F
:10CE700059FD0746AE42C4E90B97ECD13846BDE8F0
:10CE8000F8834FF0FF37F9E738B51446002944D04E
:10CE9000344B0D469FED344A93ED2E7AD3ED316A33
:10CEA000B8EEC76AB3F9D420B8EEE60AD3ED2F7A0C
:10CEB00004EE902AB3F9D020C6EE046A93ED327ADC
:10CEC00005EE902AB3F9D22005EE102AB3F9CE2050
:10CED000B3F9CC30F8EEE44A06EE102AF8EEE55A43
:10CEE000F8EEE77AB8EEC55AB8EEC77AC7EE843ADC
:10CEF00007EE903AB8EEC66AE6EEA45AF8EEE77A84
:10CF0000A6EE856AA6EEA57AE6EE867AA6EE870AF2
:10CF1000A3EEA70A76F054FF28600CB3114BF6EE8F
:10CF2000005A9FED115AD3ED2F6AB3F9C220F8EEE3
:10CF3000E66AB3F9C03007EE102A9FED0C6A07EEDF
:10CF4000903A86EE850AB8EEC77AF8EEE77A20EED8
:10CF5000070AA7EEA50A20EE060A76F031FF206048
:10CF6000012038BDA06600240000F04A0000C8423D
:10CF70000369416853EA0102F0B43B4E5DD0C56AD3
:10CF8000013390ED067A6A1C876830EE077A0361F8
:10CF9000012AC26280ED067A42D090ED075A07EE70
:10CFA000902AD0ED096A70EE455A3468B8EEE76A07
:10CFB000611AC5EE867AB94277EE857A30EE670A55
:10CFC000C0ED087AC0ED077AF0EE667AE5EE807A79
:10CFD000C0ED0A7AC0ED097A01D8F0BC7047012A89
:10CFE00028DD06EE905AF8EEE66A87EEA66AB5EE00
:10CFF000C06AF1EE10FA1DDBF1EEC67AF4EE677A44
:10D00000F1EE10FA16D6D0ED056AF4EEE76AF1EE0D
:10D0100010FA15D5037BFBB10323F0BC03707047F6
:10D02000326880ED080A521A002180ED070ABA42E0
:10D030004162D2D9DFED0D7AE5E7316841609EE7C4
:10D0400007EE903A0223F8EE677A0370F0BCC7EE61
:10D05000276AC0ED066A7047316800220361C36227
:10D0600041608261B9E700BFC43B002400000000BA
:10D0700010B5DFED4F4A844600F1480E0346DA6AE8
:10D08000B1EC017AD3ED067A013277EE877A012A84
:10D09000DA62C3ED067A71D093ED075A07EE902A53
:10D0A00093ED096A77EE455AF8EEE77AC5EEA76A7E
:10D0B00076EE857AF0EE466A37EE677AC3ED087A47
:10D0C000E5EE876AC3ED0A6AC3ED077A1833C3ED4C
:10D0D000036A7345D3D1374C416822680369521AF9
:10D0E000816801338A42036147D990ED056A0022C5
:10D0F000DFED2F5ADCF82C10F0EE657ADCED0A6AD1
:10D10000012901F1FF3E11DD07EE90EAF8EEE77A22
:10D1100086EEA77AB5EEC07AF1EE10FA45DBF1EEB5
:10D12000C77AF4EE677AF1EE10FA3ED6B4EEE76A0B
:10D1300001320CF1180CF1EE10FA26D4022AD9DDD6
:10D14000B4EEE76AF1EE10FA1FD407EE903AD0ED94
:10D15000066A90ED0C7A0223F8EE677AD0ED125A47
:10D16000037086EEA76AC7EE276A85EEA77A80ED80
:10D17000066AC0ED0C6A80ED127A10BDF0EE477AB7
:10D1800083ED087AF0EE646A9EE7037B13B1032314
:10D19000037010BD002221680361C3624160826197
:10D1A000026343648264C36510BDDFED017ABDE7AD
:10D1B00000000000C43B0024B0EEC06AF0EEE05A6C
:10D1C000F0EE407AF4EEC65AF1EE10FA0EDCB5EE4F
:10D1D000400AF1EE10FA4AD0F4EEC65AF0EE466A72
:10D1E000F1EE10FA4FD5B0EE655A03E0F0EE656A45
:10D1F000B0EE465A85EE267A9FED242A9FED243A1A
:10D200009FED244ADFED244ADFED242ADFED243AA6
:10D21000B7EE005ADFED236AF4EEC65AF1EE10FACB
:10D22000A7EE023AE7EE223AA7EE034AA7EE235A08
:10D23000E7EE044AE7EE246AB1EE667A87EE050A65
:10D2400010D4F5EEC00AF1EE10FA03D59FED167A70
:10D2500037EE400AF5EEC07AF1EE10FA48BFB1EEB3
:10D26000400A70479FED117A37EE400AE9E7F5EE84
:10D27000C00ADFED0F7A9FED0F0AF1EE10FA58BFEA
:10D28000B0EE670A7047B0EE465AB3E739094E3D33
:10D29000E3B59EBE88FA16BE45FE7FBF99FB243FCC
:10D2A00069A2163EA7DFA8B4DB0F4940DB0FC93FD8
:10D2B000A7DFA834DA0F4940D1ED007AF7EE002A53
:10D2C000D0ED043A90ED054AE7EEA73AD0ED064AD4
:10D2D00090ED075AD0ED085A90ED096AD0ED0A6A30
:10D2E00090ED0B7AC0ED043A91ED003AD1ED013AA0
:10D2F000D0ED0C7AA3EE234A80ED054AD1ED003A39
:10D3000091ED024AE3EE844AC0ED064AD1ED004AAF
:10D3100035EE245A80ED075AD1ED014A91ED005ABD
:10D32000E4EE855AC0ED085AD1ED015AA5EEA56A82
:10D3300080ED096AD1ED015A91ED026AE5EE866A47
:10D34000C0ED0A6AD1ED016A37EE267A80ED0B7ADC
:10D35000D1ED026A91ED007AE6EE877AC0ED0C7AA3
:10D3600091ED027AD1ED017A90ED0D3AD0ED0E3AC1
:10D37000A7EE273A90ED0F4AD0ED104A90ED115AE2
:10D38000D0ED127AD0ED135A90ED006A80ED0D3A8F
:10D3900075EEA25A91ED023AD0ED016AE3EE033A3E
:10D3A00090ED027AC0ED0E3AD1ED023A34EE234A06
:10D3B00080ED0F4A91ED004A74EE844AC0ED104AA8
:10D3C000D1ED014A35EE245A80ED115A91ED025A01
:10D3D000C0ED135A77EE857AC0ED127AD1ED017A5D
:10D3E000D1ED005A67EEA77A91ED025AE5EEA57AE3
:10D3F000E5EE057AA5EEA76A80ED006A91ED016A77
:10D40000E6EE276AC0ED016AD1ED026AA6EEA77AC0
:10D4100080ED027A90ED037A77EE277AC0ED037AF9
:10D42000704700BF2DE9F04F4FF00009864600F12C
:10D4300010050646034689B000F130080746484605
:10D440002C468B469C46B246CDF80CE000283CD1D9
:10D450000CF1040CA445FBD1032800F1010151D0CB
:10D460009C46AA46029398B1DCED047AAAEB090324
:10D47000B64601927246F3EC016A0EF1100E92ED7F
:10D48000007A5345E6EEC77ACCED047AF2D1019AE0
:10D49000DCED046A0CF1100C15ED047A0AF1100AA7
:10D4A000C445C6EE877ACCED007ADCD1029B043607
:10D4B000084608F10408143314351034103709F104
:10D4C00004099C46B2460028C2D0DCED007AD6465C
:10D4D000394601927246F1EC016A0EF1100E92ED9E
:10D4E000007A9942E6EEC77ACCED007AF2D10CF1DF
:10D4F000040C019A0AF1040AA445E6D1032800F1BC
:10D500000101ADD1DDF80CE00023594604AD7646AB
:10D51000774600200493059306930793F2EC017A73
:10D52000E5EC017AB0B104AC3B46B4EC017AF3EC23
:10D53000016AE6EEC77AB34245ED017AF5D10130D2
:10D5400004280BD0F2EC017A10371436E5EC017A9E
:10D550000028E8D1103714360120DFE708AD10317C
:10D560000EF1400E042875ED017AA1F10402744613
:10D5700041ED017A1ED07346F3EC016AB1EC017AF9
:10D58000A342E6EEC77AC2ED007AF5D15EED016AFC
:10D59000013887EEA67A82ED007A17D0AEF1140E2C
:10D5A000103C114675ED017A0428A1F1040241ED09
:10D5B000017AE0D15EED016A103CAEF1140E032059
:10D5C00087EEA67A01ED017A1146EBE709B0BDE8D6
:10D5D000F08F00BF60EEA00AE0EE000AF5EEC00A90
:10D5E000F1EE10FA07DBB1EEE00AB4EE400AF1EE1C
:10D5F00010FA00D670479FED010AFBE7000000001B
:10D6000060EEA00AE0EE000AE1EE010AF5EEC00AC3
:10D61000F1EE10FA07DBB1EEE00AB4EE400AF1EEEB
:10D6200010FA00D670479FED010AFBE700000000EA
:10D63000DFED297AB4EEE70AF1EE10FA28DD9FED6E
:10D64000277A30EE470AB4EEE70AF1EE10FAF8DC7A
:10D65000DFED237AB4EEE70AF1EE10FA2FDD30EEBB
:10D66000670A37EEC00A60EE007ADFED1E5A9FEDC2
:10D670001E6ADFED1E6AA7EEA56A9FED1D7A60EEB9
:10D68000275AE7EE866AA7EEA67AA5EE870A7047C4
:10D69000DFED187AB4EEE70AF1EE10FAD8D59FED77
:10D6A0000F7A30EE070AB4EEE70AF1EE10FAF8D47A
:10D6B000DFED0B7AB4EEE70AF1EE10FACFDC9FED66
:10D6C0000E7AB4EEC70AF1EE10FACCD530EE270A86
:10D6D00037EE400AC7E700BFDB0F4940DB0FC94008
:10D6E000DB0FC93F9A7C2E36FAAF4FB93587083C1D
:10D6F000A4AA2ABEDB0F49C0DB0FC9BF10B5404C3E
:10D70000B4FBF2F4A14219D3DFED3E7AF7EE005AF2
:10D71000B0EE677AB0EE676AF0EE676A0023C0ED9C
:10D72000005AC0ED017A80ED027A80ED036AC0ED07
:10D73000046A836143610362C36110BD07EE902AEE
:10D74000DFED315AB7EE006ADFED306AB8EE677A86
:10D7500007EE901AB0EE405AF8EE677A27EE257A77
:10D7600067EEA67AC6EE076AC7EEA64AFDEEE47A31
:10D7700017EE902A2032402A3FD8B0EE640AFFF715
:10D7800057FFB0EE404ADFED227A34EEA70AFDEEF5
:10D79000C07A17EE902A2032402A29D8FFF748FF96
:10D7A000F8EE006A60EE266A012B1CD0B7EE006A24
:10D7B000F6EE004A36EE406A66EE244A35EE055A29
:10D7C000F7EE007A84EE057A77EE275A37EEC75ADD
:10D7D00084EEA57AC6EE257A86EEA56AC5EE256AA0
:10D7E000F0EE475A9AE7F7EE004AB0EE666AE5E7D0
:10D7F000DFED086A9FED030AD6E79FED024AC2E714
:10D8000020A1070000000000BD378635DB0FC940AE
:10D81000DB0FC93F00000080DFED077A30EE270AFA
:10D82000FDEEC07A17EE903A2033402B00D8FFE689
:10D830009FED020A704700BFDB0FC93F00000000E8
:10D840002DE9F84F9DF828408946DDF82CB00546B3
:10D85000002C17461BF8011B0CBF4FF020084FF09F
:10D8600030081C1E08463ADB00295CD0002C53D03F
:10D870004FF0000A5B4600E064B313F8016B013C13
:10D88000002EF9D1BAF1000F2FD1264644B14D45F3
:10D890004146284600D2B847013CF8D10B9B187886
:10D8A0000146A0B14FF0FF344FF0000A00E09B4664
:10D8B0004D45284600D2B8475B4613F8011B0029A6
:10D8C000F5D10B9BF61A5E44BAF1000F10D1304629
:10D8D000BDE8F88FBAF1000F1BD15646E0E763426E
:10D8E00029B31C464FF0010AC4E70028E0D10646E0
:10D8F000002C04F1FF3AEADD54464D4541462846E6
:10D9000000D2B847013CF8D2013656443046BDE853
:10D91000F88F30B12646CBE726464FF0FF34B246AB
:10D92000C6E70646D3E72646002CB0D1CFE76FEA1C
:10D93000040A0E46E0E700BF0FB430B583B00B4CCD
:10D9400006AB53F8042BD4E9360101936CF006F9C9
:10D950000546606803685B6998470028F9D0284647
:10D9600003B0BDE8304004B0704700BFA06600249B
:10D970000EB410B583B00446084905AB01A853F8AE
:10D98000042BCDE900346CF0E9F80022019B1A70F9
:10D9900003B0BDE8104003B0704700BFD9C704080A
:10D9A0000CB4F0B53C4CADF5277DD4F8E030002B3D
:10D9B0006DD094F8E83099420BD90123D4F8EC20CB
:10D9C0008340134205D10DF5277DBDE8F04002B03C
:10D9D0007047324B4FF47A71314A1B68A2FB030245
:10D9E00006A8920901FB12332E49FFF7C1FF06ABCF
:10D9F000AC9A064603442C4901A80193ADAB0093B1
:10DA00006CF0ACF8019B0A2100225D1C0195197095
:10DA1000019BD4F8E050591C01911A70ADB12B68EC
:10DA20005B6A1BB128469847D4F8E0509DF818105F
:10DA30000029C8D00DF119042B6828461B689847A7
:10DA400014F8011B0029F7D1BDE7D4F8E470002FCA
:10DA5000B9D0304426ABFD2206A9841C1846ADF887
:10DA600010202246CDF81250ADF816507AF006F983
:10DA700002220346044402A93846CDE9023431F0BB
:10DA800019F80DF5277DBDE8F04002B07047D4F8D5
:10DA9000E430002B8DD196E7A0660024C43B00241F
:10DAA000D34D6210384D0D08CDC7040838B5184C59
:10DAB0000330D4F8F02002EB9003B3F5007F18D8C0
:10DAC00004EB810104F1F40520F00300C4F8F03008
:10DAD00005EB8205D1F8F428C3F5007310440D4A14
:10DAE0009B00C1F8F40804210020FFF759FF2846E5
:10DAF00038BD0021084A00250846FFF751FFD4F839
:10DB00007C39284643F00073C4F87C3938BD00BF27
:10DB1000A0660024444D0D08684D0D0838B5056811
:10DB20000446EB69F3B1987800B938BDB3F90A201F
:10DB3000012007EE902AF8EEE77AC4ED057AB3F9F2
:10DB40000C2007EE902AF8EEE77AF1EE677AC4ED42
:10DB5000047AB3F90E3007EE903AF8EEE77AC4EDA6
:10DB6000067A38BD09211420FFF7A0FF0346E861BB
:10DB7000D9E700BF38B505680446EB69E3B198788A
:10DB800000B938BDB3F90420012007EE902AF8EE61
:10DB9000E77AC4ED047AB3F9062007EE902AF8EE8E
:10DBA000E77AC4ED057AB3F9083007EE903AF8EE5B
:10DBB000E77AC4ED067A38BD09211420FFF776FF15
:10DBC0000346E861DBE700BF38B505680446EB694A
:10DBD000E3B1987800B938BD9A880120D2BA07EE2F
:10DBE000902AF8EEE77AC4ED047ADA88D2BA07EE22
:10DBF000902AF8EEE77AC4ED057A1B89DBBA07EEC6
:10DC0000903AF8EEE77AC4ED067A38BD092114207F
:10DC1000FFF74CFF0346E861DBE700BF38B5056856
:10DC20000C46EB697BB1987800B938BD5B8901205F
:10DC3000084ADBBA82FB0312DB17C3EB221303F2A1
:10DC40006D13238038BD09211420FFF72FFF0346F1
:10DC5000E861E8E7797878782DE9F04103EB43064D
:10DC6000964686B0034602EB4606754612F9067BD9
:10DC7000A3EB070C92F80080BCF1000FA3EB0804A3
:10DC8000B8BFCCF1000C002CB8BF6442644502DA86
:10DC900015464FFA88F70632B242E9D1688803E0A8
:10DCA0000EF1060E764518D09EF800208446BA4242
:10DCB000F6D10A1ABEF80280002AA1EB0804B8BF08
:10DCC0005242002CB8BF64429442E9DA75460EF124
:10DCD000060E4046C4467645E6D16879CDF808C0C0
:10DCE0002A78049028790192039001200091032161
:10DCF000034AFFF755FE284606B0BDE8F08100BF95
:10DD0000784D0D0803685A1C02601878704700BFF0
:10DD100003681A46591C016012F8021B0260587809
:10DD200041EA0020704700BF02681346511C0160A1
:10DD300013F802CB0360D31C5178036093781B0463
:10DD400043EA0123111D43EA0C030160D07843EA42
:10DD50000060704712B370B50446864604E0981B15
:10DD600017D114EB0C0C15D01EF8013BA3F14100A8
:10DD7000A2EB0E0C192811F8010BA0F1410598BF78
:10DD8000203300F12006192DE9D91B1A04D10028EF
:10DD9000E7D170BD604670BD184670BD1046704733
:10DDA00003880021184AA3F5FA6C70B503F0030448
:10DDB00090F802E0154E40F2B5550EF1FF3E04EB2F
:10DDC00044044FEA9C0C0EEB8403C47836F81330FD
:10DDD000013C05FB0C3390F804C02344847903EB29
:10DDE000430322444FF47A740CEBC30C437900894B
:10DDF000CCEB0C1C03EB8C03C3EB031302EB830291
:10DE0000C2FB040170BD00BF80436D3878A30C08CD
:10DE10002DE9F04116461F46404D0446394630462E
:10DE20004FF47A72002373F005FC3D4B05443D4FDF
:10DE30003D4E83FB0510E9172844C1EB601183FBBD
:10DE40000103C8170B44C0EB631087FB003CC317EA
:10DE5000C3EBAC0386FB03764FEAE37ECEEBE61E14
:10DE6000C1EB0116A5EB860CC0EB00154FEA8E0640
:10DE700084F806C0A1EB8501617103EB4301A0EBBF
:10DE8000C10040F2B55101FB1E332071B3F5896F1B
:10DE900033DA40F2DA218B4237DCB3F5B77F234F18
:10DEA000B4BF4FF0000E4FF0010E0EEB4E01754661
:10DEB0004FEA4E0807EBC101C88A08EB0E0C0B2194
:10DEC00007EBCC0C0CF1160C01E03CF8020D98426B
:10DED00010DD0139F9D1F044012137F8380006F599
:10DEE000FA6E0133A17075441B1A22812580E370FC
:10DEF000BDE8F0810131C9B2F1E7032540F2965047
:10DF00000A4F4FF00608AE46D7E7022540F22940F7
:10DF1000064F4FF00408AE46CFE700BF80BC92C763
:10DF200089888888ABAAAA2A73B06D1678A30C08D2
:10DF300030B5304C8DB086460D46EC461EF0030FD2
:10DF40000FCCACE80F000FCCACE80F0094E80F004A
:10DF50008CE80F000FD1284B284A03FB0EF3B2EBDD
:10DF6000B30F44D3264AB2EB331F34BF0122002241
:10DF7000C2F11D0200E01C220EF1FF33019240F2BB
:10DF80006D122048002B194602FB0EF21E4CB8BF42
:10DF90000EF10201EE4602EBA10280FB0310DB173B
:10DFA000ADF1040101EB8501A3EB6015C3EBE013B8
:10DFB0002A441A44253284FB0230D3171044C3EBA1
:10DFC000A003C3EBC303D31A5EF8040FC218714554
:10DFD00084FB023C4FEAE2739444C3EBAC03C3EB13
:10DFE000C303A2EB0303EFD1C01A0DB030BD1D2255
:10DFF000C2E700BFD8A30C08295C8FC2285C8F023F
:10E000000AD7A3001F85EB51932449920E4B10B5FC
:10E01000D3F88049D3F8843954EA03020AD101467F
:10E02000002340F2011218460B80C1F802208B71C8
:10E030000B8110BD054A1268121943F10003FFF766
:10E04000E7FE012010BD00BFA0660024C43B0024F1
:10E0500030B5144D83B00446D5F88019D5F884390D
:10E0600051EA03020AD1002340F20112184623802C
:10E07000C4F80220A371238103B030BD0A4A12689C
:10E08000521843F10003FFF7C3FEB5F88839204664
:10E090000DF106022146ADF8063067F091FF012030
:10E0A00003B030BDA0660024C43B002488422DE9A3
:10E0B000F04198464FF0010439D301FB04F4B0FB62
:10E0C000F4FC8C45F9D264B30025BCF1000F04FBCD
:10E0D0001C00B4FBF1F7D4BF002601266DB966B968
:10E0E000A142354619D9C6460CF1300C0EF801CBC9
:10E0F00000238EF80030BDE8F081BCF1090F18DD77
:10E10000002A0CBF57233723C6466344A14205F1BA
:10E1100001050EF8013BF046EAD83C46B0FBF7FC9F
:10E12000D3E7C64600238EF80030BDE8F081844670
:10E13000CAE73023E8E700BF2DE9F0410446154661
:10E1400008469442B4FBF2F607D205FB1644134B83
:10E150001B5D00F8013BBDE8F0819642B6FBF2F78B
:10E160000CD20E4B05FB176705FB1644DA5D1B5DF1
:10E1700000F8012B00F8013BBDE8F081BA42B7FB83
:10E18000F2F807D905FB1878044B13F8082000F8BB
:10E19000012BE7E74046FFF7CFFFF3E7B44D0D084B
:10E1A000B5EEC00ADFED357A0023F1EE10FA30B596
:10E1B000C8BF30EE270A87B0D8BF30EE670ADFED60
:10E1C000307A054603A9029320EE270ACDE90033F1
:10E1D000FDEEC07A17EE904A84EAE470A0EBE4709A
:10E1E00069F014F8002C03A8B4BF2D2320238DF868
:10E1F000003072F005FC01282AD0022834D0032810
:10E200001ED003A968467BF021FD684672F0F8FB3A
:10E21000044669462846033CE4B2224679F02EFDC6
:10E22000002328462B5572F0EBFB2E22431C0DEBEE
:10E2300004012A54E8187BF07EFD284607B030BD63
:10E24000302303A968468DF801307BF0FFFCDCE742
:10E2500043F23002302303A96846ADF801208DF85F
:10E2600003307BF0F3FCD0E743F2300303A96846A8
:10E27000ADF801307BF0EAFCC7E700BF6F12033A4C
:10E2800000007A440378202B03D110F8013F202BA3
:10E29000FBD0092BF9D02D2B63D02B2BB7EE000A26
:10E2A00008BF01300278A2F13003D9B2092961D840
:10E2B000F2EE046ADFED4D7A07EE103A10F8012F06
:10E2C000B8EEC77AA2F13003D9B2A7EEA67A09292F
:10E2D000F0EE477AF0D92E2A50D0037803F0DF030E
:10E2E000452B3BD110B442782D2A73D02B2A62D013
:10E2F000A2F130030130092B63D80024002303EB83
:10E30000830302EB430310F8012FA2F13001303BED
:10E310000929F4D9B3F59A7F1A46B7EE007A28BFD7
:10E320004FF49A72072B09D91346DFED316A083B87
:10E3300027EE267A072BFAD802F007022AB1F2EE6E
:10E34000046A013A27EE267AFBD1002C3BD0C7EEB7
:10E35000877A5DF8044B20EE270A704720EE270AE3
:10E36000704742780130BFEE000AA2F13003D9B203
:10E3700009299DD92E2ADFED1D7AAED143780130CF
:10E38000A3F13002D1B20929A8D8B2EE047AF0EE96
:10E39000475A06EE902A10F8013FB8EEE66AA3F15C
:10E3A0003002D1B2C6EE076A092927EE257A77EE48
:10E3B000A67AEED992E782780230A2F13003092BD7
:10E3C0009BD9B7EE007A67EE877A5DF8044B20EEB2
:10E3D000270A704782780230A2F13003092B01D856
:10E3E00001248BE7B7EE007AB1E700BF0000000020
:10E3F00020BCBE4C0378092B01D0202B05D110F88E
:10E40000013F202BFBD0092BF9D02D2B09D001780F
:10E410004FF0010CA1F13002D3B2092B0AD9002030
:10E420007047417801304FF0FF3CA1F13002D3B288
:10E43000092BF4D8002310F8011F03EB830302EB30
:10E440004303A1F13002D1B20929F4D90CFB03F046
:10E45000704700BFAB4BAC4A2DE9F04F4FF0000ABC
:10E4600097B09E1A41F221051F462C2200210DEB88
:10E4700002007AF02BFDA44AA44B0892CDE909765C
:10E48000DA68D10707D5A24A5A6002F188325A6089
:10E49000DB68DC070DD49D4BD3F80C21D20708D5DF
:10E4A0009B4AC3F8042102F18832C3F80421D3F84F
:10E4B0000C31002101227E2308A8149105A98DF8B2
:10E4C00054208DF81430FEF7B3FC0028C0F22981E7
:10E4D00008214FF4FC4303E05B0001399BB207D0F5
:10E4E0001AB2002AF8DA85EA4202013993B2F7D16A
:10E4F000884AADF81630884B934280F05181984697
:10E500000DF11809CDE902A7B8F802204FF0000C70
:10E51000B8F80030C2F30B0B10048DF81DC00BF1DE
:10E520000601ADF81810C3F30B014FEA1333ADF831
:10E530001A108DF81C3000F191800622494608A877
:10E54000FEF776FC0028C0F2FD80BDF81640494673
:10E550000DF11E0011F8013B082284EA032403E0B8
:10E560006400013AA4B207D023B2002BF8DA85EA9E
:10E570004303013A9CB2F7D18842EBD15A46D8F80E
:10E58000041008A8FEF754FC0028C0F2DB80D8F87D
:10E59000041001EB0B00814215D00139013811F84C
:10E5A000013F082284EA032403E06400013AA4B294
:10E5B00007D023B2002BF8DA85EA4303013A9CB274
:10E5C000F7D18142EBD1ADF8164008F11408514B58
:10E5D000984599D3DDE902A700230222494608A8FD
:10E5E000ADF81830FEF724FC0028C0F29A80BDF880
:10E5F00016300DF11A0041F2210119F8012B0824FF
:10E6000083EA022303E05B00013C9BB207D01AB20D
:10E61000002AF8DA81EA4202013C93B2F7D1484578
:10E62000EBD102220DF1160108A8ADF81630FEF765
:10E63000FFFB002875DB1398002840F089801498B0
:10E6400000286EDB9DF85420002A40F097800028B7
:10E650000DBF012200220123002364E0E246674649
:10E66000019601370622494608A8FFB28DF81D70B1
:10E67000FEF7DEFB002851DBBDF8164049460DF1E0
:10E680001E0011F8013B082284EA032403E0640021
:10E69000013AA4B207D023B2002BF8DA85EA43038B
:10E6A000013A9CB2F7D18842EBD1D8F804105A460F
:10E6B00008A801EB0A063146FEF7BAFB00282DDB5D
:10E6C00006EB0B00864215D0711E013811F8013F90
:10E6D000082284EA032403E06400013AA4B207D0CC
:10E6E00023B2002BF8DA85EA4303013A9CB2F7D152
:10E6F0008142EBD1032FDA44ADF81640B1D1019E2F
:10E7000063E700BF00000408000002080020005278
:10E7100023016745DC090E0828040E08DDE9016ABB
:10E72000039F012300220AF1010ABAF1020F02DC61
:10E73000002B7FF49AAE12B1FEF75CF828B90520E1
:10E7400006F0ACFEDDE902A7EBE717B0BDE8F08FFD
:10E75000089B099A03449342E3D80BABC0F1200213
:10E76000214618447AF0B2FB149818B90BA908A8EE
:10E77000F4F7D8F800221490139261E70A4AD1689E
:10E7800041F00101D160D168C9077FF560AFD2F8CF
:10E790000C1141F00101C2F80C11D2F80C2156E71E
:10E7A0000DF1180918E700BF0020005270B5458828
:10E7B0000B4604460021C5F30B0518462A467AF09D
:10E7C00085FB0A4A21690346914206D3084A9142D1
:10E7D00006D31846BDE8704008470029F9D170BD3E
:10E7E0002A46BDE8704079F049BA00BFDC090E083E
:10E7F0000F0F0E0810B50446C06900B110BD092105
:10E800001420FFF753F9E06110BD00BF174A02EB77
:10E810008000C06830B3164B00EB400003EB800370
:10E8200093F901C0BCF1FF3F1DD0587AD0B102EB83
:10E830000C00142210B590F88CE98C20197A002372
:10E8400000FB0CFC0B4C0CEB0100013A714434F85A
:10E85000100013FA80F3F6D1074AA2FB0320C0F39D
:10E860000F1010BD70470020704700BFA066002445
:10E87000202E002400000030CDCCCCCC036810B595
:10E880001A790446022A03D000232360237110BDA5
:10E89000987A04F03FFA0028F6D040F61A61002278
:10E8A000C1802021027204F0F1F90023236023715A
:10E8B00010BD00BF2DE9F04FBA4E85B0BA4CA6424C
:10E8C00056D21D4602E00C36A64251D273798B42D5
:10E8D000F9D13379834201D00028F4D1F3799342FE
:10E8E000F1D13468002C43D0002326606360A3601C
:10E8F000E36023616361A361E36133792371012BD9
:10E9000096F806B0C4F808B0317AE16032D0022B34
:10E910002ED1F07A04F0FEF996F90970A061B07A70
:10E92000277404F0F7F906466061F0B1DFF89482CD
:10E9300007EB47017B0058F8319008EBC1010193C8
:10E94000B9F1000F11D0887DE8B10E2200230D210E
:10E950003046F2713372B57104F098F93368B288B9
:10E960009A61204605B0BDE8F08F2046FFF786FF8C
:10E970000024F6E7F07A04F0CDF9727AB37AA06158
:10E9800022746374EDE7B1F808A0504667F012FCFA
:10E9900001214FEA5A100AF01F0A023801FA0AF15F
:10E9A000092812D8DFE810F0F6001100EE00180177
:10E9B0001001E600E000D800D0000A007B4BD3F83D
:10E9C0009C0020EA0101C3F89C107B00D91908EBD8
:10E9D000C101487904F09EF9791CCBB2014601933C
:10E9E00018B1037240F60A30C8807B000291D81932
:10E9F00008EBC000C07904F08DF90299034603903A
:10EA000020B1019A027240F60A50D8807B00029130
:10EA1000D81908EBC000807904F07CF9029982468D
:10EA200028B1019B037240F60A40AAF806007B0059
:10EA3000D8191BF0040308EBC0000293807A024649
:10EA4000084614BF4E212E2104F042F903987B00A2
:10EA50002E2103EB070B08EBCB0B9BF80B2004F0EC
:10EA600037F950469BF80C200E2104F031F99BF841
:10EA700004A0BAF1000F40F0ED80D9F8002022F098
:10EA80000102C9F800204A4A914500F0C180494A74
:10EA9000914540F0AC80454AD2F8901041F4804155
:10EAA000C2F89010D2F8901021F48041C2F8901072
:10EAB000029B002B40F098804FF000714FF0807265
:10EAC000D9F80C0040F00040C9F80C00D9F8080053
:10EAD00020F4F070C9F80800D9F80000C00727D466
:10EAE000D9F80800344B034034481843C9F80800EB
:10EAF000D9F80C00C30005D4D9F8000040F48050C8
:10EB0000C9F80000D9F80C0011432D4A02400A430D
:10EB100042F08862C9F80C20D9F8002022F4006283
:10EB2000C9F80020D9F8502022F00102C9F850207D
:10EB3000BAF1000F40F09B807B003B4408EBC30818
:10EB4000012388F8163000E7184BD3F8880020EA34
:10EB50000101C3F8881038E7144BD3F88C0020EA81
:10EB60000101C3F88C1030E7104BD86F20EA010187
:10EB7000D9672AE70D4BD3F8940020EA0101C3F8C6
:10EB8000941022E7094BD3F8800020EA0101C3F872
:10EB900080101AE7054BD3F8980020EA0101C3F86A
:10EBA000981012E7A00200088004000800440258F0
:10EBB0000030014000380040E0FFBF8F0700002018
:10EBC000FFFF39D8080500243E4BD3F8900020EA17
:10EBD0000101C3F89010F8E63A4BD3F8840020EA1C
:10EBE0000101C3F88410F0E600210A4668E7364ABE
:10EBF00091451BD1334AD2F8901041F40041C2F83C
:10EC00009010D2F8901021F40041C2F890104FE714
:10EC10002C4AD2F8981041F48051C2F89810D2F8DA
:10EC2000981021F48051C2F8981041E7274A914585
:10EC300027D0274A914532D1224AD2F8981041F480
:10EC40008011C2F89810D2F8981021F48011C2F8FF
:10EC500098102DE7504604F05DF820B1019B40F676
:10EC60000A620372C2800D2104F010F805E75046D5
:10EC700004F050F800283FF45FAF02688388936186
:10EC80005AE7104AD2F8981041F40051C2F898108F
:10EC9000D2F8981021F40051C2F8981008E70D4AF4
:10ECA00091457FF405AF02F50C32D2F89C1041F08B
:10ECB0002001C2F89C10D2F89C1021F02001C2F86B
:10ECC0009C10F5E600440258003C0040003401402E
:10ECD0000050014000140058104B70B5104CA34276
:10ECE00019D2054602E00C33A34214D293F805C0B2
:10ECF0008C45F8D193F804C00DB1AC45F3D1D87967
:10ED00009042F0D1186890F804E0E645EBD106682F
:10ED10009E42E8D170BD002070BD00BFA002000877
:10ED2000800400080379022B00D0704790F910206E
:10ED300008311C4802EB420210B41B4C83B050F85F
:10ED4000322000946944194C11F808CCA24224D016
:10ED500017498A4223D001F580618A4205D0154BBC
:10ED60009A420CBF03234FF0FF33116803EB4303B8
:10ED700021F0010100EBC30011600169936851F8B3
:10ED80002C1023F0E0430B439360136843F001031E
:10ED9000136003B05DF8044B70470023E5E70123DF
:10EDA000E3E700BF08050024000102030030014032
:10EDB000003800400034014090F91030F0B503EB0A
:10EDC0004303284E154683B056F8336004468368E3
:10EDD0009A0719D501230DF106028DF80610304669
:10EDE0000DF10701F6F766F801230DF106020DF1AA
:10EDF000070130468DF80650F6F75CF8A3689B07CC
:10EE000016D5012003B0F0BD43691BB19A8818687C
:10EE100012048261144B154A1868154BC0005768DC
:10EE2000A3FB003080095368DB1B9842FBD2D1E77B
:10EE30000D4A4FF4FA700E4B12680C4900FB02F2B7
:10EE40004868A3FB023292094B681B1A9A42FBD214
:10EE50006369002BD5D01A6801209B88936103B0A9
:10EE6000F0BD00BF08050024E4330024001000E0DA
:10EE7000D34D621010B5037984B084468E46012BC1
:10EE80000DD0022B02D0002004B010BD8368DB0738
:10EE900058BF01F07F0104B0BDE810408CE78168E5
:10EEA0000DF10F001446724601F001018DF80F407C
:10EEB000CDE900019CF811109CF91000F5F7F0FA6B
:10EEC00004B010BD2DE9F0410768642682B0B62277
:10EED0007E2180463846FFF7CDFF05F001FE04464F
:10EEE0000D4605F0FDFD001B61EB0501B0F57A7FD5
:10EEF00071F10001F5D3013EEFD102213846FFF751
:10EF000011FF7B691BB19A88196812048A6105F0A8
:10EF1000E7FD04460D4605F0E3FD001B61EB05012E
:10EF2000B0F57A7F71F10001F5D37B6913B11A68EE
:10EF30009B8893610A2605F0D3FD04460D4605F033
:10EF4000CFFD001B61EB0501B0F57A7F71F1000187
:10EF5000F5D3013EEFD132467C213846FFF78AFFD8
:10EF600005F0BEFD04460D4605F0BAFD001B61EB41
:10EF70000501B0F57A7F71F10001F5D30022592126
:10EF80003846FFF777FF05F0ABFD04460D4605F068
:10EF9000A7FD001B61EB0501B0F57A7F71F100015F
:10EFA000F5D397F910305E218D4A03EB43038DF8BA
:10EFB000071052F83340BB689A0740F1E480012300
:10EFC0000DF1070200212046F5F774FF4FF4A473FA
:10EFD000844A20460021F5F76DFFBB689B0740F18E
:10EFE000E6800A2605F07CFD04460D4605F078FD16
:10EFF000001B61EB0501B0F57A7F71F10001F5D3DB
:10F00000013EEFD1012259213846FFF733FF05F0C9
:10F0100067FD04460D4605F063FD001B61EB05012D
:10F02000B0F57A7F71F10001F5D38C22402138468A
:10F03000FFF720FF05F054FD04460D4605F050FD96
:10F04000001B61EB0501B0F57A7F71F10001F5D38A
:10F05000032241213846FFF70DFF05F041FD04462C
:10F060000D4605F03DFD001B61EB0501B0F57A7F13
:10F0700071F10001F5D35C4C0323D8F8382098F8DF
:10F080003500B4FBF2F291B2584AFEF7E5FD438831
:10F090004221B4FBF3F4C8F840400279384642F00C
:10F0A000C002FFF7E7FE05F01BFD04460D4605F024
:10F0B00017FD001B61EB0501B0F57A7F71F10001CE
:10F0C000F5D3082243213846FFF7D4FE05F008FDAA
:10F0D00004460D4605F004FD001B61EB0501B0F58B
:10F0E0007A7F71F10001F5D3042258213846FFF7E9
:10F0F000C1FE05F0F5FC04460D4605F0F1FC001BD1
:10F1000061EB0501B0F57A7F71F10001F5D30A22B8
:10F1100053213846FFF7AEFE05F0E2FC04460D46EB
:10F1200005F0DEFC001B61EB0501B0F57A7F71F1A3
:10F130000001F5D300227C213846FFF79BFE05F045
:10F14000CFFC04460D4605F0CBFC001B61EB05012E
:10F15000B0F57A7F71F10001F5D306227D213846A2
:10F16000FFF788FE05F0BCFC04460D4605F0B8FC30
:10F17000001B61EB0501B0F57A7F71F10001F5D359
:10F1800002B0BDE8F0817B691BB11A689B881B0443
:10F190009361174B17491A68174BD2004868A3FBB5
:10F1A000023292094B681B1A9A42FBD207E7104AB7
:10F1B0004FF4FA70104B12680E4900FB02F24868D7
:10F1C000A3FB023292094B681B1A9A42FBD27B695D
:10F1D000002B3FF406AF1A689B88936101E700BFDC
:10F1E0000805002408A40C0840420F0050A50C0894
:10F1F000E4330024001000E0D34D62102DE9F0410B
:10F20000816B0623654D044607686426644A90F8BE
:10F210003500B5FBF1F189B2FEF71EFD43880021F0
:10F2200080463846B5FBF3F52564FFF77BFD802269
:10F230006B213846FFF71EFE05F052FC04460D46D2
:10F2400005F04EFC001B61EB0501B0F57A7F71F112
:10F250000001F5D3013EEFD164260722682138462C
:10F26000FFF708FE05F03CFC04460D4605F038FCAF
:10F27000001B61EB0501B0F57A7F71F10001F5D358
:10F28000013EEFD1324664266B213846FFF7F2FD8E
:10F2900005F026FC04460D4605F022FC001B61EB40
:10F2A0000501B0F57A7F71F10001F5D3013EEFD190
:10F2B0000F2601226B213846FFF7DCFD05F010FC1C
:10F2C00004460D4605F00CFC001B61EB0501B0F592
:10F2D0007A7F71F10001F5D3013EEFD10F2618229C
:10F2E0001B213846FFF7C6FD05F0FAFB04460D4624
:10F2F00005F0F6FB001B61EB0501B0F57A7F71F1BB
:10F300000001F5D3013EEFD10F2618221C2138460B
:10F31000FFF7B0FD05F0E4FB04460D4605F0E0FB09
:10F32000001B61EB0501B0F57A7F71F10001F5D3A7
:10F33000013EEFD10F2698F804201A213846FFF736
:10F3400099FD05F0CDFB04460D4605F0C9FB001BF9
:10F3500061EB0501B0F57A7F71F10001F5D3013E53
:10F36000EFD1642698F8052019213846FFF782FD71
:10F3700005F0B6FB04460D4605F0B2FB001B61EB41
:10F380000501B0F57A7F71F10001F5D3013EEFD1AF
:10F3900038460321BDE8F041C4E400BF40420F00FD
:10F3A00064A50C082AE700BF00680379012B09D087
:10F3B000022B01D0002070478368F022DB0717D5AD
:10F3C000FF21F9E4826890F910C002F00102417C4B
:10F3D00060464FF0F00C10B584B00DF10F040192AF
:10F3E000FF228DF80FC00094F5F75AF804B010BD55
:10F3F0007F21E1E40068CA43037941EA0211012B4D
:10F40000CAB208D0022B01D0002070478368DB0706
:10F4100015D5D221D0E410B584B0846890F910C01D
:10F420008DF80F200DF10F0204F00104417C0092D1
:10F43000D22260460194F5F733F804B010BD522192
:10F44000BAE400BF00680379012B09D0022B01D078
:10F45000002070478368B422DB0717D5FF21ABE497
:10F46000826890F910C002F00102417C60464FF0C2
:10F47000B40C10B584B00DF10F040192FF228DF889
:10F480000FC00094F5F70CF804B010BD7F2193E491
:10F4900000680379012B09D0022B01D000207047AE
:10F4A00083680A46DB0715D5A52185E410B584B02D
:10F4B000846890F910C00DF10F0204F001048DF87A
:10F4C0000F10417C60460092A5220194F4F7E8FFFA
:10F4D00004B010BD25216FE400680379012B09D029
:10F4E000022B01D00020704783689622DB0717D5D6
:10F4F000FF2161E4826890F910C002F00102417CB2
:10F5000060464FF0960C10B584B00DF10F040192D7
:10F51000FF228DF80FC00094F4F7C2FF04B010BDB5
:10F520007F2149E400680379012B09D0022B01D027
:10F530000020704783680A46DB0715D587213BE426
:10F5400010B584B0846890F910C00DF10F0204F07A
:10F5500001048DF80F10417C6046009287220194CF
:10F56000F4F79EFF04B010BD072125E40068C9012F
:10F570000379CAB2012B05D0022B01D000207047BD
:10F58000782119E410B584B0846890F910C08DF822
:10F590000F200DF10F0204F00104417C009278224B
:10F5A00060460194F4F77CFF04B010BD0068037955
:10F5B000012B0AD0022B01D000207047836855220E
:10F5C000DB0718D5A521FFF7F7BB826890F910C0BB
:10F5D00002F00102417C60464FF0550C10B584B03A
:10F5E0000DF10F040192A5228DF80FC00094F4F7DD
:10F5F00057FF04B010BD2521FFF7DEBB006803797B
:10F60000012B0AD0022B01D00020704783682E22E4
:10F61000DB0718D5F421FFF7CFBB826890F910C043
:10F6200002F00102417C60464FF02E0C10B584B010
:10F630000DF10F040192F4228DF80FC00094F4F73D
:10F640002FFF04B010BD7421FFF7B6BB154B006847
:10F650009A8F03799201012B02F13402D2B209D0C0
:10F66000022B01D0002070478368DB0716D5F421F8
:10F67000FFF7A2BB10B584B0846890F910C08DF874
:10F680000F200DF10F0204F00104417C0092F422DE
:10F6900060460194F4F704FF04B010BD7421FFF735
:10F6A0008BBB00BFA0660024006810B5037984B04E
:10F6B000012B0FD0022B02D0012004B010BD8368B3
:10F6C0003122DB074CBFF4217421FFF775FB0120C9
:10F6D00004B010BD82680DF10F0490F910C002F063
:10F6E0000102417C60464FF0310C0192F4220094FB
:10F6F0008DF80FC0F4F7D4FE012004B010BD00BF98
:10F7000000680379012B07D0022B01D0002070473D
:10F7100001225821FFF750BB8268417C02F00102B0
:10F7200010B590F9104084B020460DF10F040192FD
:10F73000582200948DF80F30F4F7B2FE04B010BDDB
:10F7400000680379012B07D0022B01D000207047FD
:10F7500001224821FFF730BB8268417C02F00102A0
:10F7600010B590F9104084B020460DF10F040192BD
:10F77000482200948DF80F30F4F792FE04B010BDCB
:10F7800000680379012B07D0022B01D000207047BD
:10F790001A460821FFF710BB826890F910C002F0EA
:10F7A0000102417C60464FF0020C10B584B00DF1AF
:10F7B0000F04019208228DF80FC00094F4F770FE38
:10F7C00004B010BD00680379012B07D0022B01D0D3
:10F7D0000020704701220821FFF7EEBA8268417CC1
:10F7E00002F0010210B590F9104084B020460DF1EE
:10F7F0000F040192082200948DF80F30F4F750FEA8
:10F8000004B010BD2DE9F04105461F4628481646B4
:10F8100095F9103082B003EB430350F83380AB68A6
:10F820009A0716D501230DF106028DF80610404601
:10F830000DF10701F5F73EFB3B46324600214046FD
:10F84000F5F738FBAB689B0718D5012002B0BDE87F
:10F85000F0816B691BB19A88186812048261154B9C
:10F860001868154BC000A3FB0030144B80095A6880
:10F870005C68A4EB020C6045FAD2D3E70D4A4FF462
:10F88000FA700D4B12680D4900FB02F24868A3FBA9
:10F89000023292094B681B1A9A42FBD26B69002B09
:10F8A000D3D01A6801209B88936102B0BDE8F08133
:10F8B00008050024E4330024D34D6210001000E05A
:10F8C00030B5057983B084468E46012D0DD0022DCA
:10F8D00002D0002003B030BD8468E40758BF41F077
:10F8E000800103B0BDE830408CE7806814460A46CA
:10F8F000009400F001049CF811109CF91000019490
:10F90000F4F7CEFD03B030BD2DE9F04105461F46AA
:10F910002848164695F9103082B003EB430350F89F
:10F920003380AB689A0716D501230DF106028DF8D6
:10F93000061040460DF10701F5F7BCFA3B460022E0
:10F9400031464046F5F7B6FAAB689B0718D501205B
:10F9500002B0BDE8F0816B691BB19A881868120487
:10F960008261154B1868154BC000A3FB0030144B87
:10F9700080095A685C68A4EB020C6045FAD2D3E7B0
:10F980000D4A4FF4FA700D4B12680D4900FB02F25C
:10F990004868A3FB023292094B681B1A9A42FBD2B9
:10F9A0006B69002BD3D01A6801209B88936102B049
:10F9B000BDE8F08108050024E4330024D34D621033
:10F9C000001000E030B5057983B084468E46012DE5
:10F9D0000DD0022D02D0002003B030BD8468E407B2
:10F9E00058BF41F0800103B0BDE830408CE780682B
:10F9F00014460A46009400F001049CF811109CF98A
:10FA000010000194F4F760FF03B030BD2DE9F0431E
:10FA1000816B85B0804C0623076880467F4A962616
:10FA200090F83500B4FBF1F189B2FEF715F943887F
:10FA3000002181463846B4FBF3F4C8F84040FFF794
:10FA400071F980226B213846FFF714FA05F048F867
:10FA500004460D4605F044F8001B61EB0501B0F5C6
:10FA60007A7F71F10001F5D3013EEFD19626032292
:10FA700068213846FFF7FEF905F032F804460D46D6
:10FA800005F02EF8001B61EB0501B0F57A7F71F1EE
:10FA90000001F5D3013EEFD103226B213846FFF779
:10FAA000E9F905F01DF804460D4605F019F8001BAC
:10FAB00061EB05010F2871F10001F6D310226A21D4
:10FAC0003846FFF7D7F905F00BF804460D4605F068
:10FAD00007F8001B61EB05010F2871F10001F6D357
:10FAE00000226C213846FFF7C5F904F0F9FF0446FF
:10FAF0000D4604F0F5FF001B61EB05010F2871F1C5
:10FB00000001F6D399F8052019213846FFF7B2F91C
:10FB100004F0E6FF04460D4604F0E2FF001B61EB33
:10FB200005010F2871F10001F6D318221B21384678
:10FB3000FFF7A0F904F0D4FF04460D4604F0D0FF0F
:10FB4000001B61EB05010F2871F10001F6D31822AB
:10FB50001C213846FFF78EF904F0C2FF04460D461B
:10FB600004F0BEFF001B61EB05010F2871F10001DD
:10FB7000F6D399F804201A213846FFF77BF904F0F0
:10FB8000AFFF05460C4604F0ABFF8C4208BF854230
:10FB9000F9D003213846FFF7C5F8062302AA43210E
:10FBA000D8F80000FFF70EFF28B3BDF80810BDF825
:10FBB0000A30BDF80C20C9BADBBA07EE901AD2BAE7
:10FBC000F8EEE76A07EE102A07EE903AB8EEC77A29
:10FBD000F8EEE77AC8ED076A88ED097AC8ED087A89
:10FBE000FDEEE77ACDED017A9DF90430013305D0C1
:10FBF00005B0BDE8F083D8ED087AF1E7D8ED077AD3
:10FC0000FDEEE77ACDED017A9DF904300133EFD1B5
:10FC1000062005F043FC00BF40420F0064A50C081D
:10FC200070B5066882B00546F469002C3ED0337981
:10FC3000221D012B2DD0022B26D1B368304613F0A4
:10FC4000010F4FF00C030CBF8C211946FFF75CFE2F
:10FC5000A070D8B1B4F9043007EE903AF8EEE77A24
:10FC6000C5ED077AB4F9063007EE903AF8EEE77A78
:10FC7000C5ED087AB4F9083007EE903AF8EEE77A65
:10FC8000C5ED097A02B070BD0023A370002002B058
:10FC900070BDB368717C03F0010396F91000009207
:10FCA00001930C231A46F4F70FFED1E70921142023
:10FCB000FDF7FCFEF06104462E68B8E770B50668F3
:10FCC00082B00546F469002C3ED03379E21C012B4A
:10FCD0002DD0022B26D1B368304613F0010F4FF020
:10FCE0000D0314BF0C218C21FFF70EFEA070D8B1BC
:10FCF000B4F90A3007EE903AF8EEE77AC5ED077AE4
:10FD0000B4F90C3007EE903AF8EEE77AC5ED087AD0
:10FD1000B4F90E3007EE903AF8EEE77AC5ED097ABD
:10FD200002B070BD0023A370002002B070BDB368A4
:10FD3000717C03F0010396F9100000920C220193EC
:10FD40000D23F4F7C1FDD1E709211420FDF7AEFE24
:10FD5000F06104462E68B8E7006810B5037984B0F6
:10FD60000C46012B1AD0022B02D0002004B010BD8B
:10FD7000836803AA13F0010F4FF0030314BF22217D
:10FD8000A221FFF7C1FD0028EFD0BDF90D3003EB34
:10FD900083031B12E633238004B010BD836803AADB
:10FDA000417C03F0010390F910000092222201939C
:10FDB0000323F4F789FDE6E770B5066882B00546CF
:10FDC000F469002C3ED03379221D012B2DD0022B5B
:10FDD00026D1B368304613F0010F4FF00E0314BF65
:10FDE0003B21BB21FFF790FDA070D8B1A389DBBAFE
:10FDF00007EE903AF8EEE77AC5ED077AE389DBBAC9
:10FE000007EE903AF8EEE77AC5ED087A238ADBBA76
:10FE100007EE903AF8EEE77AC5ED097A02B070BDC8
:10FE20000023A370002002B070BDB368717C03F0A2
:10FE3000010396F9100000923B2201930E23F4F780
:10FE400043FDD1E709211420FDF730FE0446F0619F
:10FE5000B9E700BF006810B5037984B0012B10D05A
:10FE6000022B01D000200AE003AAF621FFF74CFD87
:10FE70000028F7D0BDF80C30094A5BBA938304B070
:10FE800010BD826803AC417C022302F0010290F9AC
:10FE90001000CDE90042F622F4F716FDE8E700BFB6
:10FEA000A0660024006810B5037984B0012B1DD032
:10FEB000022B01D0002017E0032303AAF621FFF74D
:10FEC00023FD0028F6D09DF80D309DF80CC01B02D4
:10FED0000D499DF80E2043EA0C431343B1F93C2031
:10FEE000C2F10802D3400B6404B010BD826803ACB9
:10FEF000417C032302F0010290F91000CDE9004299
:10FF0000F622F4F7E1FCDCE7A0660024006810B5F7
:10FF1000037984B0012B31D0022B09D01E49002077
:10FF2000D1F89039D1F894294B664A6404B010BDD9
:10FF3000062302AAF721FFF7E7FC0028EED09DF880
:10FF400009309DF80C209DF808C01B019DF80BE0BE
:10FF500012019DF80A1043EA0C3342EA0E329DF872
:10FF60000DC043EA11130C4942EA1C12C1F8903942
:10FF7000C1F894294A644B6604B010BD826802AC93
:10FF8000417C062302F0010290F91000CDE9004205
:10FF9000F722F4F799FCD0E7A0660024006810B5BA
:10FFA000037984B0012B1DD0022B0FD09DF80D30AA
:10FFB00001209DF80CC01B029DF80E10104A43EA68
:10FFC0000C430B43C2F88C3004B010BD836803AA05
:10FFD00013F0010F4FF0030314BF00218021FFF73E
:10FFE00093FCE3E7826803AC417C032302F0010247
:10FFF00090F91000CDE900420022F4F765FCD5E746
:020000040805ED
:10000000A0660024006810B5037984B0012B1DD0D0
:10001000022B0FD09DF80D3001209DF80CC01B0263
:100020009DF80E10104A43EA0C430B43C2F8A0306F
:1000300004B010BD836803AA13F0010F4FF003034F
:1000400014BF00218021FFF75FFCE3E7826803AC67
:10005000417C032302F0010290F91000CDE9004237
:100060000022F4F731FCD5E7A0660024006810B543
:10007000037984B0012B28D0022B01D0002022E08C
:10008000836803AA13F0010F4FF003030CBF832111
:100090001946FFF739FC0028F0D09DF80C309DF987
:1000A0000C109DF80D201B0400299DF80EC043EA9A
:1000B00002230D4AACBF00214FF07F4143EA0C03FD
:1000C0000B43C2F8BC3004B010BD826803AC0323FC
:1000D000417C02F0010290F91000CDE900421A467D
:1000E000F4F7F2FBD7E700BFA0660024006810B564
:1000F000037984B0012B28D0022B01D0002022E00C
:10010000836803AA13F0010F4FF0030314BF00210B
:100110008021FFF7F9FB0028F0D09DF80C309DF905
:100120000C109DF80D201B0400299DF80EC043EA19
:1001300002230D4AACBF00214FF07F4143EA0C037C
:100140000B43C2F8B83004B010BD826803AC417CE8
:10015000032302F0010290F91000CDE900420022D1
:10016000F4F7B2FBD7E700BFA066002490F9103087
:10017000F0B503EB4303264E154683B056F83360C3
:10018000044683689A0715D501230DF106028DF800
:10019000061030460DF10701F4F78CFE0123002212
:1001A00029463046F4F786FEA3689B0716D5012042
:1001B00003B0F0BD43691BB19A88186812048261CC
:1001C000144B154A1868154BC0005768A3FB003044
:1001D00080095368DB1B9842FBD2D5E70D4A4FF4E8
:1001E000FA700E4B12680C4900FB02F24868A3FB40
:1001F000023292094B681B1A9A42FBD26369002BA8
:10020000D5D01A6801209B88936103B0F0BD00BF70
:1002100008050024E4330024001000E0D34D6210F0
:1002200010B5037982B08E46012B0DD0022B02D07F
:10023000002002B010BD8368DB0758BF41F0800189
:1002400002B0BDE8104091E7816814467246009400
:1002500001F00104417C90F910000194F4F734FBA3
:1002600002B010BD70B5056884B004460E462B7907
:10027000012B15D0022B02D0002004B070BDAB685A
:10028000E122DB071CD528461146FEF795FD002824
:10029000F2D03246FF21206804B0BDE87040BFE7CD
:1002A000AA68697C02F0010295F910000DF10F05B2
:1002B0000192E12200958DF80F20F4F7F1F8E6E7BE
:1002C00061212846FEF778FDE1E700BF70B50568BB
:1002D00084B004460E462B79012B16D0022B02D097
:1002E000002004B070BDAB68C3222846DB074CBFBA
:1002F000E1216121FEF760FD0028F1D03246FF21A7
:10030000206804B0BDE870408AE7AA6895F910003B
:1003100002F00102697C01920DF10F020092C322EA
:100320008DF80F20E122F4F7BBF8E5E770B505681A
:1003300084B004460E462B79012B1BD0022B02D031
:10034000002004B070BDAB68F0222846DB074CBF2C
:10035000E1216121FEF730FD0028F1D02246FF2186
:1003600052F8040BFFF75CFF0028E9D023793370C3
:1003700004B070BDAA6895F9100002F00102697C12
:1003800001920DF10F020092F0228DF80F20E12270
:10039000F4F786F8E0E700BFF0B5046883B0002109
:1003A000074664262046FEF7BDFC15227E21204626
:1003B000FEF760FD04F094FB04460D4604F090FB4C
:1003C000001B61EB0501B0F57A7F71F10001F5D3F7
:1003D000013EEFD1052611227E213868FEF74AFD45
:1003E00004F07EFB04460D4604F07AFB001B61EB33
:1003F0000501B0F57A7F71F10001F5D3013EEFD12F
:100400000DF1070203213868FFF70AFF9DF8073056
:1004100003F03C03142B40F09B800C2240213868F1
:10042000FEF728FD04F05CFB04460D4604F058FB83
:10043000001B61EB0501B0F57A7F71F10001F5D386
:10044000454C0923B96B454A97F83500B4FBF1F1E7
:1004500089B2FDF701FC0346422138685A88B4FB93
:10046000F2F43C641A79FEF705FD04F039FB04460A
:100470000D4604F035FB001B61EB0501B0F57A7FFA
:1004800071F10001F5D3082241213868FEF7F2FC32
:1004900004F026FB04460D4604F022FB001B61EB32
:1004A0000501B0F57A7F71F10001F5D300224321F7
:1004B0003868FEF7DFFC04F013FB04460D4604F039
:1004C0000FFB001B61EB0501B0F57A7F71F10001B4
:1004D000F5D3102251213868FEF7CCFC04F000FB64
:1004E00004460D4604F0FCFA001B61EB0501B0F573
:1004F0007A7F71F10001F5D30A2253213868FEF7A3
:10050000B9FC04F0EDFA04460D4604F0E9FA001BCC
:1005100061EB0501B0F57A7F71F10001F5D380221E
:1005200056213868FEF7A6FC04F0DAFA04460D46B8
:1005300004F0D6FA001B61EB0501B0F57A7F71F18A
:100540000001F5D303213868FEF7ECFB03B0F0BDE2
:10055000062004F0A3FF00BF40420F00ACAA0C0825
:10056000F0B583B015461C4606460DF107020F464E
:10057000FFF756FE9DF8072005EA0203A34201D1CA
:1005800003B0F0BD22EA050239463046224303B0EB
:10059000BDE8F040FEF76EBC10B582B008210446FD
:1005A00000686A46FFF73CFE9DF80030DB0602D487
:1005B000002002B010BD06236A4600212068FFF724
:1005C00001FA0028F4D09DF801209DF800101202D5
:1005D0009DF80230DFED4A6A02EB01429DF80410FB
:1005E00014024FEA01219DF8034013449DF80520B1
:1005F00001EB044148BF03F17F430A44090207EEBF
:10060000903A404B48BF02F17F42F8EEE77A93ED13
:100610001C6A07EE102AB3F97420F8EEC65AB3F933
:100620007A10B8EEC77A04EE901AB3F97E10C7EECE
:10063000263A87EEA67A06EE902A334AD3ED1B7A45
:1006400092F88440B3F97620F8EEE66A112C06EEB3
:10065000102AB3F97820F8EEE77A05EE102AB3F9FC
:100660007C20B8EEC66A04EE102AB8EEC55AF8EE41
:10067000E44AB3F98020B8EEC44A66EEA36A27EED6
:10068000232A23D0A7EE045AA7EE246AE5EE075AE0
:10069000E5EE877A77EEA67AE6EE027AB3F96A207B
:1006A000F6EE006AC3ED217A07EE902AB3F96810DE
:1006B000F8EEE77A07EE101AB8EEC77A67EEA37A7B
:1006C000E7EE267AC3ED227A02B010BD03EE102ABF
:1006D000F8EEC32A03EE101AB8EEC33AA7EE224A88
:1006E000E7EE034AA4EE075AA4EE876AE5EE075A3E
:1006F000E5EE877A77EEA67AE6EE027ACEE700BFDD
:1007000000007848A066002478BB0024F0B50446B9
:1007100083B00D461746061D20680379012B19D0BA
:10072000022B02D0002003B0F0BD83683246FF21C7
:10073000DB075CBF3246FF21FFF718FD0028F1D030
:1007400015B12379DB07E7D4002FECD023793B7078
:1007500003B0F0BD8268417C02F0010C90F91000FA
:10076000FF22CDE9006CF4F7AFF8E7E770B5044677
:10077000051D82B020680379012B16D0022B02D010
:10078000002002B070BD83682A46FF21DE075CBFEF
:100790002A46FF21FFF7EAFC0028F1D02379DB0786
:1007A000EFD520680379012BE8D18668FF22417CD0
:1007B00006F0010690F91000CDE90056F4F784F830
:1007C000EAE700BF024630B5044652F8040B83B096
:1007D0000379012B0ED0022B01D0002008E0FF216D
:1007E000FFF7C4FC0028F8D02079C04300F00100D6
:1007F00003B030BD8568417C05F0010590F910001B
:100800000092FF220195F4F75FF8EBE770B5B42290
:1008100082B00446FF210068FEF72CFB10B90020CF
:1008200002B070BD2068251D0379012B13D0022B67
:10083000F5D183682A46FF21DE075CBF2A46FF21E7
:10084000FFF794FC0028EAD02379DB07E8D520687D
:100850000379012BEBD18668FF22417C06F001066B
:1008600090F91000CDE90056F4F72EF8EAE700BF42
:1008700070B50A4682B00446A5210068FEF7FAFA70
:1008800010B9002002B070BD2068251D0379012B2E
:1008900013D0022BF5D183682A46FF21DE075CBF07
:1008A0002A46FF21FFF762FC0028EAD02379DB0704
:1008B000E8D520680379012BEBD18668FF22417CC3
:1008C00006F0010690F91000CDE90056F3F7FCFFA1
:1008D000EAE700BF70B582B00446CDE90023FFF718
:1008E00095FF10B9002002B070BD5522A5212068E7
:1008F000FEF7C0FA0028F5D0251D2A46FF21206802
:10090000FFF78EFC0028EDD02379DB07F5D40DF13D
:10091000FF350DF1070615F8011F2046FFF7A8FF68
:100920000028DFD0B542F6D1DDE700BF002A34D081
:10093000F0B5044683B00E46051D8F1816F8012B3E
:10094000A5212068FEF796FA90B9002003B0F0BD0B
:100950008268417C02F0010C90F91000FF22CDE981
:10096000005CF3F7B1FF0028EFD02379DB070FD548
:1009700020680379012BEBD0022BE6D183682A464D
:10098000FF21DB075CBF2A46FF21FFF7EFFBEAE709
:10099000B742D3D1012003B0F0BD0120704700BFA2
:1009A000F0B5962283B00E460446FF210068FEF79C
:1009B00061FA10B9002003B0F0BD251D206803794D
:1009C000012B1DD0022BF5D183682A46FF21DF07BA
:1009D0005CBF2A46FF21FFF7C9FB0028EAD0237934
:1009E000DB07EBD4E12220681146FEF743FA00282A
:1009F000E0D03246FF21206803B0BDE8F0400FE4AC
:100A00008768FF22417C07F0010790F91000CDE9CB
:100A10000057F3F759FFE0E7002A42D0F0B504464B
:100A200083B00E46051D8F189622FF212068FEF721
:100A300021FA90B9002003B0F0BD8268417C02F039
:100A4000010C90F91000FF22CDE9005CF3F73CFFA8
:100A50000028EFD02379DB070FD520680379012B1D
:100A6000EBD0022BE6D183682A46FF21DB075CBF6F
:100A70002A46FF21FFF77AFBEAE7E12220681146C8
:100A8000FEF7F8F90028D5D03246FF212068FFF79D
:100A9000C7FB0028CED00136B742C5D1012003B034
:100AA000F0BD0120704700BFF0B50B460546164665
:100AB000044683B087211A4655F8040BFEF7DAF98D
:100AC00020680379012B19D0022B02D0002003B03B
:100AD000F0BD83682A46FF21DF075CBF2A46FF215D
:100AE000FFF744FB0028F1D02379DA07E8D4002E81
:100AF000EDD0C3F34013337003B0F0BD8768FF221D
:100B0000417C07F0010790F91000CDE90057F3F799
:100B1000DBFEE7E7F0B5782183B0164604460022F5
:100B20000068FEF7A7F910B9002003B0F0BD251D3D
:100B300020680379012B13D0022BF5D183682A4654
:100B4000FF21DF075CBF2A46FF21FFF70FFB0028CC
:100B5000EAD02379DA07EBD45B09337003B0F0BD38
:100B60008768FF22417C07F0010790F91000CDE96A
:100B70000057F3F7A9FEEAE770B5CC2282B004462D
:100B8000A5210068FEF776F910B9002002B070BD0B
:100B90002068251D0379012B13D0022BF5D1836822
:100BA0002A46FF21DE075CBF2A46FF21FFF7DEFA57
:100BB0000028EAD02379DB07E8D520680379012BE8
:100BC000EBD18668FF22417C06F0010690F9100007
:100BD000CDE90056F3F778FEEAE700BF70B5B4221E
:100BE00082B00446FF210068FEF744F910B90020E6
:100BF00002B070BD251D20680379012B21D0022B86
:100C0000F5D183682A46FF21DE075CBF2A46FF2113
:100C1000FFF7ACFA0028EAD02379DA07EBD4CC212D
:100C20002046FFF725FE0028E1D002E02379DB070C
:100C3000DED52A46FF212068FFF7F2FA0028F5D119
:100C4000D5E78668FF22417C06F0010690F9100086
:100C5000CDE90056F3F738FEDCE700BF2DE9F04F91
:100C600082468DB0002090460AF104070891069054
:100C70000A930790069B5046DC0008EBC3030593DC
:100C8000FFF7C4FD28B941E09AF8043013F00102DF
:100C900008D03A46FF21DAF80000FFF7C1FA002831
:100CA000F2D133E003929A070B9040F1CC80F0210F
:100CB0005046FFF7DDFD48B3083CDDF80C9008EB2B
:100CC0000403012409932546089B003B18BF012318
:100CD0000493049B082D8CBF002303F001039B4663
:100CE000002B5DD06E1E089B43FA06F606F0010647
:100CF000F2017821DAF80000FEF7BCF830B1DAF83A
:100D000000000379012B3FD0022B07D000220A9B61
:100D10001046069919700DB0BDE8F08F83683A4609
:100D2000FF21DB075CBF3A46FF21FFF71FFA0028CF
:100D3000ECD09AF8043013F00102E0D199094FEA9F
:100D4000531E4FEAD31C01EA5313DB074BD466450D
:100D500002D0BBF1000F73D1BCF1000F2DD005996B
:100D600011F80930234301F809306400013514F00B
:100D7000FF04EDB2ADD109F101095FFA89F9B9F1CA
:100D8000080F30D00124A4E78268417C02F0010CF6
:100D900090F91000FF22CDE9007CF3F795FDC6E73E
:100DA000069BD3B1079BAB4217D9099B13F80930B7
:100DB0001C4214BF012600269AE74EEA0101039B5C
:100DC00011F0010F059908BF2B46039311F8093064
:100DD00023EA040301F80930C7E7079B5E1BB6FA54
:100DE00086F6760984E7402D07D80A9B069A1B7879
:100DF00093423FF63FAF024689E7059BDD795C1ED3
:100E00009E1D14F801CF082182EA0C0301394FEA34
:100E10005C0C43F3000311F0FF0123F0730383EA3A
:100E20005202D2B2F0D1A642EBD19542DDD1069B5F
:100E30000133DBB20693039B002BDCD00793D4E78E
:100E40000B9E324663E70646324660E710B504461D
:100E5000006882B003796A46022B4FF006030CBF8C
:100E600043210321FEF7AEFD68B1BDF80010BDF8C7
:100E70000220BDF8043049BA52BA5BBAE1866287F3
:100E8000238702B010BDC4F83600608702B010BDE1
:100E900030B5002385B004460221C0F836300DF18C
:100EA000070243870068FFF7BBF918B19DF80730C8
:100EB000DB0703D40025284605B030BD062302AA6F
:100EC00003212068FEF77EFD0DF10702092120684D
:100ED000FFF7A6F905460028ECD09DF8073013F07F
:100EE0000C0FE7D1BDF80820BDF80C30BDF80A1092
:100EF000C2EB8232C3EB8333206889009B009200EF
:100F0000218763870A21E2860122FDF7B3FF284685
:100F100005B030BD10B50446002221210068FDF760
:100F2000A9FFFC2220212068FDF7A4FF40222421F4
:100F30002068FDF79FFF0C2223212068FDF79AFF10
:100F4000002222212068FDF795FF012010BD00BF7F
:100F500010B5044694220B210068FDF78BFF712227
:100F600001212068FDF786FF002204212068FDF79B
:100F700081FFC82205212068FDF77CFF00220621A1
:100F80002068FDF777FFC82207212068FDF772FF70
:100F9000002208212068FDF76DFFC8220921206882
:100FA000FDF768FF012010BD01207047044B0022AF
:100FB000002101201A605A609A60D960704700BF12
:100FC00060D90024104B11491A680346C868121AE8
:100FD000FA2A16D8D1ED006A012091ED017AFDEED2
:100FE000E66AD1ED027ABDEEC77AFDEEE77A16EE3B
:100FF000902ADA8617EE102A1A8717EE902A5A8757
:1010000070470020704700BFC43B002460D9002413
:101010000E4B70B51B7C82B00191ABB90C4B1D68B7
:1010200095B12B681A687AB19B686BB10446284663
:10103000984748B1019922462E6828460B463168E8
:1010400002B0BDE87040084702B070BD60D900240E
:10105000E0AA00240B4B70B51E688EB133681A6885
:1010600072B19B6863B1054630460C46984738B16B
:1010700031682A46234630460968BDE87040084773
:1010800070BD00BFF8AA0024014B5B695B6818477C
:1010900060D90024024B08305B699B68184700BF89
:1010A00060D900240120704701207047012070475B
:1010B000012070470120704731B10B4BD3ED067A08
:1010C000F8EEE77AC1ED007A6AB10749074BC969C2
:1010D000DFED076A0B4407EE903AF8EEE77A87EE09
:1010E000A67A82ED007A704760D900244D95FFFF03
:1010F0000000C84201207047012070477A4A01462B
:1011000000239446104610B490F904400C30012C92
:101110004DD00133082BF7D1734C002394F9040010
:101120000C34022858D00133082BF7D16E4C002321
:1011300094F904000C3403286BD00133082BF7D149
:10114000694C002394F904000C34052877D001334E
:10115000082BF7D1644C002394F904000C340628C2
:1011600000F083800133082BF6D1002392F90400AC
:101170000C32072800F093800133082BF6D15B4B2B
:101180001B68DC0340F1A180594B086803F58C749F
:1011900003E01433A34200F098801A689042F8D11B
:1011A000DA68D201F5D501205DF8044B704703EBF6
:1011B00043035CF8233023B34E480B7990F8D140B9
:1011C00090F8D000984218BF9C420CBF012000202C
:1011D000A2D15DF8044B704703EB43035CF8233066
:1011E0008BB145480B7990F8D04090F8D1009842E7
:1011F00018BF9C420CBF0120002097D15DF8044B22
:101200007047394C8AE7384C94F904000C340328B1
:1012100093D103EB43035CF82330002B3BD03748DA
:101220000B7990F8D04090F8D100984218BF9C42BA
:101230000CBF0120002083D15DF8044B704703EB05
:1012400043035CF8233043B32D480B7990F8D0402A
:1012500090F8D100984218BF9C420CBF012000209A
:101260007FF478AF5DF8044B704703EB43035CF801
:101270002330002B3FF47AAF22480B7990F8D0400E
:1012800090F8D100984218BF9C420CBF012000206A
:101290008AD003466AE7144C54E7134C5CE703EB2F
:1012A00043035CF82330002B3FF469AF164A0B79F7
:1012B00092F8D10092F8D0209A4218BF98420CBF01
:1012C000012000207FF45BAF6EE70B79312B04D84F
:1012D0002F2B94BF0020012066E7343B012B8CBFED
:1012E0000020012060E700BFB48A0024E4700024DD
:1012F00068050024A8090024800C0024580F00244D
:101300003012002408150024E01700240B4B8446FB
:10131000002010B503F58C7E02E014339E450BD0FF
:101320001A686245F9D1DA68441C8A42F5D0D9605E
:101330001433E0B29E45F3D110BD00BF6805002410
:10134000704700BF40F2FF72034B914203EBC003B2
:10135000A8BF11469984704760D90024112807D886
:10136000044B03EB8003D3F880300BB19B6819600A
:1013700027F0E2BB60D90024112807D8044B03EB07
:101380008003D3F880300BB19B681960704700BFB1
:1013900060D90024F0B5484D83B095F8C8303BB112
:1013A00095F8C9600446012E38D0022E54D00EB1F3
:1013B00003B0F0BD012280210068FDF75BFD012232
:1013C000FF212068FDF756FD324631462068FDF7C3
:1013D00051FD95F8CA2091212068FDF74BFD31465B
:1013E00001222068FDF746FD3246FF212068FDF707
:1013F00041FD324680212068FDF73CFD3146012247
:101400002068FDF737FD2D4B2D4901221B68087020
:1014100085F8C920C5F8CC3003B0F0BD01AA002181
:101420000068FEF7FDFE9DF80430254FDA0738709E
:1014300039D5D5F8D030002BBAD0204AD5F8CC1009
:10144000126892B2521A9342B2D24FF0FF32002386
:101450007A6085F8C930ABE701AA13210068FEF76E
:10146000DFFE9DF80430164F5B073870E1D033463D
:1014700001AA1E212068FEF7A5FABDF804302068F5
:1014800001225CBA0B21FDF7F5FC0E4BA4B2012240
:101490003870A3FB0434002385F8D420E40885F8D1
:1014A000C9307C6084E7054B02221B6885F8C9209F
:1014B000C5F8CC307CE700BF60D90024C43B0024D1
:1014C00014270024CDCCCCCC0C4A13787BB10C4B28
:1014D00093F8C81059B193F8D41059B1506800224C
:1014E000FA2883F8D420A8BF4FF0FF3070476FF080
:1014F000010070476FF00200704700BF14270024FE
:1015000060D900242DE9F041104C00251746022334
:1015100004F1D80884F8D910FF210646424684F821
:10152000D850FEF7CDF968B1424630460223FF217C
:10153000FEF748FA30B1B4F8D83028465BBA3B80A1
:10154000BDE8F0816FF00C00FAE700BF60D900241D
:101550000B4B93F8D82182B193F8D92152B10949A4
:101560000022886883F8D921B0F5967FA8BF4FF094
:10157000FF3070476FF0020070476FF00100704756
:1015800060D9002414270024024BD3F8DC315B68B7
:10159000184700BF60D90024024BD3F8DC319B68A8
:1015A000184700BF60D90024024BD3F8DC31DB6858
:1015B000184700BF60D90024014BD868704700BFAE
:1015C00014270024044B93F8E03113B1034B18693E
:1015D00070476FF00100704760D900241427002481
:1015E00070B52F4C05460323002104F5F272006804
:1015F000FEF7E8F958B96FF00103C4F8E831294A59
:10160000D4F8EC31116832338B423FD370BDB4F85B
:10161000E421F2EE046A94F8E6C1082152BA94F883
:10162000E43192B207EE902AF8EEE77A87EEA67AD6
:10163000BDEEC77A84ED7A7A58B25B00420000288A
:10164000DBB282F00702B8BFD3B20139F4D194F80B
:10165000E5210821534058B25B0042000028DBB26C
:1016600082F00702B8BFD3B20139F4D19C45C6D18C
:10167000D4F8E8312BB1D4F8E8214FF6FF739A4241
:10168000BDD14FF0FF33C4F8E831B8E7C4F8EC112E
:10169000012328683121044ABDE87040FEF710B9E3
:1016A00060D90024C43B002450DB0024014BD3F854
:1016B000E801704760D90024437A5A1C0344D2B22F
:1016C00042729972037A934200D802B97047036854
:1016D00000F10A0110B50446406898470023637280
:1016E00010BD00BF026830B5137985B00446012BE8
:1016F00061D0022B03D00025284605B030BD91688B
:1017000002AD1046C9072A464CBF19468221FEF792
:101710002DFD0028EFD09DF80830DA07EBD52A46DA
:10172000072303212068FEF74DF905460028E2D083
:1017300011220A212068FDF79DFB9DF80E301B0742
:10174000D9D42A49BDF80830B1F8F02113FB02F3CF
:10175000274A93423EDBB3F5000F39DA002BB8BFBE
:10176000FF331B125B421BB2BDF80A20E386B1F8BF
:10177000F23112FB03F31E4A93422FDBB3F5000F45
